:02000004620098
:1040000000B50E4B00F02CF80D4B00F029F80D4BCD
:1040100000F026F80C4B00F023F80C4B00F020F8D1
:104020000B4B00F01DF80B4B00F01AF80A4B00F098
:1040300017F80A4B00F014F801BC0047614B00620E
:10404000D14A0062CD4900627D4E00628D4B006214
:10405000DD410062794B00627D4500625D45006292
:104060001847C04670B50404144B240C00F09BF8AC
:10407000C0232404DB05E5181026114A114C124810
:104080001249134B148001801380124B148001805D
:104090002B802A88298840231A400B409A42F8D165
:1040A000731E1B041E0C80235B01ED18002EE4D14F
:1040B000094B00F078F870BC01BC0047614B00620E
:1040C000AAAA0060AAAAFFFF545500605555000037
:1040D0008080FFFF30300000794B006210B50C1C6F
:1040E000094B0A490A4A0B800A4B1A800A4B0B807B
:1040F00020802288218840231A400B409A42F8D120
:1041000010BC01BC00470000AAAAFFFFAAAA0060D9
:104110005555000054550060A0A0FFFF10B5041CC9
:104120000906080EE30705D5013C22780302101C9E
:10413000184304E02288FF231B021A401043211C6D
:10414000FFF7CCFF10BC01BC00470000F0B5120423
:104150000127061C0D1C140C394208D00178281CBC
:10416000FFF7DCFF631E1B04013501361C0C3C42CB
:1041700006D0631E1B041C0C2819A15DFFF7CEFF9F
:10418000002709E0737830781B02291C1843FFF7D9
:10419000A5FF0236023502373B041B0CA342F1D3C4
:1041A000F0BC01BC00471847002103E0084B013177
:1041B00099420AD0074B1A6816231A42F6D1064BC9
:1041C0001B68002B01D1002000E001207047000097
:1041D00072110100000010401400104030B5134B64
:1041E00000F0BAF91248134B0022134D012102606E
:1041F00049421A60114C0833296019600833226063
:104200001A60802302685B041A430D4B026023602E
:104210002960802302681B061A430260FFF7C4FF6F
:10422000084B00F099F930BC01BC0047614B0062BB
:104230000000104004001040080010401000104022
:10424000B0DF1000794B006210B5C022120623497E
:1042500083188B4201D801203CE0214C03198B428A
:1042600001D8022036E01F4A83188B4201D804206F
:1042700030E01D4C03198B4201D808202AE01B4B6B
:10428000C2181B4B9A4201D8102023E0194C1A4A3D
:104290000319934201D820201CE0184C03199342C3
:1042A00001D8402016E0164BC218164B9A4201D88E
:1042B00080200FE0144C03198B4202D8802040026A
:1042C00008E0124BC218124B9A4202D8802080029A
:1042D00000E0002010BC02BC08470000FF1F0000E7
:1042E00000E0FFBF00C0FFBF00A0FFBF0080FFBF16
:1042F000FF7F00000000FFBFFFFF00000000FEBFC7
:104300000000FDBFFEFF00000000F4BF00E0F3BFAF
:10431000FE1F000030B5154B051C994223D1C02368
:104320001B06C218124B9A421DD8124B00F014F90A
:10433000114B00221A60114C802322681B051A437E
:104340002260281CFFF780FF0D4B18608023226835
:104350001B061A432260094B1A6816231A42FAD127
:10436000084B00F0F9F830BC01BC0047AFEC00008E
:10437000FFFF0300614B006214001040000010407A
:1043800004001040794B006230B5274B00060D1C2D
:10439000040E9A4245D1C0231B06CA18234B9A42E9
:1043A0003FD8234B00F0D8F803222B1C9343186806
:1043B0002B1C1340012B0AD0012B04D3022B0BD052
:1043C000032B14D10DE0FF23984320430FE0194B3A
:1043D000021C1A40230208E0174B021C1A40230457
:1043E00003E0164B021C1A402306101C1843144B02
:1043F00000221A60134980230A689B051A43124B56
:104400000A602A1C1A40114B1A60083B186080236E
:104410000A681B061A430A60FFF7C6FE0C4B00F041
:104420009BF830BC01BC0047AFEC0000FFFF03006D
:10443000614B0062FF00FFFFFFFF00FFFFFFFF0077
:104440001400104000001040FCFF1F00100010403E
:10445000794B0062F0B51204140C0D1C82B0061CDE
:10446000191C002C61D0334B99425ED1324B9D42D6
:104470005BD9324B2A199A4257D8271C0DE06A1C87
:1044800030780192291C2B4AFFF77EFF7B1E1B040C
:104490001F0C0136002F48D0019D03231D42EED191
:1044A000274B00F059F8032F26D9737831781B0277
:1044B0001943B3781B041943F3781B061943214BA6
:1044C00000221A602048802302689B051A431F4B74
:1044D00002602A1C1A401E4B1A60083B1960802398
:1044E00002681B061A430260FFF75EFE3B1F1B04B7
:1044F000043604351F0CD6E7164B00F02DF80023C8
:1045000000930CE03078291C0A4AFFF73DFF009B1E
:10451000013B1B041B0C6C1C00930136251C7B42C9
:104520001B04009A1B0C9A42ECD102B0F0BC01BCF7
:1045300000470000AFEC0000FFFFFF3FFFFF03401C
:10454000614B00621400104000001040FCFF1F008F
:1045500010001040794B00621847C046A022120696
:10456000136804490B43136003490B680222134389
:104570000B60704708080000200000A0F0B5C74B92
:1045800000221A60C64B01218DB01A6049423020CA
:10459000C44B00F0C9F9FA204000C34B00F0C4F945
:1045A000C24B00F0C1F900210791089105E01222E9
:1045B000012301270792089365E000270697BC4B6B
:1045C00000F0B2F9002826D0FA2292000026131C2F
:1045D0007F211420B74C009600F0A7F94B20B64D70
:1045E00000F0A4F9FA218900B44A0520B44B0096E2
:1045F00000F09BF9B34B00F097F9322000F096F9E8
:10460000A02212061368B0490B431360AF490B6830
:10461000022213430B60AE4B002000F085F900042A
:10462000000C03041A14002AC9DB0899642900DD70
:104630002FE1012F0FD0022F31D0002F00D028E121
:10464000102A04D1069A01235A400692B7E7069B26
:10465000002BB4D01AE007990306180E41400791C9
:10466000102A0AD1069B7B400693002BA7D10899FC
:10467000984BCA5401310891A1E7069B002B08D042
:10468000032A03D102270021069198E7022A94D138
:104690008DE7089A8F4BD054013208928FE71B02A6
:1046A00007991B0E994200D0EDE008AA894D1278B7
:1046B0007E4B2A7000F038F9012149423020794BB5
:1046C00000F032F9FA20784B400000F02DF96978BB
:1046D0002B7844297BD1032B00D8D4E0AB784C2B2A
:1046E00000D0D0E0EB78542B00D0CCE02C79032C18
:1046F00016D0032C03D8012C00D0C4E005E0042C14
:1047000036D0072C00D0BEE058E0734B687900F03B
:104710000BF96B79002B00D0B3E0614B1C60B0E06B
:1047200006206E4B00F000F96549644BFA229200B6
:1047300000910391002101920293049105207F21B1
:104740005C4C00F0F2F832205B4C00F0EEF85D4B70
:1047500000F0EAF8322000F0E8F8A0221206136810
:1047600059490B431360594A13683B43136088E06F
:104770005B4B5C681B6809930A9400230C9368796F
:10478000592803D8FA21C900431801E0554A831873
:104790000993504A937909A84371D3790371137A25
:1047A0000CAC2370537A6370937AA3704E4B00F075
:1047B000BBF8201C4D4B00F0B7F862E0384B1B688B
:1047C000012B5ED1C0214A48C905042213E00BAA7F
:1047D000D170053B1B041E0CAB789370EB785370C3
:1047E0002B7913700B99A0231B06CA18414B9A42D0
:1047F00005D8681D321C404B00F096F841E03F4B55
:10480000994231D93E4B8A199A422DD8081C3D490C
:10481000059100F087F8214C2368071C034207D15B
:10482000394B0B98394900F07FF823683B432360EC
:104830000B9880190138059A00F075F82368071C59
:10484000034209D10B9880192F4B01382F4900F0F2
:104850006BF823683B4323600B99681D321C2B4B7C
:104860002B4C00F062F80CE02A4B99420BD92A4BF2
:104870008A199A4207D8081C321C2849284B00F094
:1048800053F8062000E01520144B00F04DF80027E7
:1048900095E60DB0F0BC01BC00470000749B0062BF
:1048A000709B0062054F0062254A0062C54C0062A1
:1048B000314A0062F94F006231490062C4090000C8
:1048C000AC0D0000DD4B006208080000200000A0D5
:1048D000B14C0062789B0062654000625D4C0062F2
:1048E000B89800626C07000071540062D9530062EE
:1048F000B0980062FFFF3F004D410062FFFFFF3FA5
:10490000FFFF03404942006215430062AFEC000024
:1049100055440062FFFFFF61000010627D9B006252
:10492000F556006208471047184720472847C046F9
:10493000034B18601A1C1368002BFCD17047000051
:10494000349C0062044A054B1380054B1380054BD1
:10495000012252421A80704718E000E05AA5FFFF7A
:10496000A55A000008E000E010B50C4A1368834225
:1049700010D00B4B04329A42F8D1503A0021141C4B
:104980001368002B02D18B00185103E0013104326F
:104990001429F5D110BC01BC00470000DC9B00626B
:1049A0002C9C006210B5084900220C1C0B68834245
:1049B00003D192000023135103E001320431142A81
:1049C000F4D110BC01BC0047DC9B006200B50E4A6C
:1049D000111C5031002308C28A42FBD10B4A0C4BF8
:1049E0001A800C4A043B1A800B4A0C3B1A800422A2
:1049F000524208331A800020084A0121084B00F077
:104A000064F801BC00470000DC9B00621740000016
:104A1000189000E04080FFFF88130000454A0062C4
:104A20002D4B0062014B186070470000309C006203
:104A3000034B1B680020002B00D1012070470000B1
:104A4000309C006210B5164A164B1380164B13802B
:104A5000164B012252421A80154A1368002B02D0CD
:104A60001368013B1360134A1368002B02D01368CC
:104A7000013B1360104C2268002A03D00F4B1A60D0
:104A800000F022F80E4B04349C42F4D10D4B00226E
:104A90001A80042252420C3B1A8010BC01BC004711
:104AA00018E000E05AA5FFFFA55A000008E000E06A
:104AB000349C0062309C0062DC9B0062CCBF0062D0
:104AC0002C9C00621C9000E01047184770470000C3
:104AD00010B5104B00211960203319600E4A0123D4
:104AE0005B4213600D4B0C221A60143B19601033AB
:104AF00019600B4A0B480C4C8B04136001311319DD
:104B0000186004322029F6D1024B01221A6010BC31
:104B100001BC004700F8FFFF40F8FFFF1CF8FFFF53
:104B200060F8FFFFCD4A0062DC07000030B50004EA
:104B3000000C8400E263084D01232A6883401A4375
:104B4000064BE4180F231940800408432A602060B4
:104B500030BC01BC0047000020F8FFFF60F8FFFFF9
:104B60000349044B0A681A6000230B607047000079
:104B700020F8FFFF389C0062024B1A68024B1A6053
:104B800070470000389C006220F8FFFF00B50D4B15
:104B90001A880F230C490D48134201D0002300E06E
:104BA00009230B6000F0A4F8094B00F0A2F8094BB0
:104BB00000F09FF830200021074B00F09AF801BC6C
:104BC00000470000408800C0A8990062F54C0062D0
:104BD0009C990062485A0062054F006210B50A4C69
:104BE0002368092B09D1C020084B00F082F8084B3C
:104BF00000F07FF80023236002E0064B00F079F814
:104C000010BC01BC00470000A8990062305C006243
:104C1000585B0062554E006200B5090681B0090E6E
:104C200009280ED1684603300170094B012100F0BC
:104C300060F8002809DB074B00F05BF8430704D459
:104C4000F9E7081C044B00F054F801B001BC004720
:104C5000985B0062785C0062614D006200B5044BB5
:104C60000106090E1868FFF7D7FF01BC00470000D6
:104C7000A899006210B581B009280DD16C460334A3
:104C8000201C0121084B00F034F8002802DC012030
:104C9000404205E0207803E0081C044B00F029F8AE
:104CA00001B010BC02BC0847E45B0062814D0062A9
:104CB00000B5034B011C1868FFF7DCFF02BC084776
:104CC000A899006200B5074B1B68092B04D140204E
:104CD000054B00F00EF802E0044B00F00AF801BCAE
:104CE00000470000A8990062305C00623D4D006200
:104CF0000047184700B5094A0023538053881B0416
:104D00001B0C13800920064A0D21064B00F0B4F855
:104D10000548064B00F0B0F801BC0047409C00621B
:104D2000FD4D00622D4B0062DD4D0062694900625D
:104D300000B5FFF7DFFF01BC00470000064A002175
:104D4000518053881B041B0C1380044B19800433BF
:104D500019801C3B1B887047409C0062204000C0AB
:104D60000006054B000E1880044B1A8880239B0018
:104D70001342F9D170470000044000C0144000C045
:104D80000004134B000C188012490A884B88120447
:104D90001B04934207D10E4B1B881B04002BF3D13D
:104DA0000120404212E04A881204120C53180132CA
:104DB00012041B79120C4A801B06180E4B88064AF7
:104DC0001B041B0C934201D100234B807047000051
:104DD0003C9C0062409C0062EE020000054A138881
:104DE0001B04002B05D0138803491B045B181B0C04
:104DF000138070473C9C00620000FFFF10B5114B10
:104E00001B68DA071BD5104B1B881B041A0C802368
:104E10009B00141C1C4012D10C4803881B041B0C63
:104E20001918013312061B04120E1B0C0A710380A1
:104E30000388074A1B041B0C934200D1048010BC5A
:104E400001BC0047144000C0084000C0409C006204
:104E5000EE020000064A0021518053881B041B0CFF
:104E60001380044B1980043319801C3B1B88704746
:104E7000409C0062204000C01847C04600B516485C
:104E8000164B00F0F1F9164B002018801B88154ACC
:104E90001B041B0C13801388134A1B041B0C138068
:104EA0001388124A1B041B0C1380114A114B1188E2
:104EB0000B401380104B11880B4013800F4B0422C2
:104EC00052421A80052208331A80043B50221A806D
:104ED0000B4B188001BC00476950006269490062B1
:104EE0006A9F00626C9F00626E9F0062709F00620A
:104EF0000C5000E0FF7F0000FFBF000010C000E08A
:104F0000689F006210B5041C081C002924D1E30727
:104F100006D53149314B0A8813400B80304B18803D
:104F2000A30706D52C492F4B0A8813400B802E4B24
:104F30001880E30606D52849284B0A8813400B80C1
:104F40002A4B1880A30643D52349264B0A881340D1
:104F50000B80274B18803BE0E3070CD51E490B88DC
:104F6000244A1B041B0C13431B041B0C0B801C4A00
:104F700003041B0C1380A3070DD517490B8880224F
:104F80001B04D2011B0C13431B041B0C0B80164A81
:104F900003041B0C1380E3060BD50F490B88154A3D
:104FA0001B041B0C13431B041B0C104A0B80142303
:104FB0001380A3060CD508490B8880221B04D2015C
:104FC0001B0C13431B041B0C094A0B801423138076
:104FD00010BC01BC004700000C5000E0FF7F000047
:104FE000709F0062FFBF00006E9F00626C9F0062B6
:104FF0006A9F00620080FFFF0EB470B581B0059D0E
:10500000061C002D20D006AB0024009304E0114ABA
:10501000A300985001340B1C1868191D002801D0FA
:105020000A2CF4D10B4AA3000091002199500A4A9E
:1050300033061B0E1370094A2B061B0E1370084B08
:10504000084A19600123138001B070BC08BC03B08A
:1050500018470000349F0062609F0062619F0062F9
:10506000649F0062689F006200B569490B88694AC5
:105070001B041B0C934211D00B88674A1B049B181E
:105080001B0C0B800B881B04180C002806D16349ED
:10509000634B0A8813400B80624B188062490B886F
:1050A0005C4A1B041B0C934211D00B885A4A1B0408
:1050B0009B181B0C0B800B881B04180C002806D1B6
:1050C00056495A4B0A8813400B80594B188058494F
:1050D0000B881B04002B1BD00B884F4A1B049B180A
:1050E0001B0C0B800B881B04002B11D14B4880221A
:1050F0000388D2011A4204D003884C4A1A40028025
:1051000004E003881B041B0C1343038014230B804F
:1051100044490B881B04002B1DD00B883E4A1B04FE
:105120009B181B0C0B800B881B04002B13D13B48D6
:1051300003881B04002B04DA0388394A1A400280D2
:1051400007E003883B4A1B041B0C13431B041B0C86
:10515000038014230B80384A13881B04002B55D07E
:1051600013882D491B045B181B0C138013881B0428
:10517000002B4BD13148036831499A005158013313
:10518000036000290AD12F4B042252421A800522C3
:1051900008331A805022043B1A8037E0012909D1D4
:1051A000284B042252421A80052208331A805022CA
:1051B000043B24E0244B09041B78090C234B2448AE
:1051C00000F052F81F4B0422011C52421A8005398C
:1051D000052208331A8088001E4A0B0440181B0C55
:1051E00013808300C0187D301B4B642100F03CF815
:1051F00005381A4B0004000C194A18800C331A8029
:10520000184B1B780C4A1B061B0E138001BC004771
:10521000709F0062FFFF00000000FFFF0C5000E0E5
:10522000FF7F00006C9F00626E9F0062FFBF000066
:105230006A9F00620080FFFF689F0062649F0062B7
:10524000349F006210C000E0619F0062E957006275
:10525000804F12000CC000E05D57006208C000E003
:105260005082FFFF609F00621847C0460B490A88C2
:1052700020231342FAD00B881B0410221B0C13436B
:105280001B041B0C0B80064B00221A80054A0433BA
:105290001A80054B0A8813400B80704704D000E049
:1052A00008D000E00080FFFFEFFF0000FA21890036
:1052B0000A4B1A882023134209D0094B1A88043359
:1052C0001B8812041B041B0C101C184304E001393A
:1052D0000029EDD1012040427047000004D000E0D9
:1052E00018D000E030B5041C0D1CFFF7DFFF431C95
:1052F00002D10120404205E0211C2A1C034B00F092
:10530000E8F8002030BC02BC084700009555006258
:1053100030B5041C0D1CFFF7C9FF013002D101207C
:1053200040422CE0201C291C164B00F0D2F81649F4
:105330000A8820231342FAD00B881B041B0C10226E
:1053400013431B041B0C0B800F4B1A8820231342A2
:10535000FAD003040D4A1B0C13800B4B1A88202330
:105360001342FAD00A4B020C1A8007490A882023FC
:105370001342FAD00A88074B13400B80002030BC40
:1053800002BC0847D554006204D000E01CD000E005
:1053900018D000E0EFFF000000B581B06946FFF7CC
:1053A000A1FF01B001BC004700B582B0011C6846F6
:1053B000FFF798FF02B001BC004700000378172BED
:1053C00007D843783B2B04D883783B2B01D80020A7
:1053D00001E001204042704730B582B0051CFFF764
:1053E000EDFF013002D10120404206E06846FFF7A0
:1053F000D3FF6846291CFFF78BFF02B030BC02BC0C
:105400000847000010B50468174AA318632B23D877
:105410000179002920D043791806030E0C2B1BD8E4
:1054200001220316101C9840104B184206D1A523E8
:105430001B01184205D1430706D40DE01F290ED9E0
:105440000AE01E290BD907E003231C4202D11D29C3
:1054500005D901E01C2902D90120404200E00020CA
:1054600010BC02BC0847000030F8FFFFAA1500007E
:1054700030B581B0051CFFF7C5FF013002D1012016
:10548000404206E06846FFF78FFF281C6946FFF799
:105490003FFF01B030BC02BC0847000030B5041C1F
:1054A0000D1CFFF7AFFF013009D0281CFFF786FF66
:1054B000013004D0201C291CFFF72AFF01E0012045
:1054C000404230BC02BC084700B5FFF70BFF01BCEF
:1054D00000471847F0B50768FC00E419E400E41938
:1054E000A30083B07E1EE418FB1C9B08244D019092
:1054F0000091301C6421E41800F0F8F8C821241A47
:105500004900301C00F0F2F8019A1E495279241823
:1055100065180292022A12D903231F420FD11A4E94
:10552000381C642100F0E3F8002806D1C821381C9B
:10553000490000F0DCF8002801D1144BE5181449AB
:10554000012202E008C90132ED18029B9A42F9DB00
:1055500001990B79EB180099013B1A01DB00D21875
:105560000B78D21813019B1A4A789B009B181801DC
:10557000C01A8B788000C01803B0F0BC02BC08478A
:105580005D5700625805F5FF8D5800625905F5FF1B
:10559000C4980062F0B588B04B4F049105903C214F
:1055A000161C00F0A5F8B070484D05983C2100F09D
:1055B0009DF83C21041C00F09BF83C217070201CDD
:1055C00000F094F8182100F093F8307040490598E5
:1055D00000F08CF83F4A86183F49301C00F088F8EC
:1055E0003E49041C00F082F83C490390201C00F066
:1055F0007FF83B49029000F07BF83A49041C00F028
:1056000075F838490190201C00F072F801300790BD
:105610003149301C00F06AF884002418039AA30072
:10562000E41864235343240102982D49E41800F040
:105630005DF8019A80002418A318049A1360039A55
:10564000042A02D0019A042A04D1049A0C2353712B
:105650001F2333E0049A0133136000235371079B27
:10566000214A0693009220E0009AAB009B185B68E9
:10567000069AD61A012D12D1049B1C6803231C42E2
:105680000DD1201C642100F033F8002806D1C82178
:10569000201C490000F02CF8002800D1013E002E0B
:1056A00007DD049A6B1C53710696049B5D790A2DE5
:1056B000DAD9049A6B1C53716B461B7E08B01371C8
:1056C000F0BC01BC004700008D5800625D570062CD
:1056D000805101003AF90A00B13A0200AC8E000094
:1056E000B50500006D010000C098006228473047F2
:1056F0003847C04630B5051C8446141C101C0F2AC0
:1057000004D90A1C2A4303231A420ED0631E08D36D
:1057100062469B18581C0B7813700132013182428B
:10572000F9D1281C30BC02BC08472A1C0B68136046
:105730004B6853608B689360CB681038D36010312E
:1057400010320F28F2D8041C032805D908C90438E0
:1057500008C20328FAD8041C9446D7E7002934D09D
:105760000123002210B488422CD301242407A14233
:1057700004D2814202D209011B01F8E7E400A142F0
:1057800004D2814202D249005B00F8E7884201D38B
:10579000401A1A434C08A04202D3001B5C08224363
:1057A0008C08A04202D3001B9C082243CC08A042D4
:1057B00002D3001BDC082243002803D01B0901D0C0
:1057C0000909E3E7101C10BC704700B500F0C2F8EF
:1057D000002002BC0847000003B5FFF7BFFF0EBC66
:1057E0004243891A1847C046002941D010B4041C0E
:1057F0004C40A44601230022002900D5494200283C
:1058000000D5404288422CD301242407A14204D26F
:10581000814202D209011B01F8E7E400A14204D24F
:10582000814202D249005B00F8E7884201D3401A66
:105830001A434C08A04202D3001B5C0822438C0888
:10584000A04202D3001B9C082243CC08A04202D3F2
:10585000001BDC082243002803D01B0901D00909E2
:10586000E3E7101C6446002C00D5404210BC704792
:1058700000B500F06FF8002002BC084703B5FFF741
:10588000B3FF0EBC4243891A1847C04600295AD0BC
:105890000123884200D2704710B401242407A1429A
:1058A00004D2814202D209011B01F8E7E400A142BF
:1058B00004D2814202D249005B00F8E7002288420C
:1058C00000D3401A4C08A04205D3001B9C4601247B
:1058D000E3411A4363468C08A04205D3001B9C4653
:1058E0000224E3411A436346CC08A04205D3001BBF
:1058F0009C460324E3411A4363469C46002803D098
:105900001B0901D00909D9E70E242407224018D029
:1059100063460724234214D063460324E3411A421A
:1059200001D0CC08001963460224E3411A4201D099
:105930008C08001963460124E3411A4201D04C0847
:10594000001910BC704700B500F004F8002002BC3C
:105950000847C0467047C046F0402DE990609FE57B
:10596000B000D6E18C509FE58C309FE58C209FE500
:1059700000C0A0E3010010E284E09FE584709FE591
:1059800084109FE50040E0E300C083E500C082E5AD
:1059900000C0C5E50200000A0400A0E1F040BDE837
:1059A0001EFF2FE10230A0E31030CEE55CC09FE582
:1059B0005C309FE55C209FE500C083E558309FE5A3
:1059C00000E082E5007083E500C097E50FE0A0E10C
:1059D0001CFF2FE1004050E20130A0E33C009FE5B6
:1059E000ECFFFF1A0030C5E5B030C6E1A30F00EBB5
:1059F000E8FFFFEA829F0062789F0062D0BF0062EA
:105A0000749F0062DCBF0062909A0062FD980062A1
:105A10006C9A006200C0006204C00062D8BF0062DD
:105A2000945D006204E02DE514309FE5002093E5CD
:105A300044C092E50FE0A0E11CFF2FE104E09DE4EB
:105A40001EFF2FE1D8BF006230402DE9BCC09FE5AA
:105A5000BC409FE5BC309FE50050A0E300508CE5C2
:105A60000010A0E1005083E52420A0E30400A0E1A1
:105A7000850F00EBA0309FE5A0209FE5004083E567
:105A80009C309FE59C109FE5002083E598309FE5C2
:105A9000001083E5C90000EB90309FE58820A0E36B
:105AA000B020C3E188209FE501C0A0E384309FE5DA
:105AB00000C0C2E51120A0E3B020C3E178309FE52B
:105AC00078109FE578209FE5B050C3E174309FE5E2
:105AD000182081E5272BA0E3B020C3E11430A0E318
:105AE000BC31C1E160309FE560009FE5B0C0C3E11B
:105AF000620F00EB1A00A0E30E10A0E350209FE518
:105B0000640F00EB0500A0E13040BDE81EFF2FE16F
:105B1000D0BF0062DCBF0062749F006204C00062FC
:105B2000909A0062D8BF00626C9A006200C0006266
:105B3000ACBF0062789F0062AABF0062A8BF00628B
:105B4000249A0062FD98006250C00062829F006249
:105B5000945D0062845D006210402DE92C409FE559
:105B6000B030D4E1010013E30600000A20309FE5C5
:105B7000002093E504C092E50FE0A0E11CFF2FE1B7
:105B80000030A0E3B030C4E11040BDE81EFF2FE1BB
:105B9000829F0062D8BF006204E02DE538309FE5A7
:105BA000B020D3E10118A0E1010012E30030E0E3EE
:105BB0002118A0E10500000A20309FE5002093E5B0
:105BC0000CC092E50FE0A0E11CFF2FE10030A0E146
:105BD0000300A0E104E09DE41EFF2FE1829F00622C
:105BE000D8BF006204E02DE538309FE5B020D3E156
:105BF0000118A0E1010012E30030E0E32118A0E168
:105C00000500000A20309FE5002093E510C092E5D2
:105C10000FE0A0E11CFF2FE10030A0E10300A0E1B4
:105C200004E09DE41EFF2FE1829F0062D8BF006266
:105C300030402DE9C00010E3FF4000E230509FE506
:105C40000400A0E128509F050030951514C093155D
:105C50000FE0A0111CFF2F11003095E50400A0E11A
:105C600020C093E50FE0A0E11CFF2FE13040BDE82C
:105C70001EFF2FE1D8BF006230402DE944309FE580
:105C8000B020D3E1010012E33C509FE50000E0E3C7
:105C90000A00000A003095E518C093E50FE0A0E186
:105CA0001CFF2FE1003095E50040A0E11CC093E50A
:105CB0000FE0A0E11CFF2FE1FF4004E2040480E1BB
:105CC0003040BDE81EFF2FE1829F0062D8BF006216
:105CD000C13AA0E3FF3E83E2393183E2B010D3E161
:105CE0000A2AA0E3022082E2020051E138C09FE5C7
:105CF0000920A0130410A0E30F3002E2090053E3CF
:105D0000300083E20110419201104182373083E27A
:105D10000C00C1970C30C187000051E32222A0E1A2
:105D2000F4FFFFCA00009FE51EFF2FE17D9F006288
:105D3000650EA0E338C09FE50A0080E20420A0E3DE
:105D40000F3000E2090053E3301083E20120429259
:105D500001204282373083E20C10C2970C30C28798
:105D6000000052E32002A0E1F4FFFFCA00009FE51B
:105D70001EFF2FE1799F006200009FE51EFF2FE1CB
:105D8000F498006204E02DE53B0100EB04E09DE4A3
:105D90001EFF2FE110109FE5003091E5012043E246
:105DA000000053E3002081151EFF2FE1749F006265
:105DB00004309FE5000083E51EFF2FE1D0BF0062A5
:105DC00038309FE538209FE500C0A0E3002083E540
:105DD00030109FE530209FE50C00A0E104C083E572
:105DE00008C083E5003081E50CC083E5102083E521
:105DF00014C083E518C083E51CC083E51EFF2FE1B6
:105E000088BF006284AF006284BF0062849F00622A
:105E10001EFF2FE1F0452DE980A09FE500309AE5B7
:105E20000C4093E5000054E3006093E50070A0E1AE
:105E3000043093E5140000DA010054E10140A0A110
:105E4000038084E0010A58E30450A0E1015A63C2D0
:105E5000031086E00520A0E18B0E00EB050054E165
:105E6000050087E00610A0E1042065E0090000CAF3
:105E700000309AE5082AA0E1222AA0E1042083E567
:105E80000C1093E5011064E00C1083E50400A0E120
:105E9000F045BDE81EFF2FE17B0E00EBF3FFFFEAAC
:105EA00084BF006230402DE934509FE5003095E515
:105EB000102093E50140A0E10010A0E10200A0E164
:105EC0000420A0E1700E00EB002095E50030A0E377
:105ED0000400A0E11C4082E5143082E53040BDE8BA
:105EE0001EFF2FE184BF00620C309FE5002093E588
:105EF0000C0092E5010A60E21EFF2FE184BF006200
:105F000008309FE5002093E50C0092E51EFF2FE18D
:105F100084BF006208309FE5002093E51C0092E5F5
:105F20001EFF2FE184BF006214309FE5001093E54F
:105F30000020A0E30C2081E5042081E5082081E514
:105F40001EFF2FE184BF006218309FE5002093E51B
:105F50000030A0E3102082E20C3082E5043082E5BC
:105F6000083082E51EFF2FE184BF00620C309FE500
:105F7000002093E50C0092E5010A60E21EFF2FE18C
:105F800084BF006208309FE5002093E51C0092E585
:105F90001EFF2FE184BF0062F0412DE9007052E244
:105FA0000050A0E1130000DA50809FE5014081E23B
:105FB0000060A0E3020000EA060057E1014084E22D
:105FC0000C00000A013054E50030C5E5003098E5CA
:105FD000000053E3016086E2015085E2F5FFFF0A0D
:105FE000010054E50FE0A0E113FF2FE1060057E1A7
:105FF000014084E2F2FFFF1AF041BDE81EFF2FE1ED
:10600000D0BF006230402DE980309FE500C093E5AD
:106010001C209CE5000052E30040A0E10130A0E11B
:106020000050A0D30F0000DA14009CE510109CE58E
:106030001C209CE5030052E10250A0B10350A0A136
:10604000013085E2C3E0B0E1001081E00800001AF1
:1060500014309CE5033085E014308CE51C209CE571
:10606000022065E01C208CE50500A0E13040BDE881
:106070001EFF2FE10020A0E3012082E2B230D1E038
:1060800002005EE1043084E4FAFFFF1AEFFFFFEA4A
:1060900084BF006230402DE98C309FE500C093E55D
:1060A0001C209CE5000052E30030A0D3003080D5D6
:1060B00001E0A0E10200A0D3120000DA14109CE578
:1060C00010209CE51C309CE50E0053E10340A0B17C
:1060D0000E40A0A1013084E20050A0E3C3E0B0E193
:1060E000045080E4012082E00800001A14309CE58E
:1060F000033084E014308CE51C209CE5022064E031
:106100001C208CE5020084E23040BDE81EFF2FE138
:106110000510A0E1011081E2B230D2E00E0051E1A1
:10612000043080E4FAFFFF1AEFFFFFEA84BF006249
:10613000F04F2DE938319FE5002093E50C3092E5D2
:10614000013A63E2010053E10190A0E10080A0E187
:106150000090A0D33F0000DAC9A0A0E100005AE3FC
:10616000081092E5006092E5290000DA04B19FE58D
:106170000070A0E30B0000EA043AA0E1233AA0E19A
:10618000250CA0E10600C3E700209BE5000052E3D8
:10619000014083E21800001A041AA0E107005AE146
:1061A000211AA0E11A00000A043098E40358A0E183
:1061B0002508A0E10600C1E7B8209FE5003092E580
:1061C000000053E3017087E2FF0000E2014081E23A
:1061D000E8FFFF0A0FE0A0E113FF2FE1043AA0E17E
:1061E000233AA0E1250CA0E10600C3E700209BE5CF
:1061F000000052E3014083E2E6FFFF0A0FE0A0E166
:1062000012FF2FE1041AA0E107005AE1211AA0E1D0
:10621000E4FFFF1A010019E30800000A003098E5C6
:1062200050209FE50630C1E7002092E5000052E3D0
:10623000014081E20A00001A041AA0E1211AA0E13B
:106240002C309FE5002093E5081082E50C3092E5A4
:10625000033089E00C3082E50900A0E1F04FBDE891
:106260001EFF2FE10000D8E50FE0A0E112FF2FE1B3
:10627000F0FFFFEA84BF0062D0BF006270402DE9EA
:106280000341A0E3224B84E2443094E5D0509FE5E3
:106290000338A0E12338A0E1B030C5E1C4609FE538
:1062A000B030D5E1B020D6E1033002E0010B13E3BA
:1062B0002200001AB030D5E1033002E0010A13E3F6
:1062C0001700001AB030D5E1033002E0020B13E3EF
:1062D0000900000A90309FE50020D3E5000052E35A
:1062E0000C00000A230400EB0321A0E3F73CA0E329
:1062F000222B82E2FF3083E2443082E5B030D5E1E8
:10630000B020D6E1023003E0020913E32B0C001B9E
:106310007040BDE81EFF2FE10200A0E3360400EB51
:10632000F0FFFFEAEF3CA0E3FF3083E2443084E576
:106330000000A0E3300400EBB020D6E1E0FFFFEA6C
:10634000FB3CA0E3FF3083E220209FE5443084E55E
:1063500008C092E50FE0A0E11CFF2FE1B020D6E1DC
:10636000D3FFFFEAD4BF006250C00062EC9A006223
:10637000909A006270402DE90150A0E1FF4000E2D8
:106380008EFEFFEB000050E33A00001AECE09FE5C0
:10639000EC609FE5000054E37F20E0E30510E0E3BC
:1063A0003F30E0E30720CE050720C6050810CE05E4
:1063B0000810C6050800CE150730CE150800C61512
:1063C0000730C6150030D5E5020053E3B4309F8591
:1063D000B4109FE5AC309F950320A083AC409FE5AF
:1063E0001020C3850020A0931430A083BC31C1814C
:1063F0001020C395003094E5185081850050A0E32B
:106400001250C3E5BB0300EB002094E50730D6E54E
:106410001A00A0E31130C2E50E10A0E370209FE542
:106420001C0D00EB0E22A0E33E2B82E2003092E531
:10643000013083E3003082E50E12A0E3051A81E209
:10644000B030D1E1803083E3B030C1E1052AA0E370
:10645000CE2282E2B030D2E138109FE5803083E373
:10646000B030C2E1013CA0E3B030C1E128309FE58B
:10647000B050C3E10500A0E17040BDE81EFF2FE170
:10648000F09A0062339B00625E9B0062249A006275
:1064900004C00062845D0062ACBF0062AABF0062FB
:1064A00004E02DE5050AA0E3CE0280E2B010D0E1C1
:1064B000FF3CA0E37F3083E2031001E0B010C0E1B5
:1064C0000E22A0E33E2B82E2203092E50133C3E3AB
:1064D000203082E59A0300EB4CFEFFEB14309FE581
:1064E00014209FE50000A0E3B000C3E1B000C2E1CA
:1064F00004E09DE41EFF2FE1ACBF0062AABF006272
:1065000010402DE990309FE5002093E50040A0E386
:106510001340C2E51240C2E50400A0E1430400EBD1
:106520000400A0E1021CA0E35C0400EB0400A0E175
:106530002010A0E36A0400EB0400A0E12010A0E317
:10654000600500EB0400A0E16010A0E34E0500EB45
:106550000400A0E1B90400EB40309FE50400A0E195
:106560004C10D3E5A60500EB0400A0E1930400EB7A
:106570000400A0E1770800EB24309FE5012CA0E3A4
:10658000B020C3E11C209FE52030A0E30400A0E17F
:10659000B030C2E11040BDE81EFF2FE104C0006230
:1065A000909A0062ACBF0062AABF006270402DE901
:1065B000C0309FE5B020D3E10118A0E1800012E3D4
:1065C0000060A0E12158A0E10100E0030200000A00
:1065D000000055E30200001A0000A0E37040BDE88F
:1065E0001EFF2FE145FEFFEB000050E3F9FFFF0A1D
:1065F0000E42A0E33E4B84E2203094E50133C3E336
:10660000203084E50510A0E10600A0E100FEFFEBCC
:10661000203094E560209FE5013383E3203084E55A
:10662000003092E51210D3E50008A0E1020051E32A
:106630002048A0E10100000A0400A0E1E6FFFFEA13
:1066400028FEFFEBFF0050E3FAFFFFDA2C209FE566
:10665000B030D2E10338A0E12308A0E1010050E30B
:10666000F4FFFF1A0030A0E3B030C2E1530400EBA6
:106670000400A0E1D8FFFFEAACBF006204C00062E2
:10668000C4BF006270402DE9400010E30E62A0E339
:106690000E42A0E33E6B86E23E4B84E2FF5000E2F6
:1066A0000300001A800015E30A00001A7040BDE8DC
:1066B0001EFF2FE1203094E50133C3E3203084E551
:1066C00018FEFFEB203094E5800015E3013383E3EF
:1066D000203084E5F4FFFF0A203096E50133C3E360
:1066E000203086E517FEFFEB203096E5013383E38B
:1066F000203086E5ECFFFFEA1C209FE5B030D2E1B8
:10670000803013E214209F150300A0E1B030D211B5
:106710000338A0112308A0111EFF2FE1ACBF0062B7
:10672000AABF006210402DE940309FE5B000D3E1E0
:10673000B010D3E1800011E3B030D3E1084000E2B3
:106740000200000A000054E30940A0130140A00326
:10675000010C13E304408403E8FDFFEB000050E369
:10676000024084130400A0E11040BDE81EFF2FE1A9
:10677000ACBF0062F0402DE98C119FE5B030D1E153
:10678000080013E3FFC000E280619FE50100000AFA
:10679000020010E30B00000AB030D1E1800013E3E7
:1067A0000600000A68319FE5002093E51240D2E51B
:1067B000010054E30C00000A020054E32700000A21
:1067C000F040BDE81EFF2FE1B020D1E1802082E340
:1067D000B020C1E1B030D1E1013CC3E30338A0E116
:1067E0002338A0E1B030C1E1EAFFFFEA24219FE5B0
:1067F000B030D2E13030C3E30338A0E12338A0E168
:10680000B030C2E102001CE3B030D211203083135B
:10681000B030C21101001CE3B030D211103083132C
:10682000B030C211B000D2E1821CA0E30321A0E38A
:10683000012082E0013CA0E32002A0E1131181E2EB
:10684000003082E5000081E50400A0E10410A0E32F
:10685000C90400EB0400A0E1CD0300EBD7FFFFEA81
:10686000B0209FE5B030D2E13030C3E30338A0E17F
:106870002338A0E1B030C2E104001CE3B030D211F3
:1068800020308313B030C21108001CE3B030D211A5
:1068900010308313B030C211B030D2E178409FE5A0
:1068A0002332A0E1B030C4E1832CA0E3B0C0D4E136
:1068B000B670D6E1B0E0D6E1B250D6E10210A0E168
:1068C000B460D6E10200A0E10331A0E3023083E02E
:1068D00002C98CE3132182E2231181E2330180E2B9
:1068E00000E083E5B0C0C4E1005082E5006081E5CE
:1068F000007080E50810A0E30300A0E39E0400EB15
:106900000300A0E3A20300EBACFFFFEAACBF006210
:106910001099006204C00062AABF0062A8BF0062B2
:106920000300E0E31EFF2FE1FF0000E2010040E270
:1069300004E02DE5200050E300F19F97200000EADD
:106940005C6A0062946A0062C4690062C4690062A1
:10695000C4690062C4690062C4690062C4690062FB
:10696000C4690062C4690062C4690062C4690062EB
:10697000C4690062C4690062C4690062C4690062DB
:10698000C4690062C4690062C4690062C4690062CB
:10699000C4690062C4690062C4690062C4690062BB
:1069A000C4690062C4690062C4690062C4690062AB
:1069B000C4690062C4690062C4690062D06900628F
:1069C0002C6A00620300E0E304E09DE41EFF2FE177
:1069D000F4209FE5001092E50030D1E57F3003E21E
:1069E000210053E3E4309FE5E4209FE52010A0E37D
:1069F000001083E502C0A00100C0A01300005CE30A
:106A0000EFFFFF0AC0309FE5002093E50030A0E3D0
:106A1000BA31C2E120C082E50000A0E30FE0A0E1AE
:106A20001CFF2FE10000A0E3E6FFFFEA98209FE5AE
:106A3000001092E50030D1E598209FE57F3003E219
:106A4000210053E384309FE52110A0E302C0A001A0
:106A500000C0A013001083E5E7FFFFEA68309FE560
:106A6000001093E50020D1E57F2002E2410052E3CF
:106A700064309F050120A003002083055CC09F05B2
:106A800048309FE50120A0E300C0A013002083E56B
:106A9000D9FFFFEA30309FE5001093E50020D1E5F3
:106AA0007F2002E2410052E32C309F050220A00328
:106AB0000020830524C09F0510309FE50220A0E33D
:106AC00000C0A013002083E5CBFFFFEA04C00062F2
:106AD000B0BF0062786C0062506C006208C0006257
:106AE000A06C006254309FE5003093E50020D3E5B0
:106AF0007F2002E2210052E3FF0000E20200000AD0
:106B00000310E0E30100A0E11EFF2FE1020050E3CB
:106B10000010A0E3FAFFFF0A220050E30010A0E3F8
:106B2000F6FFFF1A18209FE50530D3E5000082E547
:106B300010209FE50F3003E2B030C2E1F0FFFFEA22
:106B400004C00062B0BF0062AABF006204E02DE58D
:106B5000C13AA0E3FF3E83E2393183E2B0C0D3E122
:106B60000A2AA0E3022082E20008A0E102005CE120
:106B70002038A0E114109FE50300A0E110109F153C
:106B80000300A011E70600EB04E09DE41EFF2FE1E7
:106B9000649A00625C9A006204E02DE5C13AA0E3C9
:106BA000FF3E83E2393183E2B0C0D3E10A2AA0E399
:106BB000022082E20008A0E102005CE12038A0E1AE
:106BC00014109FE50300A0E110109F150300A01111
:106BD000D40600EB04E09DE41EFF2FE1549A00620E
:106BE0004C9A006204E02DE5C13AA0E3FF3E83E247
:106BF000393183E2B0C0D3E10A2AA0E3022082E265
:106C00000008A0E102005CE12038A0E114109FE53B
:106C10000300A0E110109F150300A011C10600EBB6
:106C200004E09DE41EFF2FE12C9A0062249A00628A
:106C3000FF1011E2FF0000E20200001A010050E321
:106C40000100A0E11EFF2F910300E0E31EFF2FE1F2
:106C50000008A0E12008B0E110309F0510009F154A
:106C6000002093050830A003B831C2011EFF2FE1B8
:106C700004C00062E49A00620008A0E12008B0E1CC
:106C800010309F0510009F15002093050830A003C9
:106C9000B831C2011EFF2FE104C00062E49A006215
:106CA0000008A0E12008B0E118309FE518309F05EA
:106CB000002093050030A001BC10D2010300A0E128
:106CC000B811C2011EFF2FE110C0006204C00062B3
:106CD0001EFF2FE11EFF2FE11EFF2FE110402DE9C7
:106CE000F4309FE5002093E51240D2E50100A0E3D7
:106CF000000054E10010A0E32B00000A0010A0E304
:106D0000660200EB0100A0E3011CA0E36D0300EBB1
:106D10000100A0E34010A0E3B90300EB0100A0E3F1
:106D2000031AA0E37E0200EB0100A0E30010A0E341
:106D30006B0200EB0200A0E30010A0E3570200EB9F
:106D40000200A0E3051DA0E34F0300EB0200A0E357
:106D50002010A0E3620200EB0200A0E30010A0E319
:106D60006F0200EB0300A0E3061CA0E34B0200EB64
:106D70000300A0E3061DA0E3430300EB0300A0E330
:106D80000010A0E3660200EB0300A0E32010A0E3E4
:106D9000530200EB44209FE5B030D2E1083083E39A
:106DA000B030C2E11040BDE81EFF2FE10400A0E1B9
:106DB0003A0200EB0400A0E1011CA0E3320300EB67
:106DC0000400A0E12010A0E3450200EB0400A0E1D4
:106DD0000010A0E3520200EBEDFFFFEA04C00062E6
:106DE000ACBF00621EFF2FE11EFF2FE11EFF2FE14F
:106DF0001EFF2FE10C209FE5B030D2E1043083E389
:106E0000B030C2E11EFF2FE1ACBF006204309FE54D
:106E1000003080E51EFF2FE1DCBF0062F0412DE96C
:106E20008C229FE5B030D2E10118A0E1800013E38D
:106E30000040A0E12168A0E10100E0033F00000A5A
:106E4000000056E30600A0013C00000AB030D2E189
:106E5000010C13E30000A0133800001AB030D2E197
:106E6000013C83E3B030C2E148329FE5002093E566
:106E70003E0056E31210D2E53E80A0830680A0912A
:106E80000870A0810870A091010051E32D00000A54
:106E9000010014E30400A0E16100000AC730A0E192
:106EA000000053E303E1A0D382EC8ED201C043E2A1
:106EB00080E08ED20A0000DA03E1A0E382EC8EE2E9
:106EC00080E08EE20130D0E501C04CE20220D0E447
:106ED00001108CE2032482E1000051E304208EE4DF
:106EE000F7FFFFCA010017E30130D0140E52A0E3F0
:106EF00000308E153E5B85E2203095E50133C3E31B
:106F0000203085E5061067E0E5FBFFEB203095E5D6
:106F10000048A0E1013383E32448A0E1203085E567
:106F20000710A0E10200A0E3044088E0120300EB98
:106F30000448A0E10200A0E3150200EB2408A0E150
:106F4000F041BDE81EFF2FE10331A0E3823C83E264
:106F50000020A0E3010014E3002083E50400A0E189
:106F60004200001AC730A0E1000053E382ECA0D336
:106F700004C0A0E1011043E213E18ED2070000DA61
:106F800082ECA0E313E18EE2011041E2B220DCE0EA
:106F9000013081E2000053E304208EE4F9FFFFCAD0
:106FA0000130C7E3030084E0010017E30130D0148F
:106FB0000E42A0E300308E153E4B84E2203094E573
:106FC0000133C3E3203084E5061067E0B4FBFFEB38
:106FD000203094E5021088E2013383E30118A0E138
:106FE000203084E52118A0E1CC309FE5400051E33A
:106FF0000020A0130120A0030048A0E1B020C3E1BD
:107000000100A0E3DC0200EB0100A0E3E00100EBE3
:107010002448A0E1044088E00448A0E12408A0E15D
:10702000C6FFFFEAC730A0E1000053E303E1A0D3AD
:1070300082EC8ED2011043E280E08ED2080000DAAA
:1070400003E1A0E382EC8EE280E08EE2011041E2F7
:10705000B220D0E0013081E2000053E304208EE44E
:10706000F9FFFFCA0130C7E3030084E09CFFFFEA99
:10707000C730A0E1020053E182ECA0D301C043E29B
:1070800013E18ED2C7FFFFDA82ECA0E313E18EE2B8
:107090000130D0E501C04CE20220D0E401108CE2C6
:1070A000032482E1000051E304208EE4F7FFFFCACD
:1070B000BCFFFFEAACBF006204C00062C6BF006252
:1070C00070402DE91C629FE5003096E5020053E315
:1070D0000500000A220053E34000000A0000A0E37C
:1070E000000086E57040BDE81EFF2FE1F8519FE5E6
:1070F0000830D5E5010013E3F0019F05EC019F1571
:10710000B030D001B030D0110130C3030338A0013A
:10711000013083132338A001B030C011B030C0015A
:107120000830D5E5020013E3B030D001B030D01103
:107130000230C3030338A001023083132338A001B7
:10714000B030C011B030C001B030D0E1020013E364
:107150004700000AB030D0E1200013E30800000A25
:107160008C319FE5B020D3E18020C2E30228A0E16A
:107170002228A0E1B020C3E1B010D3E1011C81E3DB
:10718000B010C3E1B000D0E10E42A0E32002A0E1C4
:107190003E4B84E2FF0000E275FDFFEB203094E5FA
:1071A0000133C3E3203084E55EFBFFEB203094E540
:1071B000013383E3203084E5202094E50123C2E3FA
:1071C000202084E55FFBFFEB203094E50020A0E366
:1071D000013383E3203084E50820C5E5BEFFFFEAE4
:1071E00008019FE5B030D0E1010013E32A00000A56
:1071F000FC109FE5B020D1E1802082E3B020C1E106
:10720000B030D1E1013CC3E30338A0E12338A0E171
:10721000B030C1E1B020D0E1302082E3B020C0E145
:10722000B000D0E12002A0E1FF0000E250FDFFEB42
:107230000E42A0E33E4B84E2203094E50133C3E3E9
:10724000203084E537FBFFEB203094E5013383E306
:10725000203084E5202094E50123C2E3202084E54A
:1072600038FBFFEB203094E5013383E3203084E5E5
:1072700099FFFFEA78109FE5B020D1E1802082E3FA
:10728000B020C1E1B030D1E1013CC3E30338A0E15B
:107290002338A0E1B030C1E1B9FFFFEAB030D0E15E
:1072A0003030C3E30338A0E12338A0E1B030C0E1BF
:1072B000B000D0E12002A0E1FF0000E22CFDFFEBD6
:1072C0002C109FE5B030D1E18030C3E30338A0E15A
:1072D0002338A0E1B030C1E1B020D1E1012C82E33C
:1072E000B020C1E1D1FFFFEAB0BF006208C0006278
:1072F000AABF0062ACBF006204E02DE50A32A0E341
:107300001D2EA0E3BC24C3E100C0A0E32C209FE518
:107310000311A0E3221B81E227EBA0E3163283E2F4
:107320000C00A0E1403081E5B0E0C2E140C081E561
:1073300044C081E540E081E504E09DE41EFF2FE1CB
:1073400050C000620311A0E3221B81E20130A0E3E0
:10735000403081E50020A0E3023083E2442081E553
:107360000200A0E1403081E50A2282E20730A0E37A
:10737000BC34C2E11EFF2FE138309FE50120A0E3BD
:10738000002083E50311A0E3221B81E2403091E558
:107390000338A0E1023783E32338A0E1403081E5E0
:1073A000402091E50228A0E1012782E32228A0E104
:1073B000402081E51EFF2FE154C0006234309FE57C
:1073C0000020A0E3002083E50311A0E3221B81E25B
:1073D000403091E50338A0E12338A0E10430C3E355
:1073E0000338A0E12338A0E1272B82E2403081E579
:1073F000402081E51EFF2FE154C00062FF0000E243
:10740000070050E374C19F1570C19F050000CC15A3
:107410000030DCE5050053E303F19F97050000EA27
:107420003C750062F8740062E4740062C07400622B
:1074300090740062447400620630A0E30030CCE532
:107440001EFF2FE10130DCE5013043E2FF3003E2B3
:107450000130CCE50120DCE5000052E31EFF2F11D6
:107460000331A0E3223B83E2402093E50228A0E120
:107470002228A0E11020C2E30228A0E12228A0E1F6
:107480000610A0E3402083E50010CCE51EFF2FE1AD
:107490000311A0E3221B81E2403091E50338A0E113
:1074A000013683E32338A0E1403081E50520A0E3E5
:1074B0000A30A0E30020CCE50130CCE51EFF2FE12F
:1074C0000130DCE5013043E2FF3003E20130CCE57E
:1074D0000120DCE5000052E30430A0030030CC05BD
:1074E0001EFF2FE10230A0E30320A0E30130CCE532
:1074F0000020CCE51EFF2FE184309FE50020A0E3B3
:10750000002083E50311A0E3221B81E2403091E5D6
:107510000338A0E12338A0E10430C3E30338A0E13D
:107520002338A0E1403081E5272B82E20430A0E33C
:10753000402081E50030CCE51EFF2FE140309FE583
:107540000020A0E3002083E50311A0E3221B81E2D9
:10755000403091E50338A0E12338A0E10430C3E3D3
:107560000338A0E12338A0E1403081E5272B82E2F7
:107570000630A0E3402081E50030CCE51EFF2FE17E
:10758000B4BF006254C000620008A0E10331A0E370
:107590002008A0E1223B83E2400083E51EFF2FE1AB
:1075A0000331A0E3223B83E2400093E50008A0E121
:1075B0002008A0E11EFF2FE10008A0E10331A0E3B5
:1075C0002008A0E1223B83E2440083E51EFF2FE177
:1075D0000331A0E3223B83E2440093E50008A0E1ED
:1075E0002008A0E11EFF2FE10331A0E3223B83E24C
:1075F000480093E50008A0E12008A0E11EFF2FE16C
:107600000008A0E10331A0E32008A0E1223B83E2CF
:107610004C0083E51EFF2FE10331A0E3223B83E210
:107620004C0093E50008A0E12008A0E11EFF2FE137
:10763000FF2CA0E30008A0E1F82082E20331A0E3E0
:10764000202802E0223B83E2502083E51EFF2FE149
:107650000331A0E3223B83E2500093E50008A0E160
:107660002008A0E11EFF2FE10118A0E10331A0E3F3
:10767000FF0000E22118A0E1223B83E2001183E732
:107680001EFF2FE10331A0E3223B83E2FF0000E273
:10769000000193E70008A0E12008A0E11EFF2FE110
:1076A0000321A0E3FF0000E2222B82E2003192E7F7
:1076B000763CC3E37030C3E3031081E10118A0E11D
:1076C0002118A0E1001182E71EFF2FE10331A0E3A2
:1076D000223B83E2FF0000E2000193E7060C00E298
:1076E0001EFF2FE10321A0E3FF0000E2222B82E234
:1076F000003192E7073AC3E30118A0E14030C3E349
:107700002118A0E10338A0E12338A0E1100011E323
:1077100010302312200011E320302312003182E7C1
:107720001EFF2FE10321A0E3FF0000E2222B82E2F3
:10773000003192E70139C3E30118A0E17030C3E3DF
:107740002118A0E10338A0E12338A0E1010A11E3E8
:10775000013A2312020A11E3023A2312003182E7AE
:107760001EFF2FE10331A0E3223B83E2FF0000E292
:10777000000193E7300000E21EFF2FE10331A0E398
:10778000223B83E2FF0000E2000193E7030A00E2EC
:107790001EFF2FE10311A0E3FF0000E2221B81E2A4
:1077A000002191E78F3CA0E30228A0E1BF3083E2F3
:1077B000223803E0303023E2003181E71EFF2FE161
:1077C0000311A0E3FF0000E2221B81E2002191E708
:1077D000BF3CA0E30228A0E18F3083E2223803E01F
:1077E000033A23E2003181E71EFF2FE10311A0E3FA
:1077F000FF0000E2221B81E2002191E78F3CA0E321
:10780000012C82E30228A0E18F3083E2223803E0DA
:10781000003181E71EFF2FE10311A0E3FF0000E22A
:10782000221B81E2002191E78E3CA0E30228A0E127
:107830008F3083E2223803E0003181E71EFF2FE121
:107840000311A0E3FF0000E2221B81E2002191E787
:107850008E3CA0E30228A0E18F3083E2223803E0CF
:10786000003181E71EFF2FE10311A0E3FF0000E2DA
:10787000221B81E2002191E78F3CA0E3012C82E3EF
:107880000228A0E18F3083E2223803E0003181E753
:107890001EFF2FE10311A0E3FF0000E2221B81E2A3
:1078A000002191E78F3CA0E3012C82E30228A0E1B4
:1078B0008F3083E2223803E0003181E71EFF2FE1A1
:1078C0000311A0E3FF0000E2221B81E2002191E707
:1078D0008E3CA0E30228A0E18F3083E2223803E04F
:1078E000003181E71EFF2FE10331A0E3223B83E259
:1078F000FF0000E2000193E7300000E2100050E3D7
:107900000000A0130100A0031EFF2FE10331A0E33C
:10791000223B83E2FF0000E2000193E7030A00E25A
:10792000010A50E30000A0130100A0031EFF2FE195
:107930000311A0E3FF0000E2221B81E2002191E796
:107940003E3DA0E30F3083E2032002E0002181E707
:107950001EFF2FE10311A0E3FF0000E2221B81E2E2
:10796000002191E78F3CA0E30228A0E10F3083E2E1
:10797000223803E0003181E71EFF2FE10311A0E36D
:10798000FF0000E2221B81E2002191E78F3CA0E38F
:107990000228A0E18F3083E2223803E0013983E33B
:1079A000003181E71EFF2FE10311A0E3FF0000E299
:1079B000221B81E2002191E78F3CA0E30228A0E195
:1079C0008F3083E2223803E0403083E3003181E7E7
:1079D0001EFF2FE10321A0E3FF0000E2222B82E241
:1079E000003192E7010913E31EFF2F01003192E7F6
:1079F000073AC3E37030C3E30338A0E12338A0E1C2
:107A0000013983E3003182E71EFF2FE10321A0E368
:107A1000FF0000E2222B82E2003192E7400013E3F4
:107A20001EFF2F01003192E7073AC3E37030C3E332
:107A30000338A0E12338A0E1403083E3003182E73E
:107A40001EFF2FE103C1A0E3FF0000E222CB8CE286
:107A500000219CE78F3CA0E30228A0E18F3083E265
:107A6000223803E0FF1001E2013083E100318CE7AE
:107A70001EFF2FE10331A0E3223B83E2FF0000E27F
:107A8000000193E70F0000E21EFF2FE103C1A0E316
:107A9000223B8CE28001A0E1502093E50700C0E387
:107AA0000118A0E1800AA0E10228A0E1A00AA0E15B
:107AB000A118A0E1220880E002C98CE28110A0E1B7
:107AC00080108CE71EFF2FE10331A0E3223B83E20D
:107AD0008001A0E1502093E50700C0E30118A0E178
:107AE000800AA0E10228A0E1A00AA0E1A118A0E17B
:107AF0000239A0E3220880E08110A0E1233183E273
:107B0000801083E71EFF2FE10311A0E3223B81E2F7
:107B10008001A0E1502093E50700C0E3800AA0E1C6
:107B20000228A0E1A00AA0E1220880E0021981E277
:107B3000800091E70008A0E12008A0E11EFF2FE1EE
:107B40000331A0E3223B83E28001A0E1502093E5D2
:107B50000700C0E3800AA0E10228A0E1A00AA0E19A
:107B60000239A0E3220880E0233183E2800093E71A
:107B70000008A0E12008A0E11EFF2FE10331A0E3EF
:107B8000223B83E28001A0E1502093E50700C0E39F
:107B9000800AA0E10118A0E10228A0E1A00AA0E16A
:107BA0000239A0E3220880E02118A0E1133183E22A
:107BB000801083E71EFF2FE10118A0E12128A0E13A
:107BC0003E0052E30800009AA11AA0E1013041E210
:107BD0000338A0E11F0012E32318A0010135A0E142
:107BE000023983E3003080E51EFF2FE1A118A0E1F8
:107BF000010012E3011081120135A0E1003080E59F
:107C00001EFF2FE104E02DE50331A0E38001A0E198
:107C1000223B83E2502093E50118A0E10700C0E376
:107C2000800AA0E121C8A0E10228A0E1A00AA0E109
:107C300002E9A0E33E005CE3222880E033E18EE22B
:107C40000900009AA11AA0E1013041E20338A0E145
:107C50001F001CE32318A0010135A0E1023983E3D2
:107C600082308EE704E09DE41EFF2FE1A118A0E121
:107C700001001CE3011081120135A0E182308EE782
:107C8000F7FFFFEA0331A0E3223B83E28001A0E19A
:107C9000502093E50700C0E3800AA0E10228A0E19C
:107CA000A00AA0E10239A0E3220880E0133183E2B8
:107CB000802093E7FF0FA0E3030080E2000002E0D2
:107CC0001EFF2FE10331A0E3223B83E28001A0E10C
:107CD000502093E50700C0E3800AA0E10228A0E15C
:107CE000A00AA0E10239A0E3220880E0333183E258
:107CF000802093E7FF0FA0E3030080E2000002E092
:107D00001EFF2FE110402DE903E1A0E3224B8EE29C
:107D10008001A0E150C094E50700C0E30118A0E194
:107D2000800AA0E1A00AA0E10CC8A0E1A118A0E18E
:107D30002CC880E002E98EE28110A0E18C108EE771
:107D4000503094E50228A0E10338A0E1230880E048
:107D5000A228A0E10239A0E38220A0E1233183E23E
:107D6000802083E71040BDE81EFF2FE103C1A0E3A0
:107D7000223B8CE28001A0E1502093E50700C0E3A4
:107D80000118A0E1800AA0E10228A0E1A00AA0E178
:107D9000A118A0E1220880E002C98CE28110A0E1D4
:107DA00080108CE71EFF2FE10331A0E3223B83E22A
:107DB0008001A0E1502093E50700C0E30118A0E195
:107DC000800AA0E10228A0E1A00AA0E1A118A0E198
:107DD0000239A0E3220880E08110A0E1233183E290
:107DE000801083E71EFF2FE10311A0E3223B81E215
:107DF0008001A0E1502093E50700C0E3800AA0E1E4
:107E00000228A0E1A00AA0E1220880E0021981E294
:107E1000800091E70008A0E12008A0E11EFF2FE10B
:107E20000331A0E3223B83E28001A0E1502093E5EF
:107E30000700C0E3800AA0E10228A0E1A00AA0E1B7
:107E40000239A0E3220880E0233183E2800093E737
:107E50000008A0E12008A0E11EFF2FE1FF1001E2D1
:107E600010402DE9010051E302E8A0E1FFC000E26B
:107E70002E48A0E11300000A020051E30100000AAD
:107E80001040BDE81EFF2FE10301A0E3220B80E2BA
:107E9000501090E58CC1A0E10118A0E10239A0E3E7
:107EA00021188CE0133183E2814083E7502090E574
:107EB000133143E20228A0E122C88CE0333183E28F
:107EC0008C4083E7EDFFFFEA0331A0E3223B83E22E
:107ED000502093E58CC1A0E10228A0E10219A0E3A3
:107EE0003E0054E322088CE0131181E21900009A4D
:107EF0001F0014E3AE2AA0E1013042020338A001C2
:107F00002328A0010235A0E1023983E3803081E714
:107F10000331A0E3223B83E2502093E50219A0E362
:107F20000228A0E13E0054E322088CE0331181E2F4
:107F30000E00009AA432A0E11F0014E301304302B6
:107F40000338A0012338A0010335A0E1023983E3FF
:107F5000803081E7C9FFFFEAAE28A0E1010014E309
:107F6000012082120235A0E1803081E7E7FFFFEABD
:107F7000A430A0E1010014E3013083120335A0E135
:107F8000803081E7BDFFFFEAFF1001E202C8A0E1F7
:107F9000010051E304E02DE5FF0000E22CE8A0E140
:107FA0000D00000A020051E30100000A04E09DE414
:107FB0001EFF2FE10331A0E3223B83E2502093E533
:107FC0008011A0E10228A0E10239A0E3221881E09B
:107FD000133183E281E083E7F3FFFFEA0331A0E39B
:107FE000223B83E2502093E58011A0E10228A0E12A
:107FF0000209A0E33E005EE3221881E0130180E263
:108000000500008AAC28A0E101001EE301208212D5
:108010000235A0E1813080E7E3FFFFEA1F001EE3A5
:10802000AC2AA0E1013042020338A0012328A001BC
:108030000235A0E1023983E3813080E7DAFFFFEA0D
:10804000FF1001E202C8A0E1010051E304E02DE5C8
:10805000FF0000E22CE8A0E10D00000A020051E35D
:108060000100000A04E09DE41EFF2FE10331A0E3BC
:10807000223B83E2502093E58011A0E10228A0E199
:108080000239A0E3221881E0333183E281E083E703
:10809000F3FFFFEA0331A0E3223B83E2502093E5A4
:1080A0008011A0E10228A0E10209A0E33E005EE306
:1080B000221881E0330180E20500008AAC28A0E1AB
:1080C00001001EE3012082120235A0E1813080E729
:1080D000E3FFFFEA1F001EE3AC2AA0E101304202E9
:1080E0000338A0012328A0010235A0E1023983E36F
:1080F000813080E7DAFFFFEA0331A0E3223B83E22D
:108100008001A0E1502093E50700C0E3800AA0E1D0
:108110000228A0E1A00AA0E10239A0E3220880E041
:10812000133183E2802093E7FF0FA0E3030080E296
:10813000000002E01EFF2FE10331A0E3223B83E2B7
:108140008001A0E1502093E50700C0E3800AA0E190
:108150000228A0E1A00AA0E10239A0E3220880E001
:10816000333183E2802093E7FF0FA0E3030080E236
:10817000000002E01EFF2FE104E02DE503E1A0E393
:108180008001A0E122EB8EE20700C0E350109EE5E3
:10819000800AA0E10229A0E3A00AA0E10118A0E161
:1081A00002C0A0E1211880E0332182E2813092E711
:1081B0003F0B13E313C18CE20120A0E30500001A7A
:1081C00050309EE50338A0E1233880E083209CE70F
:1081D000022BB0E10220A0130200A0E104E09DE424
:1081E0001EFF2FE1FF1001E20321A0E3010051E394
:1081F000222B82E2FF0000E20B00000A0321A0E331
:10820000020051E3222B82E21EFF2F11003192E780
:10821000073AC3E37030C3E30338A0E12338A0E199
:10822000013983E3003182E71EFF2FE1003192E73D
:10823000073AC3E37030C3E30338A0E12338A0E179
:10824000403083E3003182E71EFF2FE1FF1001E29F
:10825000001481E10118A0E12108A0E11EFF2FE137
:108260000038A0E12304A0E1FF0C00E2230C80E130
:108270001EFF2FE103C1A0E3FF0000E222CB8CE24E
:1082800000319CE70338A0E1FF1001E22338A0E1B0
:10829000010051E3012AC3E300218C071EFF2F01D7
:1082A0001030C3E3020051E300318C071EFF2FE1C1
:1082B0000008A0E12008B0E104E02DE50900000A73
:1082C00034309FE5002093E500C092E50FE0A0E187
:1082D0001CFF2FE124309FE5002093E5120082E28D
:1082E00004E09DE41EFF2FE110309FE5002093E5A0
:1082F0000130A0E3B831C2E1F8FFFFEA00C000623C
:1083000004C000620008A0E12008B0E104E02DE50F
:108310000900000A34309FE5002093E508C092E58B
:108320000FE0A0E11CFF2FE124309FE5002093E542
:10833000140082E204E09DE41EFF2FE110309FE56F
:10834000002093E50130A0E3B831C2E1F8FFFFEA75
:1083500000C0006204C000620008A0E12008B0E193
:1083600004E02DE52C00000ADC309FE5DC009FE5F1
:10837000002093E50030A0E3B030C0E10030D2E54A
:108380007F3013E21100001A1120D2E5200012E321
:108390000030D015023083130030C015400012E3C6
:1083A0001900001A0030D0E50130C3E30030C0E509
:1083B0009C309FE5002093E510C092E50FE0A0E11E
:1083C0001CFF2FE184009FE504E09DE41EFF2FE1E8
:1083D000010053E3FBFFFF0A020053E30000A01378
:1083E000F8FFFF1A0930D2E5800013E30F2003E203
:1083F0000E00001A0331A0E3223B83E2022193E73F
:10840000032A02E2010A52E3E8FFFF1A0030D0E536
:10841000013083E30030C0E5E4FFFFEA28309FE548
:10842000002093E50230A0E3B831C2E1E5FFFFEAA6
:108430000331A0E3223B83E2022193E7302002E2F2
:10844000100052E3D9FFFF1AEFFFFFEA04C00062F9
:10845000C0BF006200C0006230402DE948219FE5A6
:10846000001092E50030D1E57F0013E20400001A0D
:108470001130D1E52030C3E31130C1E53040BDE813
:108480001EFF2FE1020050E30100000A0300E0E3B9
:10849000F9FFFFEAB430D1E1000053E3FAFFFF1A1D
:1084A0000830D1E5000053E3F7FFFF1A0930D1E5AA
:1084B000FFE003E280001EE37F0003E20331A0132C
:1084C0000331A003223B8312223B83020021931736
:1084D00000219307D4309FE530C0021203CA020284
:1084E0000020D3E50041A0110041A00100005CE3A1
:1084F00002005011E4FFFF2A1230D1E5000053E3DF
:10850000E1FFFF0A80001EE31200000A0331A0E32E
:10851000223B83E2032094E7302002E2100052E382
:108520000500001AFF4000E20400A0E136FDFFEB69
:108530000400A0E13010A0E369FCFFEB70309FE580
:10854000002093E514C092E50FE0A0E11CFF2FE1AD
:108550000000A0E3C8FFFFEA0351A0E3225B85E22D
:10856000053094E7033A03E2010A53E3F2FFFF1AEE
:10857000000050E30A00001A38309FE54C10D3E5A4
:108580009FFDFFEB053094E70139C3E37030C3E38F
:108590000338A0E12338A0E1033A23E2053084E761
:1085A000E5FFFFEA0AFDFFEBF5FFFFEA04C000620A
:1085B000E09A006200C00062909A0062F0412DE9EA
:1085C00050719FE5004097E5185084E2B811D4E15E
:1085D00008C095E500005CE3000051131E00000A8E
:1085E000B460D5E1010056E10160A021B230D5E1CF
:1085F0000628A0E12208A0E1033080E0B230C5E106
:108600001220D4E5013060E0010052E3B831C4E14A
:108610003200000A0FE0A0E11CFF2FE10040A0E1C2
:108620000000A0E345FDFFEB013086E2C310A0E1AE
:108630008000A0E1030180E2000051E3020980E232
:108640000500000A00C0A0E301C08CE2043090E401
:1086500001005CE1B230C4E0FAFFFF1AB000D5E1DE
:10866000000050E3B0309F15032AA013B020C311BF
:10867000B430D5E1000053E10400008A002097E502
:108680000330A0E31030C2E5F041BDE81EFF2FE14A
:10869000000050E30D00001A001097E50620A0E34B
:1086A0001020C1E50331A0E3223B83E2501093E5A3
:1086B0000229A0E3132182E20118A0E15C309FE5CA
:1086C000A10782E73020A0E3B020C3E1EDFFFFEA7D
:1086D000002097E50530A0E31030C2E5E9FFFFEA8E
:1086E0003C809FE5003098E5010053E3C8FFFF1A86
:1086F0000000A0E311FDFFEB8000A0E1030180E298
:10870000020980E20610A0E188F6FFEBB831D4E15F
:10871000B430C8E1D0FFFFEA04C00062BCBF006211
:10872000BABF006208C0006224309FE50008A0E1E3
:1087300000C093E52008B0E1BA21DCE1B430D101FA
:10874000003091150330620002008310B831CC0173
:108750001EFF2FE104C0006204E02DE55C309FE5C0
:1087600000E0D3E500005EE3FF0000E20D00000A38
:1087700003C1A0E322CB8CE20010A0E3FF2001E2C2
:1087800002319CE7073AC3E37030C3E30338A0E14A
:108790002338A0E1011081E2023083E101005EE1B3
:1087A00002318CE7F4FFFF8A0331A0E3802080E3ED
:1087B000223B83E24C2083E504E09DE41EFF2FE191
:1087C000E09A006210402DE99C409FE5003094E55E
:1087D0001030D3E5050053E3030053131700000ADC
:1087E000070053E30820A0E31800000A003094E5D6
:1087F0001020C3E574209FE50000A0E34C10D2E5F3
:10880000FFFCFFEB003094E51000D3E5080050E3D7
:108810000500001A58309FE5012AA0E3B020C3E10B
:1088200050209FE51030A0E3B030C2E1090050E3D2
:108830000000A0130100A0031040BDE81EFF2FE1BF
:108840005DFFFFEB003094E51020D3E5E7FFFFEA82
:1088500024309FE5002093E528C092E50FE0A0E1D9
:108860001CFF2FE10820A0E3DFFFFFEA04C0006245
:10887000909A0062BCBF0062BABF0062D8BF0062BB
:108880001EFF2FE1F0412DE9C8609FE50351A0E3F1
:10889000225B85E20680A0E1443095E50338A0E143
:1088A0002338A0E1B030C6E1B020D6E17F1CA0E3C0
:1088B000020912E3FF1081E29C709FE52300000A89
:1088C000441085E5B030D8E10F1003E20010C7E591
:1088D000013195E70338A0E12348A0E17C309FE512
:1088E0000121A0E1020914E3032082E00E00001A36
:1088F000800014E3E7FFFF0A0010D7E5012195E7A8
:10890000072AC2E3F020C2E30228A0E150309FE52D
:108910002228A0E1012185E7013183E004C013E5AD
:108920000FE0A0E11CFF2FE1DAFFFFEA013195E73C
:108930007030C3E3033AA0E1233AA0E1013185E7B7
:1089400004C012E50FE0A0E11CFF2FE1E7FFFFEA02
:10895000F041BDE81EFF2FE1D4BF0062B8BF006246
:10896000AC990062E8990062F0472DE91CA29FE5EE
:1089700000109AE51030D1E5040053E30000A01385
:108980000100A003040053E3020053132200001A65
:10899000B851D1E1000055E30060A013016000026E
:1089A000000056E3E8319F151020A013187081E2F3
:1089B000B020C3110710A0131B00000A00309AE575
:1089C0001010C3E5FF2001E200309AE51020C3E556
:1089D000C0219FE50000A0E34C10D2E588FCFFEB2E
:1089E00000309AE51000D3E5080050E30500001AB6
:1089F000A4319FE5012AA0E3B020C3E190219FE5C7
:108A00001030A0E3B030C2E1090050E30000A01331
:108A10000100A003F047BDE81EFF2FE1060053E36D
:108A20003000000A0820A0E3E6FFFFEAB420D7E107
:108A3000020055E10290A0830490A093020055E14A
:108A40000250A0210538A0E12388A0E10800A0E1A0
:108A500008C097E50FE0A0E11CFF2FE10040A0E176
:108A60000600A0E127FCFFEB013085E28000A0E1D9
:108A7000030180E2C3C0B0E1020980E20800000AFD
:108A80000610A0E10030D4E50120D4E5011081E218
:108A9000023483E101005CE1043080E4024084E2BE
:108AA000F7FFFF1A0810A0E10000A0E332FCFFEB83
:108AB000B230D7E1B020D7E1033088E0B230C7E16F
:108AC000022068E0C8309FE5B020C7E13020A0E375
:108AD000B020C3E1C0209FE5033AA0E3FF1009E204
:108AE000B030C2E1B4FFFFEA0130D1E5050053E345
:108AF0000600000AA4309FE5002093E524C092E51B
:108B00000FE0A0E11CFF2FE10820A0E3ADFFFFEA8A
:108B10000030D1E57F2013E2F5FFFF1A80309FE59A
:108B200000E0D3E500005EE30510D1E50D00000A8A
:108B300003C1A0E30200A0E122CB8CE2FF2000E20F
:108B400002319CE7073AC3E37030C3E30338A0E186
:108B50002338A0E1010080E2023083E100005EE101
:108B600002318CE7F4FFFF8A38209FE50331A0E350
:108B7000801081E3223B83E24C1083E5003092E5D4
:108B800020C093E50FE0A0E11CFF2FE1D8FFFFEA32
:108B900004C00062BABF0062909A0062BCBF00626B
:108BA000D8BF0062E09A006200C00062F0472DE981
:108BB0000361A0E3226B86E2501096E5D4879FE51F
:108BC0000239A0E30118A0E1233183E2005098E5C7
:108BD000A12793E71000D5E50228A0E12218A0E123
:108BE0000331A0E3090050E3023983E28140A0E1B0
:108BF0001200000A8120D3E7013183E20020C5E59D
:108C0000073183E28120D3E7024984E20120C5E5F0
:108C10000B4184E2B200D4E190FDFFEBB400C5E16A
:108C2000B600D4E1005098E58CFDFFEBB800C5E13B
:108C3000003098E5BA40D4E1BC40C3E10350A0E164
:108C4000BC40D5E10130A0E3000054E31030C5E59D
:108C50003300001A0030D5E57F3013E20170D5E50E
:108C60005100000A010053E3A500000A020053E38B
:108C7000DC00000A20379FE50700A0E1002093E513
:108C800030C092E50FE0A0E11CFF2FE1050070E38A
:108C900009C0A0030D00000A000050E3BD00001A47
:108CA0000331A0E3223B83E2500093E50219A0E3E5
:108CB000131181E20008A0E10030A0E3DC269FE56B
:108CC000A03781E73010A0E3B010C2E106C0A0E3F6
:108CD000003098E510C0C3E5C4369FE50000A0E36E
:108CE0004C10D3E5C6FBFFEB003098E51000D3E550
:108CF000080050E30500001AA8369FE5012AA0E30A
:108D0000B020C3E194269FE51030A0E3B030C2E16B
:108D1000090050E30000A0130100A003F047BDE8E4
:108D20001EFF2FE10110D5E5060051E35800000AAF
:108D3000000051E33100001AB430D5E1000053E3E4
:108D40000100001A020054E30D01000A48469FE5A5
:108D5000003098E5002094E50100D3E52CC092E5B1
:108D60000FE0A0E11CFF2FE1050070E38B00000A7B
:108D700000C098E5FF3CA0E3B8E1DCE1FF3083E20E
:108D800003005EE10930A0031030CC05D1FFFF0ADB
:108D9000040070E30100000A00005EE38300001A93
:108DA0000830A0E31030CCE5CAFFFFEA090057E322
:108DB0004800000A050057E36A00000A030057E371
:108DC000DD00000A010057E3A9FFFF1A0530D5E5D1
:108DD000010053E3A6FFFF1AB830D5E1000053E3CA
:108DE000A3FFFF1A1130D5E5200013E3A0FFFF0A0F
:108DF00098FDFFEB000CA0E1400CA0E13D0000EA73
:108E0000080051E37200000A0A0051E3CEFFFF1A86
:108E10000030D5E57F3003E2010053E3CAFFFF1ABB
:108E20001230D5E5000053E3C7FFFF0AB430D5E1A7
:108E3000000053E3C4FFFF1A0810D5E5000051E31A
:108E4000C1FFFF1A010054E3BFFFFF1A48459FE529
:108E50000900D5E5003094E534C093E50FE0A0E1CA
:108E60001CFF2FE1000050E33C259F051700001A6E
:108E7000003098E50010A0E3202083E5BA11C3E19B
:108E80000000A0E30FE0A0E112FF2FE10000A0E34B
:108E9000B6FFFFEA0030D5E57F0013E3AAFFFF1A13
:108EA0000430D5E5010053E3C000000A020053E39B
:108EB0009100000A030053E3A3FFFF1AD8449FE583
:108EC000003094E5402093E5000052E3E7FFFF1AED
:108ED000003098E59EFFFFEAD0349FE50520D5E5F8
:108EE0000110D3E5010052E16C00009AFC30A0E3D0
:108EF000033CA0E1430CA0E1000050E367FFFF0A40
:108F00005BFFFFEA0B0057E359FFFF1A88349FE528
:108F10000510D5E5002093E50900D5E534C092E5BC
:108F20000FE0A0E11CFF2FE1002098E51230D2E510
:108F3000000053E30700000A000050E30500001A98
:108F40000830D2E5000053E30200001A0430D2E5F5
:108F5000000053E36C00000AFC00A0E3003CA0E129
:108F6000430CA0E1E3FFFFEA0530D5E5800013E301
:108F70000800001A0430D5E5000053E30500001A8C
:108F8000B830D5E1000053E30200001A1230D5E5F5
:108F9000000053E341FFFF0A08C0A0E34BFFFFEAD4
:108FA000002098E50930A0E31030C2E549FFFFEA50
:108FB0000030DCE5800013E38000001AE4239FE525
:108FC0000330A0E3031AA0E31030CCE5B010C2E1F7
:108FD00040FFFFEA0030D5E57F0013E3D0239F0573
:108FE000A2FFFF0A58FFFFEA010057E37FFFFF0AD5
:108FF000030057E31EFFFF1A0930D5E5FFC003E267
:1090000080001CE37F1003E20131961701319607BF
:1090100030000312030A030290339FE50020D3E5DA
:1090200001E1A01101E1A001020051E1AEFFFF2A20
:10903000B420D5E1013070E20030A033000052E3EB
:1090400001308313000053E3A7FFFF1A1230D5E568
:10905000000053E3A4FFFF0A80001CE3C300000AE2
:109060000321A0E3222B82E202309EE7073AC3E30A
:109070004030C3E30338A0E12338A0E1103023E2FD
:1090800002308EE72C339FE5002093E518C092E56F
:109090000FE0A0E11CFF2FE10030A0E393FFFFEA07
:1090A0000430D5E5000053E38FFFFF1AB830D5E157
:1090B000000053E38CFFFF1AC13A83E2FF3E83E2D4
:1090C000393183E2B010D3E10A2AA0E3022082E220
:1090D000020051E10110A0130210A003D4329FE559
:1090E0001210C5E5002093E504C092E50FE0A0E171
:1090F0001CFF2FE10430A0E17CFFFFEA98429FE5CE
:10910000003094E53C2093E56EFFFFEAA4329FE532
:10911000002093E50CC092E50FE0A0E11CFF2FE1D9
:10912000003098E50910D3E50520D3E50400A0E15F
:109130001420C3E51310C3E587FFFFEA0530D5E52A
:10914000010053E3CAFEFF1AB830D5E1000053E333
:10915000C7FEFF1A1130D5E5200013E3FF3003E20C
:10916000C3FEFF0A203083E31130C5E544229FE5AA
:10917000003092E51CC093E50FE0A0E11CFF2FE159
:10918000C6FEFFEA0830D5E5000053E3EEFEFF1A05
:109190000030D5E57F3013E24D00001AB830D5E13C
:1091A000000053E3E8FEFF1A0C229FE52FFFFFEAC1
:1091B000E4419FE5003094E5382093E541FFFFEA64
:1091C000BC30DCE10E0053E1B831CC31C8319FE551
:1091D000002093E5B8E1DC311010DCE54C30D2E53D
:1091E00000005EE304005103BC31CCE1AC319F05CB
:1091F0001010A0030E50A0E100A0A01301A0A00336
:1092000018608CE20720A003B010C3012D00000AF3
:10921000B420D6E102005EE10290A0830490A09306
:10922000020055E10250A0210538A0E12378A0E119
:109230000700A0E108C096E50FE0A0E11CFF2FE1C8
:109240000040A0E10A00A0E12EFAFFEB013085E228
:109250008000A0E1030180E2C3C0B0E1020980E226
:109260000800000A0A10A0E10030D4E50120D4E58E
:10927000011081E2023483E101005CE1043080E40A
:10928000024084E2F7FFFF1A0000A0E30710A0E10C
:1092900039FAFFEBB230D6E1B020D6E1033087E0F7
:1092A000B230C6E1022067E0F0309FE5B020C6E1B1
:1092B0003020A0E3B020C3E1E8209FE5033AA0E31B
:1092C000B030C2E1FF2009E2003098E51020C3E58C
:1092D00080FEFFEA010053E30D00001AB8409FE54D
:1092E0000900D5E5003094E534C093E50FE0A0E136
:1092F0001CFF2FE1000050E3F4FEFF1A003098E558
:109300001220D3E5000052E391FEFF0AA8209FE55A
:10931000D6FEFFEA020053E38BFEFF1A0930D5E5C3
:10932000800013E30F1003E2700003E2013196178F
:109330000131960730C0031203CA03026C309FE567
:109340000020D3E5020051E10010A0230110A0335A
:10935000000050E30010A013000051E37AFEFF0A62
:1093600000005CE378FEFF0A4C209FE5BFFEFFEAA9
:109370000321A0E3222B82E202309EE70139C3E3FE
:109380007030C3E30338A0E12338A0E1013A23E2BF
:1093900002308EE73AFFFFEA04C00062D8BF0062E5
:1093A000BABF0062909A0062BCBF00620483006290
:1093B000E09A0062B082006200C0006258830062DE
:1093C000F0452DE9CC829FE50351A0E3225B85E2C5
:1093D00008A0A0E1443095E50338A0E12338A0E1DE
:1093E000B030C8E1B020D8E1020912E36400000AFD
:1093F0007F3CA0E3FF3083E2443085E5B020DAE132
:1094000094629FE50F2002E2000052E30020C6E5CF
:109410005D00001A001095E5000095E5003095E527
:109420000139C3E37030C3E30338A0E12338A0E17E
:10943000023A23E2003085E5002095E5072AC2E3E1
:109440004020C2E30228A0E12228A0E1202022E25D
:10945000002085E5B030DAE140629FE540729FE58B
:10946000031A01E2300000E2100013E3B010C6E17D
:10947000B000C7E16400000A003095E50338A0E1C0
:109480002348A0E1800014E37000001A020B14E3EB
:109490006700001A020914E31A00000A003095E57B
:1094A0007030C3E3033AA0E1F8419FE5233AA0E11D
:1094B000003085E5002094E51030D2E5050053E347
:1094C000030053136900000A070053E36B00000A0E
:1094D000003094E50820A0E31020C3E5C8219FE5F3
:1094E0000000A0E34C10D2E5C5F9FFEB003094E595
:1094F0001020D3E5080052E3013AA003B030C601C2
:109500001030A003B030C7010311A0E3221B81E299
:10951000003091E50139C3E3B020D6E17030C3E3F8
:109520000338A0E12338A0E1010A12E3013A231233
:10953000020A12E3023A2312003081E5003091E57D
:10954000073AC3E3B020D7E14030C3E30338A0E1DA
:109550002338A0E1100012E310302312200012E3A0
:1095600020302312003081E5443095E50338A0E136
:109570002338A0E1B030C8E1B020D8E1020912E3FD
:109580009AFFFF1AF045BDE81EFF2FE1023195E773
:109590000338A0E12348A0E1020914E30211A0E18D
:1095A0000E00001A800014E389FFFF0A0030D6E5A0
:1095B000032195E7072AC2E3F020C2E30228A0E1D5
:1095C000E8109FE52228A0E1032185E7031181E04F
:1095D00004C011E50FE0A0E11CFF2FE17CFFFFEAD2
:1095E000023195E77030C3E3033AA0E1233AA0E1EA
:1095F000023185E7B8209FE5022081E004C012E532
:109600000FE0A0E11CFF2FE1E5FFFFEA003095E548
:10961000073AC3E3F030C3E30338A0E12338A0E105
:10962000003085E5CFFCFFEB003095E5220B13E31E
:10963000B4FFFF0A003095E57030C3E3033AA0E1C0
:10964000233AA0E1003085E557FDFFEBADFFFFEACF
:10965000003095E5073AC3E3F030C3E30338A0E1F7
:109660002338A0E1003085E5BEFCFFEB86FFFFEA72
:10967000D1FBFFEB003094E51020D3E595FFFFEA26
:1096800030309FE5002093E528C092E50FE0A0E18F
:109690001CFF2FE18DFFFFEAD4BF0062B8BF00625C
:1096A000BCBF0062BABF006204C00062909A006250
:1096B000E8990062AC990062D8BF006230402DE9A1
:1096C0002FF2FFEB000050E30301A0E33E10A0E304
:1096D0009C509FE5820C80E20C0000DA6CF2FFEBFC
:1096E0000018A0E1400050E30030A0130130A003B7
:1096F0002118A0E10100A0E3B030C5E11EF9FFEBA5
:109700000100A0E322F8FFEB3040BDE81EFF2FE18F
:10971000B030D5E10338A0E12348A0E10301A0E384
:10972000010054E3820C80E23E10A0E344209FE558
:109730000500000AB030D2E1013CC3E30338A0E1E8
:109740002338A0E1B030C2E1EEFFFFEA50F2FFEBB8
:109750000018A0E10030A0E30400A0E12118A0E17E
:10976000B030C5E104F9FFEB0400A0E108F8FFEB1D
:10977000E4FFFFEAC6BF0062ACBF006210402DE903
:109780000100A0E34EF9FFEB34409FE50010A0E19B
:109790000301A0E30130A0E3820C80E2B030C4E119
:1097A00062F2FFEBF0F1FFEB7F0050E30100A0E37A
:1097B0000030A0C3B030C4C100F8FFCB1040BDE8FA
:1097C0001EFF2FE1C4BF006204E02DE5ECF1FFEBCA
:1097D000000050E30301A0E3820C80E23E10A0E30E
:1097E00040209FE5800080E2080000DA04F2FFEBF1
:1097F0000018A0E12118A0E10200A0E3DEF8FFEBD1
:109800000200A0E3E2F7FFEB04E09DE41EFF2FE17E
:10981000B030D2E1013CC3E30338A0E12338A0E13A
:10982000B030C2E1F7FFFFEAACBF006204E02DE513
:1098300044209FE5B030D2E103C1A0E3020913E365
:1098400083CC8CE20300A0E30210A0E30100001A25
:1098500004E09DE41EFF2FE1B030D2E10F3003E2BF
:10986000B030C2E1B020D2E100208CE5C2F8FFEBBD
:109870000300A0E3C6F7FFEBF4FFFFEAA8BF006216
:1098800000C09FE51CFF2FE16949006200C09FE511
:109890001CFF2FE1F556006200C09FE51CFF2FE181
:1098A0002D4B006252494656303130360A000000D6
:1098B0004F534521000000000000000000000000A0
:1098C000000000001F0000001C0000001F0000003E
:1098D0001E0000001F0000001E0000001F0000000E
:1098E0001F0000001E0000001F0000001E000000FE
:1098F0001F000000525246563031303400120330FF
:109900000030003000300030003000300031000006
:10991000A120000000000200000000000C03300045
:1099200031002E003000310030034200610072002F
:1099300063006F006400650020004400650076004D
:10994000690063006500200043006F006D00200087
:1099500050006F007200740024034F005000540048
:109960004F002D0045006C0065006300740072001C
:109970006F006E006900630073002E000403090489
:109980000000A0E30010A0E10020A0E100B0A0E1F1
:109990000070A0E108A09FE51AFF2FE1060000EF8C
:0899A0001EFF2FE101400062EF
:1099A800090000007C97006280880062808800625D
:1099B80080880062808800628088006280880062F7
:1099C80080880062808800628088006280880062E7
:1099D80080880062808800628088006280880062D7
:1099E800BC960062C89700622C980062808800626A
:1099F80080880062808800628088006280880062B7
:109A080080880062808800628088006280880062A6
:109A18008088006280880062808800627C99006289
:109A28000400000058990062240000002899006290
:109A3800300000001C9900620C00000000000000CB
:109A480000000000339B006219000000F09A0062D9
:109A5800430000005E9B0062120000004C9B006205
:109A680012000000D86C0062DC6C0062E46D0062D9
:109A7800E86D0062D06C0062D46C0062EC6D00622C
:109A8800F06D0062F46D006274630062A0640062AD
:109A9800006500621C6E0062AC650062846600624C
:109AA800F86600622467006274670062C070006232
:109AB8002069006228690062E46A0062306C006212
:109AC8004C6B0062986B0062E46B00620C6E006283
:109AD80000000000400000000402000000C2010075
:109AE8000000080001000000090243000202008093
:109AF800FA09040000010202010005240010010512
:109B0800240100010424020205240600010705833C
:109B18000308000A09040100020A00000007050101
:109B280002400000070582024000000902190001F6
:109B3800010080FA0904000001FF00000007058108
:109B48000240000012011001020000405A0602A063
:109B580001010102030112011001000000405A0630
:089B68000900010101020301E3
:04000005620099807C
:00000001FF
:0200000460009A
:100010005345435245545859000000000000000069
:1000200000B500F0E3FC00F0D5FC03F01BFC01F090
:1000300039FC01F0C7FC03F047F800F0F7FC013091
:1000400005D101210320494201F0FAF8FEE700F052
:10005000D9FD01F043FB0FF087F90CF0F1FC06F03D
:1000600071FB0DF033FB00200CF0EEF9002804D0FA
:1000700001200CF0CDFA01F0F3FC0CF0B5FC0AF015
:1000800041FE09F08BF801F0B7FC01F0B5FD10F06E
:100090000DF808F069FF002803D005F075FB0EF09D
:1000A00023FA074B1B6800F00DF8002801D100F07F
:1000B000F1FC0EF00BFB01F0D3FC01BC004700008B
:0800C000080001621847C04668
:1001000052424756303231380000000000000000F3
:100110008401006001002DE900004FE1C00080E390
:1001200000F061E10100BDE81EFF2FE101002DE9B3
:1001300000004FE18000C0E300F061E10100BDE894
:100140001EFF2FE101002DE9D300A0E300F061E1E3
:100150000100BDE81EFF2FE158069FE51EFF2FE1BD
:1001600054069FE5000090E51EFF2FE110402DE9A9
:100170000D00A0E1DE2601EB00009DE51040BDE88A
:100180001EFF2FE130402DE900404FE1200014E335
:10019000B2405E11FF4CC41304401E05FF44C4036B
:1001A00018569FE5044195E70FE0A0E114FF2FE109
:1001B0003040BDE80EF0B0E1020000EF00369FE5F0
:1001C000000083E51EFF2FE1140100602C01006098
:1001D0005801006044010060600100605801006047
:1001E0006C010060E10A0060D52100600D13006021
:1001F00041120060C9190060E1190060790D0060CA
:10020000210B0060E91100609D1000602D0B006063
:10021000C90B00609D080060C90A00601D91006064
:100220009D8F0060318F0060D18F00604D8F006026
:10023000698F006051370060153400603D35006003
:10024000A137006045370060653700609137006076
:10025000893600605935006075210060451F0060D7
:10026000B91D00603D210060B9210060151E0060CD
:10027000111D0060D91D00602D1C0060FD0D006087
:10028000210D0060990D0060350D0060D50D0060F6
:10029000B10C0060150D00603D220060A5240060D7
:1002A00091240060B1240060C524006079220060C0
:1002B000611A006019C3006011C60060B5C4006017
:1002C000DD1300607118006079190060F517006097
:1002D0008906016065090160DD030160A106016016
:1002E000CD090160A90B0160FD0901604133006087
:1002F000C9330060853100600933006061320060FD
:10030000E1310060A52A0060BD250160E9D80060E8
:100310009DD800602DD800605DF50060D1F50060CB
:10032000C9F50060CDF5006049F4006089F5006012
:100330001DF50060F9F40060A9F4006059760260D0
:1003400099F50060B4070060B4070060B40700606E
:10035000DDF5006041F30060B9F20060B4070060B1
:10036000DD75026025760260B4070060B4070060A6
:10037000FD750260C9750260EDF3006045760260AC
:1003800015F4006025F400600DF3006021F30060B7
:1003900059000160B4070060D1F200603D9900602F
:1003A00025AB00606D940060AD3F0060DD3F0060F4
:1003B0000D40006025AB006051B50060E59900601C
:1003C000F52F026001300260A9300260C130026086
:1003D000513102607531026081320260493202603F
:1003E0007933026069330260953302607D320260C6
:1003F000DD320260AD330260D9320260C533026083
:10040000C53402603D340260E1340260B9360260F6
:1004100019360260693B026079380260113C026063
:100420008D3B0260293C0260953C0260093D026000
:10043000513D02608D3D0260993D0260A13D026028
:10044000BD3D0260693F02607D3F0260913F0260F6
:10045000B5450260A1460260094702609947026003
:10046000215102601D510260795A0260495A0260AE
:10047000995A02605D5A0260155A0260C95A0260B8
:10048000AD5A02603D5B0260ED5A0260515B026052
:10049000995B0260A56002608D600260B9600260D5
:1004A000E160026005610260216102602962026010
:1004B0006962026035630260AD620260756302606A
:1004C000E962026091630260E1630260616402605C
:1004D000E96402604965026091650260F565026049
:1004E000BD66026061880260A57B0260A18802602F
:1004F00009A1026029A10260B9A10260EDA1026018
:100500000DA20260DDA2026005A302603D2202602E
:10051000DD330260193F0260B13E0260D1440260E7
:100520003D4502605D1F0060E58F0060FD5B02607D
:100530009120026045B70260C1B70260D1B7026086
:1005400065B8026075B802603DB9026015BA026014
:1005500015BA026015BA0260DCBD02605CBD0260C3
:1005600034BD026018BA026088BD026024BA02601D
:1005700034BD026024BA0260C8BD026020BA0260C5
:10058000C8BD02605CBD0260DCBD026088BD026067
:1005900020BA0260D8C0026048BE0260D8C00260C3
:1005A00048BE0260DCC30260F4C20260F4C20260B2
:1005B000E4C2026094C3026078C30260ECC20260CD
:1005C000C4C30260ECC202600CC40260F4C30260E7
:1005D000F4C20260ACC3026094C30260E4C2026071
:1005E00024C4026024C40260D1670060410D006031
:1005F0004D0D00600DCB0060BDD00060590D006056
:10060000690D0060CD3700606120026051200260FA
:1006100051740260FD72026085670260C1720260FF
:10062000DD7202604520026080C4026080C4026006
:10063000D10A0060650B00600D0B0060F50A0060D8
:1006400069D80060A52A006021C50060891E00608D
:10065000FD4400602D4800601DCB0060A51F0060B8
:10066000152000609D400060E1D00060B9D10060BD
:100670007DC400601D9B00600DA500608D92006030
:1006800005990060F9980060E598006059140060D1
:10069000F5A90060B407006035CB0060B9D50060F3
:1006A00005B10060113D0060F9F80060B40700601A
:1006B000B4070060B4070060B4070060B4070060CE
:1006C000B4070060B4070060B4070060B4070060BE
:1006D000B4070060B4070060B40700604D8F00608D
:1006E000911C0060351D00600521006059210060EB
:1006F0009121006055200060D9C40060F935006088
:10070000F1360060E5CA0060EDCA006035D20060D5
:1007100005D20060CDCA006065D200608514026019
:10072000211A026091130260751402600D170260B5
:10073000C9580060159000607D1E0060F5CA006019
:1007400095200060B4070060B4070060B407006043
:10075000B4070060B4070060B4070060B40700602D
:10076000B4070060B4070060B4070060B40700601D
:10077000B4070060B4070060B4070060B40700600D
:10078000B4070060B4070060B4070060B4070060FD
:10079000B4070060B4070060B4070060B4070060ED
:1007A000B4070060B4070060B4070060B4070060DD
:1007B000B40700601EFF2FE1E401006034740020E4
:1007C000C80100602800016258209FE5B430D2E1E2
:1007D0000010A0E3BC11C2E14C009FE5B000D0E1E5
:1007E000030010E30EF0A00140009FE5B010D0E13F
:1007F000021081E2020C51E30EF0A081B010C0E1C2
:100800002C009FE5001090E5013083E2B230C1E09A
:10081000B020D2E1032042E0012082E2B220C1E018
:10082000B010C0E10EF0A0E100A000E032130162C0
:100830004C23016240230162F0B581B0009001F0C9
:10084000C3F801251DE06F00381C16E0124BEA18B2
:100850000133C118552316780C78137056235B4268
:100860000B701378552B03D1400016700C7004E008
:1008700001F0B6F8012040420AE0009A9042E5D328
:100880003D1C009A53109D42DDD301F0A9F80020D1
:1008900001B0F0BC02BC08470000006210B5424B3A
:1008A000424A9C1A424B9C4201D8002009E0802019
:1008B0004002FFF7C1FF013001D1002071E080202C
:1008C00040023C4B9C420AD980208002FFF7B4FFD3
:1008D000013002D18020400263E080208002364B4C
:1008E0009C420AD98020C002FFF7A6FF013002D146
:1008F0008020800255E08020C002304B9C420AD903
:1009000080200003FFF798FF013002D18020C00251
:1009100047E0802000032A4B9C420AD980204003F4
:10092000FFF78AFF013002D18020000339E08020E8
:100930004003244B9C420AD980208003FFF77CFFB0
:10094000013002D1802040032BE0802080031E4B29
:100950009C420AD98020C003FFF76EFF013002D10C
:10096000802080031DE08020C003184B9C420AD9E0
:1009700080200004FFF760FF013002D18020C00317
:100980000FE080200004124B9C420AD980204004D2
:10099000FFF752FF013002D18020000401E08020E7
:1009A000400410BC02BC0847000000630000006265
:1009B000FFFF0000FFFF0100FFFF0300FFFF070034
:1009C000FFFF0F00FFFF1F00FFFF3F00FFFF7F0043
:1009D000FFFFFF00034A044901E0002308C28A42E6
:1009E000FBD3704700000162E0BF01620448054A82
:1009F000054901E008C808C28A42FBD370470000DD
:100A0000E09D0460606D0020C07D00200448054A20
:100A1000054901E008C808C28A42FBD370470000BC
:100A2000E09D0460606D0020D06F002000B581B0B3
:100A3000FFF734FF144A154B80181860904202D11A
:100A4000012040421CE0421E012082431388694677
:100A50001B0402311B0C0B8013881B041B0C0B8026
:100A6000002313801023138013881B041B0C0B809E
:100A700013881B041B0C0B80054B10801380002077
:100A800001B002BC0847000000000062FC2F0162B8
:100A90001F9DFFFF00B509490948102225F0AAFD56
:100AA000002808D101F0B6F90120962100F0A6F93E
:100AB000044B00F0A5F801BC00470000D882046098
:100AC0000000014000010140004870470001006043
:100AD00000B5024925F008FD01BC00470001006097
:100AE00000B5034B1B6800F08BF802BC0847000000
:100AF0000400016210B5041CFFF7F2FF011C201C6A
:100B000025F0F2FC10BC01BC0047000000B5034911
:100B1000102225F0D3FD01BC00470000100000604A
:100B2000014B1868704700003474002030B594B051
:100B3000684624F06FFF0AAC6B4607CB07C407CBAF
:100B400007C407CB07C41B6804482360044BC01AC2
:100B5000119B14B0C01A30BC02BC084700000162EF
:100B600000400062F0B58AB0041C0E1C0092002800
:100B700001DB019104E02D230B704B1C01934442D7
:100B8000104F002202AB1E25DA770CE00099201CE2
:100B90002AF0D4FEC25D02AB5A55201C00992AF0FF
:100BA00017FE013D041C002C01D0002DEED10AAB34
:100BB000E9181F39019825F097FC301C0AB0F0BCE9
:100BC00002BC0847EC82046010B50A4A1368041C92
:100BD000002B01D1084B13601068084B4118994253
:100BE00004D901200C234042236000E0116010BCB6
:100BF00002BC084700000162004000620000016280
:100C00001847C04600B5114B1A1C5032002102C3D0
:100C10009342FBD10E4A0F4B1A800F4A043B1A80B5
:100C20000E4A0C3B1A800422524208331A800C4BA5
:100C300019600C4B19600C4B19600C4B0C4A196075
:100C40000020022100F014FE01BC00478452016222
:100C500017400000189000E04080FFFF881300005C
:100C6000D8520162DC520162E4520162E052016238
:100C7000BD0E0060064A074B1A80074A04331A80EB
:100C8000064A103B1A800422524208331A807047E9
:100C90004080FFFF149000E0174000008813000020
:100CA000024A50231380043213807047149000E0EE
:100CB00000B5054B186001E00BF032FC024B1B68DD
:100CC000002BF9D101BC0047E45201620004064B3D
:100CD000000C434381B001E0009B013B0093009B6B
:100CE000002BF9D101B070475C4400000004000CF7
:100CF00043011B1A9B001B18DA0081B0D21A009224
:100D000002E0009B013B0093009B002BF9D101B056
:100D100070470000014B186070470000E05201620C
:100D2000034B1B680020002B00D1012070470000FE
:100D3000E0520162014B186870470000E052016206
:100D4000014B186870470000E4BF0162014B186056
:100D500070470000E4BF0162024B18880004000CD9
:100D600070470000E0BF0162024B0004000C1880D5
:100D700070470000E0BF0162054B1B68002B05D1E6
:100D8000044B1B68002B01D1002000E001207047BC
:100D9000A45301628458016210B50C4A136883425F
:100DA00010D00B4B04329A42F8D1503A0021141C57
:100DB0001368002B02D18B00185103E0013104327B
:100DC0001429F5D110BC01BC004700008452016217
:100DD000D452016210B5084900220C1C0B688342F2
:100DE00003D192000023135103E001320431142A8D
:100DF000F4D110BC01BC004784520162012802D129
:100E000000292DD012E0032821D0032804DC00287B
:100E100026D0012848D109E010282AD0202835D032
:100E2000052841D1214A012313600CE0312901D862
:100E3000322103E01E4B994200D9191C1B4B19604B
:100E40001A681C4B1A601C4A002313602CE01A4BD2
:100E50001B68002B28D1174B1A68144B1A6023E02B
:100E6000124B002119601A68124B1A60124B19605C
:100E70001AE00E4B00221A600F4A1368FA21013360
:100E8000890013608B420FDD11600DE00A490B6889
:100E9000012B05D1074B1A68044B1A60002302E0AE
:100EA000002B01DD013B0B6070470000DC5201624A
:100EB00020BF0200D85201628052016230B5624AFE
:100EC000136801331360614A138880211B044902AF
:100ED0005B181B0C13805E4A1368002B02D013684A
:100EE000013B13605B4A1368002B02D01368013B7F
:100EF000136000F091FD584B1B68002B04D1574B39
:100F00001B68002B00D197E008F012F8041C08F0D1
:100F10001DF8231C0340524C002B2DD02268514B4E
:100F20009A420ED14C4B1B68002B06D14B4B1B68D1
:100F3000002B02D1FA22920000E0FA22484B1A60FC
:100F40001CE02368484DAB4218D02368013B236066
:100F50002368002B04D0FA2322689B009A420DD903
:100F60000BF0CCFA002804D0256005200BF044F8E3
:100F700004E000F065FD01E03A4B23603B4B1B6849
:100F8000DA0704D5A0231B061B68590701D500F01A
:100F900057FD374C2368002B2ED020F09BFB0028F8
:100FA00026D10BF087FA002822D108F065F9002835
:100FB0001ED108F06BF900281AD100F00FFA0028B2
:100FC00016D107F0B5FF002812D107F0BFFF0028A7
:100FD0000ED12368013B23602368002B0CD1254BE5
:100FE0001A6801239340244A13600BF011FB03E0BD
:100FF000224B1A681E4B1A60214C2268002A0DD021
:10100000154B1B68002B05D01E4B9A4202D91E4B74
:101010009A4203D91D4B1A6000F03EF81C4B043471
:101020009C42EAD11B4B00221A80042252420C3B04
:101030001A8030BC01BC004707F07AFF041C07F09F
:1010400085FF231C034366E7E4BF0162E0BF016242
:10105000E4520162E0520162A453016284580162C9
:10106000D06F00205A5A0000A5A50000080000A07B
:10107000DC52016204F8FFFF40F8FFFFD852016222
:1010800084520162FFFF0040FEFF03400C0001623A
:10109000D45201621C9000E01047C046054B042268
:1010A00052421A80052208331A805022043B1A80CB
:1010B0007047000010C000E010B50E4B9B7A041C76
:1010C0009A0703D50BF0F6F9002810D1002C09D0AF
:1010D000094B1A8809491204120C0A431204120C13
:1010E0001A8004E00449064B0A8813400B8010BCA8
:1010F00001BC00473C0001620C5000E00080FFFF93
:10110000FF7F000010B50F4B9B7A041C9A0703D594
:101110000BF0D0F9002811D1002C0AD00A4B1A8804
:1011200080211204120CC9010A431204120C1A8005
:1011300004E00549054B0A8813400B8010BC01BC34
:10114000004700003C0001620C5000E0FFBF0000BF
:1011500000280AD0084B1A8880211204120C890139
:101160000A431204120C1A8004E00349034B0A8854
:1011700013400B80704700000C5000E0FFDF0000C0
:10118000144B1B881B04002B07DA134B1B88984257
:1011900003D1124B1B8899421BD002040E4B120C38
:1011A0001A8009040D4B090C198004200C4B404295
:1011B000053A188012040833052005391880120CEE
:1011C0000C3B09041A80090C043B064A19800C33B5
:1011D0001A80704714C000E0EA520162E8520162CE
:1011E00010C000E05082FFFF30B509040004090C74
:1011F000030C02290ED0022902D8012906D107E0EA
:10120000032909D0042901D15A2506E0322504E03A
:10121000632502E0622500E06125191C07482AF0D9
:10122000D7FA041C281C604364212AF08BFA011CA5
:10123000201CFFF7A5FF30BC01BC0047804F120007
:1012400030B5051C0C1C00291ED11123184206D0F4
:101250000020FFF731FF274B1C80274B1C802223E7
:101260001D4206D00020FFF74DFF244B1C80244B6D
:101270001C8044231D423AD00020FFF769FF214B18
:101280001C80214B1C8032E0112318420DD001201C
:10129000FFF712FF2304174A1B0C1380EB0601D53E
:1012A0000A2200E00022144B1A8022231D420DD096
:1012B0000120FFF727FF2304104A1B0C1380AB0605
:1012C00001D50A2200E000220D4B1A8044231D4262
:1012D0000DD00120FFF73CFF23040A4A1B0C1380AA
:1012E0006B0601D50A2200E00022074B1A8030BCB1
:1012F00001BC0047545301625053016252530162D2
:101300004E5301624C5301624A5301620EB4F0B570
:1013100085B00A9D0190022D10D0022D02DC012D16
:1013200010D108E0032D02D0042D0BD101E0612281
:1013300002E05A2309E06322029207E0622304E0FC
:10134000039A26E0002D37D0322302930BAB002600
:10135000049317E0721C4B1E1A4CB7000092012B2D
:1013600002D8161C39510CE017482AF0EBF9029B01
:101370003851642158432AF0E5F9009A9300185136
:101380000236039B19681A1D03920029D8D0132E28
:10139000E0DD04920B4AB30000219950019A130634
:1013A0000A4A1B0E13700A4A2B061B0E1370094BB8
:1013B000094A19600123138005B0F0BC08BC03B0D2
:1013C00018470000EC520162804F12004053016246
:1013D000415301624453016248530162034B188830
:1013E0000004000C4042C00F7047000048530162E7
:1013F000154B1A881B881204120C1B041349524205
:101400001B0CD00F8B4201D108231843104A1388BC
:101410001B04002B01D00223184313881B041B0C50
:101420008B4201D1802318430A4A13881B04002BE6
:1014300001D00423184313881B041B0C8B4202D1D8
:1014400080231B011843704754530162FFFF0000C3
:10145000525301624C53016200B50D4B5B79082B6E
:1014600011D80C4A9B009B589F4601210CE0032198
:101470000AE0052108E0142106E0192104E02821F2
:1014800002E0642100E00A21FFF7DAFE01BC004718
:101490003C00016240A00360094B1A79C0231A4046
:1014A000402A0AD0C02A02D0002A04D001E00A2033
:1014B00004E0052002E0012000E003207047000066
:1014C0003C00016270B577490B88774A1B041B0CFE
:1014D000934213D00B881B04002B0FD00B88734A48
:1014E0001B049B181B0C0B800B881B041C0C002C72
:1014F00004D10020FFF7E0FD6D4B1C806D490B8887
:10150000694A1B041B0C934213D00B881B04002B4D
:101510000FD00B88654A1B049B181B0C0B800B8893
:101520001B041C0C002C04D10020FFF7EBFD624BC8
:101530001C8062490B885C4A1B041B0C934213D02D
:101540000B881B04002B0FD00B88584A1B049B18D8
:101550001B0C0B800B881B041C0C002C04D10020DE
:10156000FFF7F6FD564B1C80534C23881B04002BC1
:1015700016D023884D4A1B049B181B0C23802388FC
:101580001B04002B0CD14F4B1A888023DB01134224
:1015900001D0002000E00120FFF7B4FD0A232380E2
:1015A000434C23881B04002B15D023883F4A1B047F
:1015B0009B181B0C238023881B04002B0BD1414B51
:1015C0001B881B04002B01DA002000E00120FFF73C
:1015D00073FD0A2323803A4C23881B04002B16D06A
:1015E0002388324A1B049B181B0C238023881B046E
:1015F000002B0CD1334B1A8880239B01134201D05E
:10160000002000E00120FFF7A3FD0A2323802E4ED7
:1016100033881B04002B42D03388244A1B049B18B8
:101620001B0C338033881B041D0C002D37D1274839
:10163000036827499A00545801330360022C05D1EE
:10164000056003689A00013354580360002C02D0EF
:10165000012C17D10AE01F4B042252421A800522A6
:1016600008331A805022043B1A8018E0194B0422D8
:1016700052421A800521083319805022043B1A80F7
:1016800031800CE003689A00013351580360201C3C
:10169000FFF776FD104B1B781B061B0E338070BCCA
:1016A00001BC004754530162FFFF00000000FFFF30
:1016B00050530162525301624E5301624C53016216
:1016C0004A5301620C5000E04853016244530162E6
:1016D000EC52016210C000E04053016200B51B48AB
:1016E000FFF75AFB1A4B002018801B88194A1B046D
:1016F0001B0C13801388184A1B041B0C13801388BF
:10170000164A1B041B0C13801549164B0A881340FC
:101710000B80154B0A8813400B80144B18801B88D4
:10172000134A1B041B0C1380124B0A8813400B80B6
:101730000422114B52421A80052208331A80043BBE
:1017400050221A800D4B188001BC0047C514006060
:101750004E5301625053016252530162545301626D
:101760000C5000E0FF7F0000FFBF00004A53016201
:101770004C530162FFDF000010C000E048530162DB
:1017800000B5084B1B791A0709D4074B1B881B04AB
:10179000002B04D101200321044AFFF7B7FD01BC4F
:1017A000004700003C00016248530162C409000088
:1017B00000B50E4B1A79130716D4C0231340402BE3
:1017C0000AD0C02B02D0002B04D001E00A2004E094
:1017D000052002E0012000E00320FA22400005215C
:1017E00092000023FFF792FD01BC00473C0001621C
:1017F0007047000070B5174D174C184B184A2978E0
:1018000020781B78127809060006000E1B061206C7
:10181000090C120E01431B0C13430E1C1E40002327
:101820002B7023700F4C0025331C2B41DA0706D593
:101830002268002A03D00C4B1A6000F037F90135FA
:101840000434102DF0D1094B00221A7070BC01BC79
:1018500000470000381000E03C1000E0281000E0D5
:101860002C1000E05C5301620C0001621C1000E0CF
:1018700030B50004000C8400E263084D01232A689F
:1018800083401A43064BE4180F2319408004084391
:101890002A60206030BC01BC0047000020F8FFFF38
:1018A00060F8FFFF10B51E4B00211960203319604E
:1018B0001C4A01235B4213601B4B0C221A60143B31
:1018C000196010331960194B194A196019481A4CDC
:1018D0008B04136001311319186004322029F6D1EA
:1018E0000F4B01221A60154A111C4031002308C217
:1018F0008A42FBD1124A05200C21FFF7B9FF11499A
:101900000B781B0602221B0E13431B061B0E0B70CB
:101910000D4B1A6828231A6010BC01BC0047000058
:1019200000F8FFFF40F8FFFF1CF8FFFF585301626B
:1019300060F8FFFFF1170060DC0700005C530162F4
:10194000F5170060241000E0100100600749000452
:101950000A68000C012383409A43054B80000A600B
:10196000C21800231360034BC363704720F8FFFFC6
:1019700060F8FFFFF1170060F0B506048024360C14
:1019800064020D04B440240C2D0C201C00212D06F3
:10199000171C2D0E00F0C8F8201C00F007F9291CB8
:1019A000201C00F09BF8054BB600F750201C0121CD
:1019B00000F0BAF8F0BC01BC004700005C530162C3
:1019C00000DF704701DF70470349044B0A681A6063
:1019D00000230B607047000020F8FFFF585301629E
:1019E0000348044A016813680B431360036070479F
:1019F00020F8FFFF58530162064BFF221A80012294
:101A0000524204331A8001220C331A800322143B01
:101A10001A80704704E000E0024B034A1A80034A30
:101A20001A80704718E000E05AA5FFFFA55A000091
:101A3000024A00231380143A1380704714E000E038
:101A4000A0221206136804490B43136003490B6874
:101A5000022213430B60704708080000200000A01A
:101A600000B50F4B00221A80143B1A801420FFF798
:101A70001FF90AF031FD032805D1092000F0D6F83E
:101A80003220FFF715F9A0221206136805490B430F
:101A9000136005490B68022213430B6001BC004729
:101AA00014E000E008080000200000A01047C04635
:101AB000094B00221A700C331A7004331A70043365
:101AC0001A7004331A7004331A7004331A70183BF6
:101AD0001A701A70704700001C1000E010B5000466
:101AE0000906040C000E00290BD10E4A13781B06C0
:101AF0001B0EA3431370043A13781B061B0E83437B
:101B00000CE0084A13781B061B0E23431B061B0E12
:101B10001370043A13781B061B0E0343137010BC9A
:101B200001BC0047341000E010B500040904040CA7
:101B3000000E00290DD00E4A13781B061B0E2343FE
:101B40001B061B0E1370043A13781B061B0E03436F
:101B50000AE0074A13781B061B0EA3431370043ACE
:101B600013781B061B0E8343137010BC01BC004787
:101B70002C1000E0064A1378000609041B06000E2C
:101B80001B0E090C8343012900D1034313707047D6
:101B9000241000E0044B1878043B1B7800061B0659
:101BA0001B0C000E184370473C1000E0074A1378E6
:101BB00000041B06010C1B0E8B431370043A1378B0
:101BC0001B06000E1B0E8343137070473C1000E091
:101BD000024B01221A7000221A7070471C1000E09C
:101BE000032807D0052805D00C2803D00D2801D0E4
:101BF000002000E00120704700B596210902002274
:101C0000074800F039FB48F08DF8064848F08EF898
:101C1000054A01235B4213600AF0E0F901BC00476A
:101C2000004000C00DC20060D46F002010B5041C3D
:101C3000FFF7D6FF002802D0201C1FF0CDFD092C95
:101C400008D1094B1B68023304D0C02048F072F859
:101C500048F074F8044A01235B421360034800F023
:101C600021FC10BC01BC0047D46F0020004000C024
:101C700000B50AF031FC002806D0032801D1092064
:101C800003E00120404200E0022002BC08470000BF
:101C900030B50906041C0D0E81B003200021FFF7AA
:101CA000ADF8002C04D1FFF7E3FF041C431C25D042
:101CB000201CFFF795FF002807D02004000C291CEA
:101CC0001FF04AFF00281CD118E0092C11D16846EA
:101CD00003300570012148F035F8002804DC0DE0E0
:101CE0000AF0FAFB032809D148F030F84307F7D58A
:101CF00007E00648291C00F0DBFB02E0012040421F
:101D000000E0002001B030BC02BC0847004000C029
:101D100000B50006010E06480368002B02DA012018
:101D2000404202E00068FFF7B3FF02BC0847000032
:101D3000D46F002070B50B041D0C1D4B81B0041C2A
:101D40000E1C1D80002805D009E0194B1B881B04C0
:101D5000002B26D0FFF78CFF041C431CF5D0201C61
:101D6000FFF73EFF002805D02004291C000C1FF0BF
:101D7000EDFC18E0092C0FD16C460334201C012126
:101D800047F0E8FF002805DC094B1B881B04002BEB
:101D900007D0F1E7207806E0311C064800F092FBFE
:101DA00001E00120404201B070BC02BC08470000C5
:101DB00016000162004000C000B5011C0548036820
:101DC000002B02DA0120404202E00068FFF7B2FF78
:101DD00002BC0847D46F002000B50C480368002BF4
:101DE00002D00368002B04DAFFF742FF431C01D145
:101DF00006E00068092803D1402047F09BFF02E07D
:101E0000034800F01BFA01BC00470000D46F00201B
:101E1000004000C010B5041C431C02D1134B1868CD
:101E200020E0FFF7DDFE00280AD0201C1FF004FD93
:101E3000002802D00120404214E00C4B1C6010E04E
:101E4000092C04D147F06EFF094847F06FFF074B9C
:101E50001C60084B0848D9689A7800F00DFAFFF723
:101E6000BBFF002010BC02BC08470000D46F00205C
:101E70000DC200603C000162004000C0014B1860D0
:101E8000704700009C53016270B52A4B1A68061C0B
:101E90000D1C002A0AD0284C2368012B06D00123F0
:101EA000236000F0C9F90023236040E0234C23683D
:101EB000002B38DB03200021FEF7A0FF2368002B56
:101EC00005D1FFF7D5FE041C431C01D12BE024688B
:101ED000201CFFF785FE002809D020042A04000CEE
:101EE000120C311C1FF05CFC002812D11BE0092CE5
:101EF0000FD1301C291C47F025FFA84213DB03E05B
:101F00000AF0EAFA03280ED147F020FF4307F7D57D
:101F10000CE0002404E0315D094800F0C9FA013406
:101F2000AC42F8DB02E00120404200E0002070BC3F
:101F300002BC08479C530162A0530162D46F002089
:101F4000004000C010B5041C24F0FEFA011C201C47
:101F5000FFF79AFF10BC02BC0847000000B5090457
:101F6000090CFFF791FF01BC0047000070B5051C8C
:101F70000E1C0AF0B1FA032801D0002409E0281C45
:101F8000311C47F0DFFE07E0295D054800F090FABC
:101F90000134B442F8DB002070BC02BC08470000EA
:101FA000004000C030B51A4C051C2068FFF718FE31
:101FB000002803D0281C1FF021FB26E02368092BF2
:101FC00006D02368002B20D10AF086FA03281CD102
:101FD00047F0BCFEC30409D5002D07D147F0B6FE7B
:101FE000830401D502200EE000200CE047F0AEFE95
:101FF000C3040AD4002D08D047F0A8FE830401D5FD
:10200000032000E0012047F095FE30BC01BC0047F2
:10201000D46F002010B50E4C2068FFF7E1FD0028BA
:1020200002D01FF0F1FA10E02368092B06D02368D4
:10203000002B09D10AF050FA032805D147F086FE9B
:10204000C30501D4012000E0002010BC02BC0847F9
:10205000D46F002010B50E4C2068FFF7C1FD00289A
:1020600002D01FF0DDFA10E02368092B06D02368A8
:10207000002B09D10AF030FA032805D147F066FE9B
:10208000830501D4012000E0002010BC02BC0847F9
:10209000D46F002030B51A4C051C2068FFF7A0FD56
:1020A000002803D0281C1FF0B5FA26E02368092B6E
:1020B00006D02368002B20D10AF00EFA03281CD189
:1020C00047F044FE830409D5002D07D047F03EFEBB
:1020D000C30401D501200EE000200CE047F036FEDD
:1020E00083040AD4002D08D147F030FEC30401D583
:1020F000032000E0022047F01DFE30BC01BC004779
:10210000D46F002030B509060B01090F051C1B0F09
:10211000092901D9373100E03031092B02D91C1CC3
:10212000373401E01C1C3034281CFFF7B1FD281C9B
:10213000211CFFF7ADFD30BC01BC004700B5000617
:10214000010E04480368002B02DB0068FFF7DAFF8A
:1021500001BC0047D46F002010B50906041C090E0D
:10216000FFF7D0FF201C2021FFF792FD10BC01BC1F
:102170000047000000B50006010E04480368002B6C
:1021800002DB0068FFF7E8FF01BC0047D46F0020C6
:1021900030B509040D0C2D06041C2D0E090EFFF799
:1021A000B1FF291C201CFFF7ADFF201C2C21FFF7DD
:1021B0006FFD30BC01BC004700B50004010C0448B1
:1021C0000368002B02DB0068FFF7E2FF01BC004759
:1021D000D46F002010B5041C0AF07EF9032804D146
:1021E000201C47F0BBFD092002E0002323600220F1
:1021F00010BC02BC0847000000B50B490B68012B5E
:102200000ED90A68531C0B60032A03D0042A05D197
:10221000064B01E0064B1B68036003E0054BFBE740
:1022200047F09CFD01BC0047A453016200D4016249
:10223000FC2F0162E8BF01621047C0460A4B98427A
:1022400001D10A4A03E00A4B984206D1094A002309
:10225000538053881B041B0C138001235B420384AF
:102260008384038970470000004000C08C53002025
:10227000005000C0C449002070B583891B04151CA0
:102280001B0C802213431B041B0C83818389802237
:102290001B04D2001B0C13431B041B0C8381012362
:1022A0005B4283840384674B82891340061C8381CD
:1022B00004200C1C00F00AFB24014000211C29F022
:1022C00041FA0130C003000C30805F4BB2891340EB
:1022D000B381B3891B041B0C092213431B041B0C81
:1022E000B381C0231D4011D0B3891B041B0C0722EE
:1022F00013431B041B0CB381802D07D1B3891B042E
:102300001B0C202213431B041B0CB381B3898024B4
:102310001B0464001B0C23431B041B0CB381301CE7
:10232000FFF78CFFB3891B041B0C23431B041B0CFE
:10233000B381338A1B0401221B0C13431B041B0CA7
:1023400033824248FEF728FD414B9E4216D1414A56
:102350000C210920FFF78CFA3F4A404913880B40B3
:102360001380043213881B041B0C23431B041B0C17
:10237000138004321388194011805FE0384B9E426D
:102380005CD1384A0A200C21FFF772FA32483649EC
:1023900003880B400380354D2B8880221B04D2001C
:1023A0001B0C13431B041B0C2B80314C238819403E
:1023B0002180038880221B0412011B0C13431B0481
:1023C0001B0C03802B881B041B0C13431B041B0CCE
:1023D0002B8023881B041B0C13431B041B0C238022
:1023E000244D25492B880B402B80244C23888022A8
:1023F0001B04D2011B0C13431B041B0C238020481D
:102400000388194001802B881E491B041B0C0B43B9
:102410001B041B0C2B801C4B228813402380038839
:102420001B041B0C0B431B041B0C0380174A138853
:102430001B041B0C0B431B041B0C138070BC01BC46
:1024400000470000BFFF0000C0FF000061250060E2
:10245000004000C09D250060003000E0FFFE00004D
:10246000005000C011260060FFFB0000043000E0B7
:10247000083000E0004000E0FFBF0000044000E042
:10248000084000E00080FFFFFF7F00000C4000E0FC
:1024900000B5034BD9689A78FFF7EEFE01BC004700
:1024A0003C00016200B5FFF7C9FE01BC0047000017
:1024B0000906090E81808023828A9B001342FAD18B
:1024C000704700001F4B984210D10B041E4A1B0C92
:1024D00013801E490A884B8812041B04934219D1A9
:1024E000194B1B881B04002B28D0F2E7184B98428D
:1024F00024D10B04174A1B0C138017490A884B88F8
:1025000012041B04934205D1124B1B881B04002BA1
:1025100014D0F2E74A881204120C53180132120444
:102520001B79120C4A801B06180E4B880B4A1B04A1
:102530001B0C934204D100234B8001E00120404258
:1025400070470000004000C0160001628C5300205C
:10255000005000C018000162C4490020C4090000F6
:102560000B4A13881B04002B05D0138809491B0450
:102570005B181B0C1380084A13881B04002B05D022
:10258000138804491B045B181B0C13807047000060
:10259000160001620000FFFF1800016230B5184B01
:1025A0001B68DA0728D5174B1B881B041C0C8023DB
:1025B0009B00251C1D401FD109F08EFF002805D06F
:1025C00001204042FFF726FC022815D12406240EE4
:1025D000201C09F01BFE0C490B881B041B0C5A180D
:1025E00001331B041B0C14710B800B88074A1B045E
:1025F0001B0C934200D10D8030BC01BC0047000091
:10260000144000C0084000C08C530020C4090000E2
:1026100010B5134B1B68DA071FD51248124B1B88E5
:102620001B041A0C80239B00141C1C4011D103882E
:102630001B041B0C1918013312061B04120E1B0C71
:102640000A7103800388094A1B041B0C934200D1C2
:102650000480034B1B68DA07E0D410BC01BC0047C0
:10266000145000C0C4490020085000C0C409000034
:1026700010B50B4C23881B04302200061B0C93431F
:10268000000D0343072209069343090E873A1143BD
:102690000906090E1943218010BC01BC0047000047
:1026A0004C0000A00006000E01280FD0012822D304
:1026B000022802D003283ED137E01F490B680122CF
:1026C00093430B600B680822134303E01A490B681D
:1026D000082293430B60A0221206136804218B4347
:1026E000136016490B680722934303221343802289
:1026F00093430B601FE010490B68082213430B60E3
:102700000E4B1B6807221340072B03D00A4B1B6894
:102710009A07FBD5A0221206136804218B4313608D
:1027200005490B6801221343E3E7A0231B061A683F
:1027300004210A431A607047080000A0180000A096
:10274000A0231B061B68590701D503200BE0064A8E
:102750001368190701D4012005E01368DA0701D5D1
:10276000002000E002207047080000A0034B1B88F7
:10277000DB050020002B00DA012070474C0000A090
:10278000044B1B680120DB0B9843012358400006D3
:10279000000E7047080000A00004000C012806D1BC
:1027A000064980230A681B021A430A6004E0034BAF
:1027B00003491A680A401A6070470000080000A028
:1027C000FF7FFFFF05490B881B04032200061B0C3B
:1027D000000E934303430B8070470000400000A0AD
:1027E00005490B881B04032200061B0C000E9343B3
:1027F00003430B8070470000440000A005490B888C
:10280000054A1B0400061B0C1340000C03430B80FD
:1028100070470000440000A0FFFCFFFF05490B8843
:10282000054A1B0400061B0C1340000C03430B80DD
:10283000704700004C0000A0FFFEFFFF09040004E9
:10284000090C000C012904D1A022120613680343CD
:1028500003E0A02212061368834313607047000050
:10286000034B00041B68000C184000D00120704787
:10287000080000A0034A00041368000C034313601F
:1028800070470000080000A00F4B1A68DC23DB0033
:10289000101C1840802814D0802804D820280CD080
:1028A000402808D10BE080239B0098420AD0802367
:1028B000DB00984206D0002004E0202002E0402007
:1028C00000E0802070470000080000A030B52D4BCC
:1028D0001A680123D20B93430122534000061B06C2
:1028E000040E002B01D0284D00E0284D002C2CD0E8
:1028F000FFF726FF01280DD001280DD3022824D090
:10290000032804D18025012101202D021FE0002190
:1029100000201CE0102119E01D4B1B689B06980F3E
:10292000012809D0012805D3022807D0032806D1A1
:10293000102004E0142002E00C2000E01820144BCA
:102940001B6807221340591C01E001210120032CC0
:1029500005D0042C08D0022C0DD10E4B05E00E4BF7
:102960001B889B059B0F03E00B4B1A880323134026
:1029700099400B06190E684328F0E4FE30BC02BCF7
:1029800008470000080000A080841E0000093D00E8
:10299000180000A0400000A0440000A030B50006D0
:1029A0000906040E00200D0EFFF790FF0D4B984214
:1029B00004D90D4B1A6880210A4303E00A4B1A68B8
:1029C00080218A431A6008490B6830229343220110
:1029D0001343072293432B43402213430B6030BC25
:1029E00001BC0047C0C62D00180000A0D022000680
:1029F0001206030E80180906000E090E092801D8D8
:102A0000021C02E0373B1B061A0E0B1C303B1B0658
:102A1000180E092803D90B1C373B1B06180E13018F
:102A200018430006000E7047F0B5164B5C681B6833
:102A300083B00093019400230293067981783306D2
:102A40001B0E027847788C46C5786C4602A94079FF
:102A5000592B04D81306FA221B0ED20002E01306EB
:102A6000094A1B0E9B180093634667710D704E70E8
:102A700088702371684600F007FE03B0F0BC01BC0B
:102A80000047000090A003606C07000000B5044BF5
:102A90000106090E1868FFF7FBF801BC00470000AB
:102AA000A8530162F0B5CC4B1B688BB0002B00D053
:102AB000DDE201204042FFF7ADF9C84A106011681D
:102AC0000D290CD801238B40191CC54B194203D189
:102AD000C44B194209D102E01068FFF7A7F80020A3
:102AE000FFF798F9BD4A00231360BF498B7A022291
:102AF00093438B7204200021FEF7A2FB01213020BA
:102B00004942FEF79DFB0020002108F00BF8002051
:102B10000021FEF773F9002047F008F9AE4A0123BF
:102B20001360002205920692089207920BE015208E
:102B3000FFF7ACFF01200521AC4A0023FEF7E6FBBE
:102B400001E001220892AA4B00221A60A94B1A60E8
:102B5000A94B0993A14C32212068FFF7EBF810280C
:102B600000D095E0A24A00231360A24A012313601B
:102B70009A4B32211868FFF7DDF80028EADB9C4EFB
:102B80003268012A19D0012A02D3022A6DD147E006
:102B90009849102803D10B680122534020E00B68AC
:102BA000002BD7D000220A600228D3D10123336042
:102BB000924B1A60924A1223D9E7914C03061D0EDC
:102BC00023686B4023608B4910280DD10B68012BC3
:102BD00008D100230B6089498A4A0B689D54013350
:102BE0000B60C5E70A60C3E70B68002B11D0002516
:102BF0000D60022802D0032809D105E07F4B1D603B
:102C0000122332602360B3E702233360B0E73560FC
:102C1000A0E77A4B7B491A68555401321A60A7E73E
:102C2000774B02061B68120E934207D1704B0022AD
:102C30001A60724B1C68032C25D91BE003280DD1A8
:102C40006E4B1B68012B09D16E4B1A78002A05D1F7
:102C5000674B06201A60FFF719FF7BE71520FFF787
:102C600015FF634A0023136074E7624B0022326051
:102C70001A606FE763486449032223F0BBFC002815
:102C800001D10427C7E0042C00D863E70327C2E082
:102C90001B2850D120683221FFF74CF85A280FD159
:102CA00020683221FFF746F8312800D052E720682B
:102CB0003221FFF73FF80D2800D04BE70127AAE0AB
:102CC000582800D046E720683221FFF733F84C2817
:102CD00000D03FE720683221FFF72CF8542800D0BD
:102CE00038E720683221FFF725F804380A2800D990
:102CF00030E7464A83009B589F460527ADE10627EB
:102D0000ABE10727A9E10AF045FA0026051C2B785C
:102D1000A34200D01EE7314B32211868FFF70AF8B2
:102D2000731C1B041E0C041C0135062EEFD10D284C
:102D300000D00FE76CE03A2800D00BE72368032BA4
:102D400000D107E72368052B00D103E72068322173
:102D5000FEF7F0FF0004050C002800DAFAE6322145
:102D60002068FEF7E7FF0004010C002800DAF1E616
:102D700028060906000E090EFFF738FE099A1070A2
:102D8000043000040132070C002609921FE0134CA6
:102D900032212068FEF7CEFF0004050C002800DA7F
:102DA000D8E632212068FEF7C5FF0004010C002898
:102DB00000DACFE628060906000E090EFFF716FE18
:102DC000099B187001330993731C1B041E0CBE422F
:102DD000DDD102271FE00000A4530162A853016265
:102DE00028300000050200003C000162C409000018
:102DF000B8530162B4530162F4530162F0530162AB
:102E0000B0530162BC5301620083046098A0036068
:102E10007A1C00D197E6984C2368002B02D1FEF76C
:102E200027FF20607B1E072B00D98CE6934A9B006E
:102E30009B589F46924B1A78FF2105320A4000208A
:102E400000211C1C04E01B5DC3181B04180C01317D
:102E50000B041B0C9342F6D3FF230022184200D12F
:102E60000122002A00D1C8E0854BDB78052B00D970
:102E7000C3E0844A9B009B589F46814D069A6B781D
:102E80001104AA781B0213430E1C1E43059B002B42
:102E900000D105962C1D2D78211C2A1C301C21F0F8
:102EA000FFFB301C211C2A1C21F0CCFB002800D089
:102EB0003DE60620FFF7EAFD45E6714B1A795B799E
:102EC0001202D2181204120C0692F2E70620FFF743
:102ED000DDFD6D4A00231360059A01239A436B4B75
:102EE00005921A6000F0EEF82DE665490B794A79F3
:102EF0001B029B188A79C97912021B051B0C5218F8
:102F0000D21806930592D4E75D490B794A791B02E2
:102F10009B188A791B029B18CA791B029B18059380
:102F2000C7E75B4A1368053B13605A4E1B041D0C30
:102F300073780AAAD370B3789370F37853703379A7
:102F400013700A9CA0231B06E218534B9A4203D825
:102F5000701D211C2A1C4DE0504B9C4227D9504B20
:102F600062199A4223D8201C0CF092FE079A041C86
:102F7000024205D10A980CF003FF079B23430793F5
:102F80000A98401901380CF083FE079A041C02428B
:102F900007D10A98401901380CF0F2FE079B234331
:102FA0000793701D0A992A1C0CF064FF81E73D4BC2
:102FB0009C4222D93C4B62199A421ED83B49201CA4
:102FC0002A1C21F06DFB74E7324BDB78013B072BA9
:102FD00013D8374A9B009B589F462E4B187900F018
:102FE000DBF866E73348FFF71FFD62E7C021324890
:102FF000C905042200F0C0F95BE715205AE701F08B
:103000007DFAA0E50620FFF741FD2C492C4B0091ED
:103010000391FA22002192000491052005210192DA
:103020000293FEF773F91E20FDF742FEFEF718FD2E
:1030300089E5089A002A0CD10AF0ACF80024051C96
:10304000285D0134FFF722FD062CF9D10D20FFF792
:103050001DFD0023089376E50827074B32211868E9
:10306000FEF768FE041C0D2800D1D1E64BE60BB03C
:10307000F0BC01BC00470000A8530162C4A003607B
:10308000F4530162E4A00360A4530162AC530162F3
:10309000F0530162BC530162FFFF3F00FFFFFF3F9F
:1030A000FF3F0C40FFFFFF6100001062C15301624F
:1030B000FCA00360C053016204830460AC0D0000F7
:1030C000C40900001047C04610B5FEF779FC254B37
:1030D00000F09EF9041CFEF775FC234B234A802167
:1030E0001C60490023141180BF2B38D1204B201CB9
:1030F0001840204B98422DD098420FDC1F3B98423D
:1031000022D0984203DC013B984226D11CE01A4BA6
:1031100098421CD0013398421FD118E09E239B0196
:1031200098420DD0984203DC144B984215D111E01F
:10313000134B984206D0083398420ED140230BE03F
:10314000802309E0118008E080239B0004E08023B5
:10315000DB0001E080231B0113800CF087FD10BC15
:1031600001BC0047717D0020200001621C0001624B
:10317000FFFF00006A2300005A2300006B230000B9
:10318000812700008020C00370470000014B1868B1
:10319000704700002000016230B50F4B1A88041CF4
:1031A000531E00D50F331B119C4212DCFEF708FCA6
:1031B000C0222304D2059C181025201C074B00F0C8
:1031C00027F980235B01013DE418002DF5D1FEF7BE
:1031D000F9FB30BC01BC00471C000162E97C002007
:1031E00000B580231B0118420CD1032815DD0C4BC0
:1031F0001A88531E00D50F331B1198420DDCFFF7C0
:10320000CBFF0AE0984208DD064B984205DC064BEE
:1032100018400004000C0CF0C1FD01BC0047000088
:103220001C00016203080000FFF7FFFF10B50A4B06
:103230001B88013B041C98420ADCFEF7C1FBC0233B
:10324000DB052003C018054B00F0E2F8FEF7BAFBDF
:1032500010BC01BC004700001C000162E97C00209A
:1032600000B503050ED43F281BDD0F4B1A88531EF3
:1032700000D50F331B111B011033984211DAFFF7F1
:10328000D5FF0EE0094B1840062805D0072805D0C9
:10329000052806D1064802E0064800E006480CF082
:1032A0006FFD01BC004700001C000162FFF7FFFF3B
:1032B00000000140000002400000034030B50D0452
:1032C000041C2D0CFEF77CFB281C211C034B00F07A
:1032D0009FF8FEF777FB30BC01BC0047317D002032
:1032E00000B50906090EC30705D5013802780B029F
:1032F000111C194304E00288FF231B021A401143EA
:10330000FFF7DCFF01BC004700B5094BC218094BB1
:103310000906090E9A4202D8FFF7E2FF06E0064BC3
:10332000C218064B9A4201D80CF06AFD01BC004756
:103330000000FC9FFEFF03000000FFBFFEFF020035
:1033400000B5094BC218094B0904090C9A4202D86E
:10335000FFF7B4FF06E0064BC218064B9A4201D8AD
:103360000CF034FD01BC00470000FC9FFEFF030091
:103370000000FFBFFEFF0200F0B50127061C0D1C78
:10338000141C394206D00178281CFFF7A9FF01352B
:103390000136013C3C4204D0013C2819A15DFFF7F5
:1033A0009FFF002708E0737831781B02281C19431F
:1033B000FFF784FF023602353B041B0C0237A342A1
:1033C000F1D3F0BC01BC004710B50D4B141C994261
:1033D00007D90C4B8A189A4206D8221CFFF7CCFF5B
:1033E0000AE0094B994207D9084B0A199A4203D8B7
:1033F0002204120C0CF03EFD10BC01BC0047000082
:10340000FFFF0360FFFF0760FFFF0040FFFF034077
:103410001847C04600B50F490A8820231342FAD046
:103420000B881B0410221B0C13431B041B0C0B806A
:10343000094B00221A80094A04331A80084B0A8873
:1034400013400B80074A03200221FEF711FA01BC4A
:103450000047000004D000E008D000E00080FFFF3B
:10346000EFFF000025350060064B1A882023134229
:10347000FAD0054B188804331B881B041B0C00046E
:103480001843704704D000E018D000E01F490A88B4
:1034900020231342FAD00B881B041B0C1022134369
:1034A0001B041B0C0B8019490A8820231342FAD0F5
:1034B0000A88174B13400B80144B1A8820231342A1
:1034C000FAD0144B1A881204120C0A210A4312046F
:1034D000120C1A800D4B1A8820231342FAD00304D1
:1034E0000D4A1B0C1380094B1A8820231342FAD073
:1034F0000A4B020C1A8005490A8820231342FAD08D
:103500000A88074B13400B807047000004D000E08E
:10351000F5FF000000D000E024D000E020D000E063
:10352000EFFF000000B5FFF79FFF034BC018FFF748
:10353000ADFF01BC00470000805101000378172B4C
:1035400007D843783B2B04D883783B2B01D8002045
:1035500001E001204042704710B50468174AA318E3
:10356000632B23D80179002920D043791806030E54
:103570000C2B1BD801220316101C9840104B18422C
:1035800006D1A5231B01184205D1430706D40DE03F
:103590001F290ED90AE01E290BD907E003231C427C
:1035A00002D11D2905D901E01C2902D90120404280
:1035B00000E0002010BC02BC0847000030F8FFFF0C
:1035C000AA15000000B50B7889B002934B780193DF
:1035D0008B780093037903934379013B0493054A65
:1035E000036868469B18059321F0FEF909B002BCF8
:1035F0000847000094F8FFFF70B5041C0D1CFFF78E
:1036000033FF291C061C201CFFF7DCFF864201D972
:10361000301A00E0801B70BC02BC084700B5FFF701
:10362000D1FF15490A8820231342FAD00B881B04C6
:103630001B0C102213431B041B0C0B800E4B1A880F
:1036400020231342FAD003040C4A1B0C13800A4BAC
:103650001A8820231342FAD0094B020C1A8006491B
:103660000A8820231342FAD00A88064B0020134010
:103670000B8002BC0847000004D000E01CD000E032
:1036800018D000E0EFFF000030B5041C0D1CFFF760
:1036900063FF013009D0281CFFF750FF013004D030
:1036A000201C291CFFF7BAFF01E00120404230BC7A
:1036B00002BC084730B58AB00D1C009001A96846CD
:1036C000141C20F03FFB039B2370029B6370019B43
:1036D000A370049B2B71059B01336B71034A069BFE
:1036E0000AB09B182B6030BC01BC00476C0700007F
:1036F00070B50C1C051C081C111C161CFFF762FF82
:10370000211C4019321CFFF7D5FF201CFFF724FFB6
:10371000002804D1301CFFF711FF002801D0012040
:10372000404270BC02BC084730B50D1C041CFFF7BA
:103730009BFE2A1C211CFFF7BDFF002030BC02BCF1
:103740000847000000B5FFF7EFFF01BC004700008D
:1037500000B582B0011C6846FFF7E6FF02B001BC6D
:103760000047000030B581B0051CFFF7F5FE0130C1
:1037700002D10120404206E06846FFF7E9FF281C1D
:103780006946FFF74BFF01B030BC02BC08470000A0
:1037900000B581B06946FFF7C7FF01B001BC004723
:1037A00030B582B0051CFFF7C9FE013002D10120FF
:1037B000404206E06846FFF7EBFF6846291CFFF72A
:1037C0002DFF02B030BC02BC0847000030B5090430
:1037D00082B0051C002926D11D490A8820231342E6
:1037E000FAD00B881B041B0C102213431B041B0C68
:1037F0000B8017490A8820231342FAD00A88154BF8
:1038000013400B80124B1A8820231342FAD0124B1C
:103810001B880F490A8820231342FAD00A880F4BCD
:1038200013400B8010E06846FFF7B2FF6846291C82
:10383000FFF7C8FE041CFFF717FE844201D2084BB5
:10384000E418201CFFF722FE02B030BC01BC004788
:1038500004D000E0F5FF000000D000E0EFFF000022
:103860008051010000B546F07DFA0C4B1A680C4BF4
:103870001168196051680B4B196091680A4B196007
:10388000D1680A4B19601169094B19605169094BDC
:1038900092691960084B1A6001BC00472800016258
:1038A00004000162340001622C00016230000162F8
:1038B00024000162380001620800016210B50A4C60
:1038C000FF21201C082220F067FF201CFF21082276
:1038D0001034083020F060FF201CFF21042220F06B
:1038E0005BFF10BC01BC0047DD01016204480549D3
:1038F0000022535C135401321C2AFAD17047000095
:103900006D0101629CA40360044A111C1C31002358
:10391000137001328A42FAD17047000089010162B6
:1039200000B50348FF21022220F036FF01BC00470A
:103930006B01016200B50348FF21382220F02CFF03
:1039400001BC0047A501016230B518490B7C402439
:1039500023430B74881CC37F3F2280256D42134094
:103960002B43C377CB7A202293431343CB724B7BF9
:103970006022934323434B738B79934323438B718F
:103980004B7D2B434B750B7E012213430B768B7FB4
:1039900003229343022213438B770631CB7F042209
:1039A0001343CB7730BC01BC0047000038010162F3
:1039B00000060906000E090E012A2CD1031C303B1B
:1039C0001B061B0E162B00D9A7E0031C3A3B1B0657
:1039D0001B0E062B00D8A0E00B1C303B1B061B0E59
:1039E000162B00D999E00B1C3A3B1B061B0E062B2D
:1039F00000D892E0392801DC302300E03723C31AD5
:103A00001801392901D8302300E03723CB1A1B06CF
:103A10001B0E184383E036282DD036280BD83128CA
:103A200017D0312804D8242858D0302875D109E07F
:103A3000352872D116E039282ED0512846D03728A3
:103A40006BD120E00B1C413B1B061B0E192B64D8CD
:103A500042E00B1C413B1B061B0E192B5DD8081CBA
:103A600040385CE00B1C413B1B061B0E0F2B54D84F
:103A7000081C213853E00B1C413B1B061B0E062B78
:103A80004BD8C81F4BE00B1C413B1B061B0E052BE4
:103A900043D8081C1A3042E0462912D0462902D8E1
:103AA00041293AD30AE0472906D00B1C543B1B0698
:103AB0001B0E032B31D806E0002030E0081C26380E
:103AC0002DE07F202BE0081C273028E00B1C303B2A
:103AD0001B061B0E092B20D8081C20E00B1C413BA9
:103AE0001B061B0E192B02D90120404201E0081CC5
:103AF0002030312901D1AD2011E0322901D1AF2090
:103B00000DE0332901D1AE2009E0342901D1AC20E8
:103B100005E0362903D1AB2001E001204042704787
:103B200000060906000E090E382834D0382804D8BB
:103B3000242864D037286AD104E039284AD056288E
:103B400065D14FE04839122961D8324A8B009B5821
:103B50009F46DE205DE0B1205BE0B22059E0B3205B
:103B600057E0B42055E0F32053E0B62051E0B720F1
:103B70004FE0BC204DE0FB204BE0D82049E0B820CE
:103B800047E0D92045E0DA2043E0DB2041E0DC20BB
:103B90003FE09F203DE04A390B2938D81E4A8B0070
:103BA0009B589F46D22034E0F02032E0E22030E003
:103BB000C9202EE0CA202CE0CB202AE0CC2028E02F
:103BC000CD2026E0CE2024E0F22022E0D02020E00C
:103BD000F1201EE0532903D0582918D1B02018E055
:103BE000BE2016E0522908D0532902D051290ED107
:103BF00001E0BB200DE0B9200BE0BA2009E0382934
:103C000003D0392903D1FC2003E0DF2001E00120AB
:103C100040427047C8C0036014C103600006010E33
:103C20000020064A835C8B4202D1531EC05C03E035
:103C300002306628F5D1FF207047000037A40360EA
:103C4000054B0006000EC0180138044A03789B1883
:103C50003433597070470000BDA40360380101621D
:103C6000054B0006000EC0180138044A03789B1863
:103C70005033597070470000BDA4036038010162E1
:103C800010B50D4B1C1C333400062278000E824206
:103C90000ED0191C34310B78834209D0FF2A04D08E
:103CA000FF2B04D00120404203E0207000E00870A8
:103CB000002010BC02BC0847380101620006074A18
:103CC000000E00211378834202D10B06180E04E087
:103CD00001310C322929F5D1FF207047E4A103609E
:103CE0000006020E000F092801D8302300E0372318
:103CF000C3180B70101C0F2318404A1C092801D848
:103D0000302300E03723C318137000238B707047F3
:103D1000024B1860024B0020196070472C5401625E
:103D200028540162F0B55D4A002313705C4A0123F8
:103D300013605C4B196882B0009000293AD05A4A4F
:103D40001368002B36D101235B421360574B1F6869
:103D500000220D1C019222E02C1C201C0099042240
:103D600022F048FC0C35061C002815D12289504B46
:103D700060689A4206D103F0ABFA002812DA4A4B87
:103D80001E6085E0217A03788B43627A0370616854
:103D90000B781A430A7005E0019B01330193019AE5
:103DA000BA42D9DB404A00231360404B019A1B689A
:103DB0009A426BD1009822F0C7FB032805D0042853
:103DC00005D0022864D100255CE0002530E0002603
:103DD0000027002514E0374BEC18201C0099042222
:103DE00022F008FC002808D1607AFF2802D1237A4B
:103DF000FF2B32D02F4BFB183CE001360C350C3733
:103E00001C2EE8D144E06B002B4A5B199B009C18E8
:103E1000201C0099032222F0EDFB002807D1607AD4
:103E2000FF2802D1237AFF2B17D0234A1EE0013549
:103E3000AA2DE8D12CE06B00204A5B199B009C184E
:103E4000201C0099022222F0D5FB002819D1607AAB
:103E5000FF280AD1237AFF2B07D1636803F039FAD0
:103E60000E4B1B78002B11D012E0144A6B005B192B
:103E70009B009B1859681A7A0B78934303430B7085
:103E800004E001350E4B9D42D5D101E0002001E058
:103E90000120404202B0F0BC02BC0847DE020162D1
:103EA000882301622C54016230540162285401625B
:103EB000FFFF0000E4A4036034A603602CAE03609F
:103EC0008D01000010B51548FFF72CFF1448FFF7CF
:103ED00029FF1448FFF726FF1348FFF723FF134875
:103EE000FFF720FF1248FFF71DFF124CE37E402230
:103EF0001343E3761048FFF715FF1048FFF712FF52
:103F0000237E042213432376E37C03229343E3744A
:103F1000FFF71AFD10BC01BC004700000C830460D1
:103F20001083046014830460188304601C8304609D
:103F300020830460380101622483046028830460C4
:103F400000B51148FFF7EEFE1048FFF7EBFE1048F2
:103F5000FFF7E8FE0F48FFF7E5FE0F48FFF7E2FE28
:103F60000E48FFF7DFFE0E48FFF7DCFE0D48FFF7B7
:103F7000D9FE0D49CB7C0122134302229343CB741B
:103F8000FFF7E2FC01BC00470C830460108304606F
:103F900014830460188304602C83046030830460FD
:103FA00024830460348304603801016270B50A4CD4
:103FB0000D1C00210AE00278135DDE0701D4131CFA
:103FC00001E0131C2033037001310130A942F2D308
:103FD00070BC01BC00470000F06D046070B50A4C75
:103FE0000D1C00210AE00278135D9E0701D4131C0A
:103FF00001E0131C203B037001310130A942F2D3D0
:1040000070BC01BC00470000F06D046070B50A4C44
:104010000D1C00210BE003781A5D960701D5203BAB
:1040200002E0D60701D52033037001300131A942E7
:10403000F1D370BC01BC0047F06D046070B5041C86
:104040000D1C002610E0921B201C611C20F028FB98
:104050002B68013B2B60227880231A4202D02A6809
:104060009642F0D3013401362B689E42F3D370BCE4
:1040700001BC004730B5041C0D1C06E0201C611C6F
:1040800020F00EFB2B68013B2B602378302B02D1F4
:104090002A68012AF2D830BC01BC00470006000E95
:1040A000C023184203D0044A9843831801E0034B0D
:1040B000C318013B18787047B8A40360BDA403601F
:1040C00010B500060906000E0C0EFFF7E7FF0D4BBA
:1040D00042009B181A1C011C6D3200201378FF2B24
:1040E00007D1084A4B001B189B186C3300205C70EA
:1040F00005E0013001320228F0D10120404210BC1D
:1041000002BC0847380101620906084B090E5B181A
:104110001A1C0006000EB9321C23013B1B061B0EA5
:1041200010700432002BF8D1704700003801016292
:104130000906084B090E5B18074900065A18000EBD
:104140001C23013B1B061B0E10700432002BF8D100
:1041500070470000380101622901000000B5074BDB
:104160000748084A186008231370FF21082220F02E
:1041700013FB054A0223137001BC00479823016218
:10418000DD010162612301623601016200B5074B66
:104190000748084A186008231370FF21082220F0FE
:1041A000FBFA054A0223137001BC00479823016201
:1041B000E5010162612301623601016200B5074B2E
:1041C0000748084A186004231370FF21042220F0D6
:1041D000E3FA054A0223137001BC004798230162E9
:1041E000ED010162612301623601016200B5022224
:1041F0000448FF2120F0D0FA034A0323137001BCC6
:10420000004700006B0101623601016200B50348FE
:10421000FF21022220F0C0FA01BC00476B010162BD
:1042200000B538220448FF2120F0B6FA034A0423DF
:10423000137001BC00470000A50101623601016254
:1042400000B5074B0748084A186010231370002177
:10425000102220F0A1FA054A0B23137001BC00477D
:10426000982301621A010162612301623601016231
:1042700030B5114B1B780D2B17D1104B1B78002B31
:1042800003D00F4B1A68002313700E4D0E4C281CE0
:10429000211C102222F0AEF9002806D0201C291C77
:1042A000102222F00BFA00232374034A0123137017
:1042B00030BC01BC0047000036010162612301628D
:1042C000982301621A0101628100016200B5074B67
:1042D0000748084A18600C23137000210C2220F0B4
:1042E0005BFA054A0C23137001BC00479823016256
:1042F0002A010162612301623601016270B50E4B31
:104300001E78002E12D10D4B1B780E2B0ED10C4DAA
:104310000C4C281C211C0C2222F06CF9002805D022
:10432000201C291C0C2222F0C9F92673034A012300
:10433000137070BC01BC0047612301623601016249
:104340002A010162740001620006000EC0231842B7
:1043500011D118280FD0182805D8431E1B061B0E94
:10436000072B06D807E01C2803D31D2803D92628CD
:1043700001D0002000E00120704700000B4B000638
:10438000000EC0180138007809490A4A4318825CB7
:1043900034335A703531084B084A401818600123ED
:1043A0001370074A0523137070470000BDA4036013
:1043B000380101629CA403609823016261230162B9
:1043C000360101620A4B0006000EC0180138007861
:1043D00008494318503300225A705131064B074A9E
:1043E0004018186001231370054A062313707047A4
:1043F000BDA4036038010162982301626123016258
:1044000036010162014A08231370704736010162C8
:104410000006010E0022064BD01803788B4201D112
:10442000407803E00232662AF5D1FF207047000091
:1044300036A403600006010E0022064BD018037854
:104440008B4201D1407803E00232662AF5D1FF2089
:1044500070470000D0A30360F0B5171C0F4A0E1C74
:1044600000250024116888420ED31379CB18984296
:104470000AD20B4BE25CE31832701A7A5B689B1825
:104480001B1A00203B7006E001350C340C32292D3C
:10449000E8D101204042F0BC02BC0847E8A103601B
:1044A000E4A1036000B589B0002368460230C3541C
:1044B0000133202BF9D16B460D220333DA7721210A
:1044C000FDF7E2FC09B001BC0047000000B599B05F
:1044D0006A4620230232137001331B061B0E013281
:1044E0007F2BF8D16B460D22613368461A7002307B
:1044F000FDF728FD19B001BC0047000030B586B0BB
:10450000FCF7E2FA051CFCF7EBFA6C460234031CDC
:104510002A1C0549201C21F0A7FE201CFDF712FDD6
:1045200006B030BC01BC00473883046030B5114A86
:10453000114982B0002504E01378EB181B041D0C10
:1045400001328A42F8D36C460334280A211CFFF753
:10455000C7FB28066946000E0531FFF7C1FB0D2396
:10456000201C05212371FDF78FFC02B030BC01BC7B
:10457000004700000000006040AE0460F0B584B069
:10458000151C02930A9A099B09061B0612061B0EAC
:10459000120E0C0E039001930092092C01D82020DA
:1045A00006E0201C0A2127F0CDF830300006000E6E
:1045B000039A0A211070201C27F05CF9039B30300D
:1045C0005870039A2023161C937003360024281C6D
:1045D00021F0BAFF844201D3202300E02B5D013497
:1045E0003370721C102C01D0161CF0E720231370BE
:1045F000009BB41CFF2B5AD09A00434B9B181D1CE8
:10460000341DB9350026A71E2878391CFFF768FB32
:1046100001362022227001350334042EF3D1A31E6B
:104620001A70009B9A00384B9B18384ABC1D9D1885
:104630000027A61E2878311CFFF752FB01372023E4
:10464000237001350334042FF3D12022A31E1A70E6
:1046500032712D4D009B5C19231C34335878711D29
:10466000FFF73EFB2022F2715034311C6078083194
:10467000FFF736FB2023B372F372009A5300341C09
:10468000ED180C346D35002620232370611C28782A
:104690000136FFF725FB03340135022EF4D1022247
:1046A0002023013A23700134002A07D0F8E72A2298
:1046B0002023013A23700134002AF9D1002614E0A6
:1046C000019F029BA51C013F002B04D0985D211C7B
:1046D000FFF706FB02E02023237063702C1CBE4210
:1046E00002D020232B706C1C0136019A9642E7D32E
:1046F0000D232370002363700398FDF723FC04B09F
:10470000F0BC01BC00470000380101622901000033
:10471000F0B582B00192079A1B06071C1B0E120609
:104720000093160E21F0E0FE381C21F00DFF00254D
:104730003C181DE0019B211C585DFFF7D1FA009A3F
:10474000013AA31C954201D11C1C02E02023A37056
:104750000334002E0BD0954209D0281C311C27F0C1
:10476000EDF8731E984202D12023237001340135E5
:10477000009B9D42DEDB0D2323700023381C6370F9
:10478000FDF7E0FB02B0F0BC01BC004710B51B0612
:1047900081B01B0E00240094FFF7BAFF01B010BCDB
:1047A00001BC00478020400070470000F0B582B097
:1047B000151C1E1C002400270190009123E0002FEF
:1047C00010D0301C0A2127F0B9F8002810D10D2391
:1047D0006355611C281CFDF757FB281C124921F06A
:1047E00083FE0624301C0A2127F0A8F8002802D0F6
:1047F0002D2363550134019A2919D05DFFF770FA12
:10480000023401370136009B9F42D8DB079A002A09
:1048100002D00D2363550134281C211CFDF734FB05
:1048200002B0F0BC01BC00471C9A0460F0B59EB019
:1048300076210D23694477226F460B376A440B704B
:1048400000231370FE49381C21F04EFEFCF73CF9A2
:10485000011C381C21F09CFD76216944381C21F094
:1048600097FDF849381C21F093FDFCF739F9011C3C
:10487000381C21F08DFD76216944381C21F088FD1B
:10488000F149381C21F084FD45F070FA011C381CF8
:1048900021F07EFD76216944381C21F079FDEB4939
:1048A000381C21F075FD381CFDF74CFB0BF064F84B
:1048B00076216944381C21F017FEE549381C21F0A7
:1048C00067FD76216944381C21F062FDE149381CFE
:1048D00021F05EFD08F0FAF8011C381C21F058FDAB
:1048E00076216944381C21F053FDDB49381C21F046
:1048F0004FFD08F0FFF8011C381C21F049FD76211E
:104900006944381C21F044FD381CFDF71BFBD349DA
:10491000381C21F0E9FD08F0E9F8011C381C21F0F1
:1049200037FD76216944381C21F032FDCC49381C12
:1049300021F02EFD08F0D6F8011C381C21F028FDCE
:1049400076216944381C21F023FD76216944381C06
:1049500021F01EFD381CFDF7F5FAFEF717FC1CAA26
:1049600004231C90BF49381CFFF710FFBE49381CB8
:1049700021F0BAFD381CFDF7E5FA76226A44131CD3
:10498000BA49381C21F070FC381CFDF7DBFAB84C32
:104990000025201C53213A1C00230095C434FFF746
:1049A00005FF0123201C0093002103233A1CFFF77D
:1049B000FDFE7622AF496A44381C21F055FC381CB4
:1049C000FDF7C0FA0121AC4800913A1C18210023E0
:1049D000FFF7ECFE76226A44131CA849381C21F02C
:1049E00043FC381CFDF7AEFAA54C0323A54A0093FF
:1049F000381C231C01210195FFF7C0FD0321012371
:104A0000A14A00910193381C022100230226FFF7DE
:104A1000B5FDE31C9D4A381C032100960196FFF763
:104A2000ADFD03219A4A0191381C04210023FF2582
:104A30000096FFF7A3FD631D964A381C05210195DA
:104A40000096FFF79BFD944A381C06210023019530
:104A50000096FFF793FD032100910421E31D8F4A87
:104A60000191381C0721FFF789FD032305258C4A96
:104A70000093381C082100230195FFF77FFD231CBC
:104A80000621884A0A330191381C09210096FFF754
:104A900075FD854A381C0A21002301950096FFF711
:104AA0006DFD0321231C00910821804A0C330191E4
:104AB000381C0B21FFF762FD0323009309237C4A76
:104AC0000193381C0C210023FFF758FD0421231CFF
:104AD00000910A21774A0F330191381C0D21FFF70D
:104AE0004DFD231C0B21744A13330191381C0E21F8
:104AF0000096FFF743FD231C0C21704A15330191EA
:104B0000381C0F210096FFF739FD231C14216C4A35
:104B100017330191381C10210096FFF72FFD231C3D
:104B20001321684A19330191381C11210096FFF7AF
:104B300025FD231C0D21644A1F330191381C1221CD
:104B40000096FFF71BFD231C0E21604A1D330191C7
:104B5000381C13210096FFF711FD15235C4A0193C1
:104B6000381C142100230096FFF708FD231C0F2199
:104B7000584A21330191381C15210096FFF7FEFC9D
:104B8000231C1021544A1B330191381C1621009616
:104B9000FFF7F4FC231C1121504A23330191381CE8
:104BA00017210096FFF7EAFC0121231C0091122136
:104BB0004B4A25330191381C1821FFF7DFFC0321F4
:104BC000231C00911621474A26330191381C1921D4
:104BD000FFF7D4FC231C1921434A29330191381CC7
:104BE0001A210096FFF7CAFC231C1A213F4A2B33D7
:104BF0000191381C1B210096FFF7C0FC0121231CEA
:104C0000009117213A4A2D330191381C1C21FFF7DE
:104C1000B5FC0121231C00911821364A2E33019145
:104C2000381C1D21FFF7AAFC231C1B21324A2F33FD
:104C30000191381C1E210096FFF7A0FC5EE00000E9
:104C40004083046050830460608304607083046068
:104C5000808304608C830460A4830460BC8304604C
:104C6000D4830460EC830460FC83046008840460E3
:104C700054000162288404603C00016234840460B2
:104C80003A0101628084046094840460A884046012
:104C9000BC840460D0840460E4840460F88404600C
:104CA0000C850460208504603485046048850460B8
:104CB0005C85046070850460848504609885046068
:104CC000AC850460C0850460D4850460E885046018
:104CD000FC850460108604602486046038860460C5
:104CE0004C86046060860460748604608886046074
:104CF0009C860460B0860460C4860460221C20493F
:104D0000A332381C0823FFF741FD221C1D49AB329A
:104D1000381C0823FFF73AFD221C1B49B332381C0C
:104D20000423FFF733FD221C18493132381C0223BB
:104D3000FFF72CFD164AA4180B231649381C221C19
:104D4000FFF724FD144D2B68002B15D0134C23685E
:104D5000002B11DD76226A44131C1149381C21F006
:104D600083FA381CFDF7EEF80123286821683A1C05
:104D700000930023FFF71AFD1EB0F0BC01BC0047F2
:104D8000D8860460F0860460088704602087046089
:104D90009701000038870460F82F0162D82F016264
:104DA00050870460094A3F21937849420B4393702E
:104DB00053790B435371D3790B43D371137B0B435B
:104DC0001373537A0B43537270470000380101622A
:104DD00030B50006050E0124254249D02E4A937BAA
:104DE000052083439373537CA3435374537DA343A0
:104DF0005375D37DA343D375537EA3435376D37E9C
:104E000003218B43D376537FA3435377D37F8343CD
:104E1000D377911CCB7FA343CB77111DCB7FA343CB
:104E2000CB77911DCB7FA343CB770231CB7FA343BD
:104E3000CB7793783E210B40937053790B4053719D
:104E4000D3790B40D371137B0B401373537A101C2F
:104E50000B4028305372037813218B430370111CCD
:104E60002F310B78A3430B7030321378A3431370A8
:104E7000AB070DD5084A111C2B310B78A3430B70DF
:104E800002310B78A3430B7031321378A3431370B4
:104E900030BC01BC004700003801016200B50320AE
:104EA000FFF796FF01BC004730B500060906050E66
:104EB000002902D0FFF7F2FF10E0384A93783F2133
:104EC0000B40937053790B405371D3790B40D371DE
:104ED000137B0B401373537A0B405372EB0749D586
:104EE0002E4A937B052423439373537C0120034371
:104EF0005374537D03435375D37D0343D375537E5E
:104F000003435376D37E03210B43D376537F03436E
:104F10005377D37F2343D377911CCB7F0343CB7746
:104F2000111DCB7F0343CB77911DCB7F0343CB7701
:104F30000231CB7F0343CB7793780343937053794C
:104F400003435371D3790343D371137B0343137327
:104F5000537A141C034328345372237813210B43D0
:104F60002370111C2F310B7803430B7030321378F0
:104F700003431370AB070ED5084A111C2B310B7875
:104F8000012003430B7002310B7803430B70313265
:104F900013780343137030BC01BC00473801016231
:104FA00000B502200121FFF77FFF01BC0047000090
:104FB00000B501200121FFF777FF01BC0047000089
:104FC00000B502200021FFF76FFF01BC0047000081
:104FD00000B501200021FFF767FF01BC004700007A
:104FE00000B503200021FFF75FFF01BC0047000070
:104FF00000B5FFF7F5FFFFF7D5FE0948437E012115
:105000008B434376821DD37F8B43D3770232D37F8A
:105010008B43D377837B04229343837301BC004784
:105020003801016200B50120FFF7D2FE01BC004744
:1050300000B50220FFF7CCFE01BC004700B5FFF72A
:105040002DFF044B31331A7801210A431A7001BC39
:10505000004700003801016200B5FFF71FFF034B56
:105060009A7B01210A439A7301BC0047380101620F
:1050700000B5FFF713FF034B5A7C01210A435A7412
:1050800001BC00473801016200B5FFF707FF034B81
:105090005A7F01210A435A7701BC00473801016257
:1050A00000B5FFF7FBFE044B0233DA7F01210A4310
:1050B000DA7701BC004700003801016200B5FFF754
:1050C000EDFE034BDA7F01210A43DA7701BC00478A
:1050D0003801016200B5FFF7E1FE044B0433DA7FCB
:1050E00001210A43DA7701BC004700003801016260
:1050F00000B5FFF7D3FEFFF755FE01BC00470000E7
:10510000054A937801210B43937053790B435371F4
:10511000D3790B43D37170473801016200B5FFF7B3
:10512000BDFEFFF7EDFF01BC00470000054A937884
:1051300040210B43937053790B435371D3790B4345
:10514000D37170473801016200B5FFF7A7FEFFF782
:10515000EDFF01BC00470000064A802193784942D8
:105160000B43937053790B435371D3790B43D37132
:10517000704700003801016200B5FFF78FFEFFF7AE
:10518000EBFF01BC00470000044A137B01210B43E5
:105190001373537A0B435372704700003801016256
:1051A000044A137B40210B431373537A0B4353720E
:1051B0007047000038010162044A8021137B494294
:1051C0000B431373537A0B435372704738010162D8
:1051D00000B5FFF763FE034B1A7B01210A431A73E4
:1051E00001BC00473801016200B5FFF757FE034BD1
:1051F0001A7B40210A431A7301BC0047380101623F
:1052000000B5FFF74BFE044B80211A7B49420A434D
:105210001A7301BC004700003801016200B5FFF7B6
:105220003DFE034B5A7A01210A435A7201BC0047E2
:105230003801016200B5FFF731FE034B5A7A402175
:105240000A435A7201BC00473801016200B5FFF7FA
:1052500025FE044B80215A7A49420A435A7201BC06
:10526000004700003801016200B5FFF717FE034B4D
:105270005A7D01210A435A7501BC00473801016279
:1052800000B5FFF70BFE034BDA7D01210A43DA7507
:1052900001BC00473801016200B5FFF7FFFD034B79
:1052A000DA7E01210A43DA7601BC00473801016247
:1052B00000B5FFF7F3FD034BDA7E02210A43DA76ED
:1052C00001BC004738010162074AD37D08218B43A6
:1052D000D375537D8B435375537E8B435376D37E67
:1052E0008B43D3767047000038010162074AD37DB3
:1052F00008210B43D375537D0B435375537E0B43EA
:105300005376D37E0B43D376704700003801016299
:10531000074AD37D10218B43D375537D8B4353753F
:10532000537E8B435376D37E8B43D37670470000F6
:1053300038010162074AD37D10210B43D375537D99
:105340000B435375537E0B435376D37E0B43D37677
:10535000704700003801016200B5FFF79FFD044B64
:1053600028331A7813210A431A7001BC0047000041
:105370003801016200B5FFF791FD044B28331A781C
:1053800001210A431A7001BC004700003801016284
:1053900000B5FFF783FD044B28331A7802210A4336
:1053A0001A7001BC004700003801016200B5FFF728
:1053B00075FD044B28331A7810210A431A7001BC7A
:1053C000004700003801016200B5FFF767FD034B9D
:1053D0005A7E01210A435A7601BC00473801016216
:1053E00000B5FFF75BFD044B0833DA7F01210A4368
:1053F000DA7701BC004700003801016200B5FFF711
:105400004DFD044B0633DA7F01210A43DA7701BCF4
:10541000004700003801016200B5FFF73FFD044B73
:105420002F331A7801210A431A7001BC004700008B
:1054300038010162024B1A7C0F218A431A747047AB
:105440003801016200B5FFF729FD044B2B331A78B0
:1054500001210A431A7001BC0047000038010162B3
:1054600000B5FFF71BFD044B2D331A7801210A43C9
:105470001A7001BC004700003801016200B5FFF757
:105480000DFD044B30331A7801210A431A7001BC18
:10549000004700003801016200B5FFF7FFFC034B35
:1054A0009A7B04210A439A7301BC004738010162C8
:1054B000044A537D01210B435375D37D0B43D375B0
:1054C0007047000038010162054A111C2B310B782E
:1054D000082003430B702D32137803431370704779
:1054E00038010162054A111C2B310B7808208343D7
:1054F0000B702D32137883431370704738010162AB
:10550000044A537920210B435371D3790B43D37150
:105510007047000038010162044A537920218B430F
:105520005371D3798B43D371704700003801016206
:10553000044A53790C218B435371D3798B43D37134
:105540007047000038010162054A537904200821A0
:1055500003438B435371D37903438B43D371704718
:1055600038010162054A53790820042103438B4323
:105570005371D37903438B43D37170473801016270
:10558000044A53790C210B435371D3790B43D371E4
:105590007047000038010162084A93783E210B40B1
:1055A000937053790B405371D3790B40D371137BB4
:1055B0000B401373537A0B405372704738010162EA
:1055C000054A937801218B43937053798B43537130
:1055D000D3798B43D371704738010162054A9378C0
:1055E00040218B43937053798B435371D3798B4311
:1055F000D371704738010162054A93787F210B40CF
:10560000937053790B405371D3790B40D37170472A
:1056100038010162044A137B01218B431373537ACF
:105620008B4353727047000038010162044A137BB8
:1056300040218B431373537A8B435372704700009E
:1056400038010162044A137B7F210B401373537AA4
:105650000B4053727047000038010162044A537DC9
:1056600001218B435375D37D8B43D3757047000065
:105670003801016210B51949CB7A20229343CB72CD
:105680004B7B60222024934323434B738B799343BA
:1056900023438B714B7D7F2213404B750B7E012280
:1056A00093430B768B7F032293438B770B7C4022B3
:1056B00093430B74881CC37F3F2213404022134343
:1056C000C3770A1C0832D37F2343D3770631CB7FBD
:1056D00004229343CB7710BC01BC00473801016220
:1056E0000649CB7B40229343CB73CB7C042293436C
:1056F000CB740B7E93430B76704700003801016238
:105700000649CB7B40221343CB73CB7C042213434B
:10571000CB740B7E13430B76704700003801016297
:1057200005490B7E02221343202293430B76CB7E46
:1057300040221343CB7670473801016204490B7E47
:10574000222293430B76CB7E40229343CB76704745
:1057500038010162024B1A7E20210A431A767047F3
:105760003801016200B507498A7A930708D40223F9
:1057700013438B7206F09EFE002801D006F0C8FE8F
:1057800001BC00473C00016270B5104A937A0221C7
:105790000B4217D08B43937206F08CFE002811D079
:1057A000FBF726FE04040126250C600C3040354032
:1057B000A40CFBF7A7FC3440281CFBF77DFC201C45
:1057C000FBF7C6FC70BC01BC004700003C00016256
:1057D0000E4A937B202003439373111DCB7F034319
:1057E000CB77537C02210B435374537D0343537592
:1057F000D37D0343D375537E03435376D37E034354
:10580000D376537F10210B435377704738010162E1
:105810000E4A937B202083439373111DCB7F8343D8
:10582000CB77537C02218B435374537D8343537551
:10583000D37D8343D375537E83435376D37E834393
:10584000D376537F10218B43537770473801016221
:105850000349CB780C22934304221343CB70704747
:105860003C0001620349CB780C2293430822134386
:10587000CB7070473C0001620549CB78402213434E
:10588000CB7004490A78F72313400B70704700006F
:105890003C0001621400016200B50948CE225200AA
:1058A000835C08218B438354064B1B781B06002B1B
:1058B00003D10020002105F035F901BC00470000AC
:1058C000380101625123016210B5431C0ED00C4C0B
:1058D000002805D0CE235B00E25C04210A4304E0EB
:1058E000CE235B00E25C04218A43E254044BCE22C7
:1058F0005200985C4007C00F10BC02BC0847000073
:1059000038010162034B52331A780F218A431A700F
:105910007047000054000162044952310B780F2295
:105920009343022213430B7070470000540001623E
:10593000044952310B780F229343052213430B7015
:105940007047000054000162044952310B780F2265
:1059500093430A2213430B70704700005400016206
:10596000014A9623D36070473C000162024A9623A5
:105970005B00D360704700003C000162024A96233E
:105980009B00D360704700003C000162024A9623EE
:10599000DB00D360704700003C000162024A96239E
:1059A0001B01D360704700003C000162024A96234D
:1059B0005B01D360704700003C000162024A9623FD
:1059C0009B01D360704700003C000162024A9623AD
:1059D000DB01D360704700003C000162024A96235D
:1059E0001B02D360704700003C000162024AE123C1
:1059F0001B02D360704700003C000162024AE123B1
:105A00005B02D360704700003C00016209060B0195
:105A1000090F1A0F092902D90B1C373301E00B1C9F
:105A200030330370092A02D9131C373301E0131CE9
:105A30003033437070470000F0B5120687B0090696
:105A4000120E051C0F0E0092FF2A01D1FF2F58D015
:105A50003248854224DB031C18339D4220D22D1A84
:105A60006C4606343B230A21281C237025F0B0FE27
:105A7000303060700A21281C25F060FF3030A070A3
:105A800068463B230A30391CE370FFF7BFFF3B2316
:105A9000A371684600990D30FFF7B8FF092131E086
:105AA0006E461A361B22281C311C6A44FEF7D4FCB1
:105AB000013026D06C4606343B23237020236370CC
:105AC0003378A3703B23E3706B46DD7E0A21281CEC
:105AD00025F038FE303020710A21281C25F0CAFE3E
:105AE0003030607168463B230D30391CA371FFF7DD
:105AF0008DFF3B236372009904A8FFF787FF0C21F9
:105B000000E0002168460D2306300B540131FCF7FC
:105B1000BBF907B0F0BC01BC004700003C000162CB
:105B2000F0B50D4B1968071C002911D00B4B1E68EE
:105B30000C1C00250AE0211C381C042220F05AFD10
:105B40000C34002801D1012003E00135B542F2DB1D
:105B50000020F0BC02BC08472C54016228540162AA
:105B6000F0B584B06B460E330D2200901A700022FF
:105B70005A70644D00270026634BF418201CFFF771
:105B8000CFFF002810D1201C0221FCF77DF9009BDB
:105B9000002B05D0286829796A79FFF74DFF03E0CB
:105BA00068460E30FCF7CEF9584B01370C360C35F1
:105BB0009F42E1D1564C0026002553482818FFF794
:105BC000AFFF002811D1534803212818FCF75CF9D6
:105BD000009B002B05D0206821796279FFF72CFF0C
:105BE00003E068460E30FCF7ADF901360C350C3495
:105BF000AA2EE2D1484C0026002543482818FFF77A
:105C00008FFF002811D1454804212818FCF73CF9E2
:105C1000009B002B05D0206821796279FFF70CFFEB
:105C200003E068460E30FCF78DF901360C350C3474
:105C30001C2EE2D13A4B1B68002B26D000260025F3
:105C40001FE0374B1B685C19201C20F07DFC0428EA
:105C500001D9042100E0011C201CFCF715F9009B70
:105C6000002B08D02E4B1B685B195868197A5A7A9A
:105C7000FFF7E2FE03E068460E30FCF763F90136F9
:105C80000C35284B1B689E42DBDB20252B061F0EA4
:105C900020242306281C211C00221E0EFDF788FE4E
:105CA000431C05D1281C211CFDF73AFF431C16D0CC
:105CB00001AA17705670009B002B01D1022108E049
:105CC0003B2301066846090E93700730FFF79EFEDE
:105CD000052101A80D230B540131FCF7D5F801343F
:105CE0005B2CD6D101355B2DD0D101AC0E490D22F4
:105CF000201C20F0B9FA201CFCF724F904B0F0BCF9
:105D000001BC004730AE03602CAE03608D01000083
:105D100038A6036034A60360E8A40360E4A403602B
:105D20002C540162285401627487046000B501207C
:105D3000FFF716FF01BC004700B50020FFF710FF7A
:105D400001BC0047074B00061A1C000E3F32507082
:105D500002321070043210704933023250701870E1
:105D6000704700003801016200B50520FFF7EAFF27
:105D700001BC004700B50320FFF7E4FF01BC00476A
:105D800000B50120FFF7DEFF01BC0047024B0122F6
:105D90003E335A707047000038010162024B032203
:105DA0003E335A707047000038010162024B0522F1
:105DB0003E335A707047000038010162024B0122E5
:105DC0003D331A707047000038010162024B032214
:105DD0003D331A707047000038010162124A111CED
:105DE000703101235B42137004328A42F9D16F3A59
:105DF000111C703101235B42137004328A42F9D1C5
:105E00006F3A111C703101235B42137004328A42D5
:105E1000F9D16F3A111C703101235B4213700432C7
:105E20008A42F9D17047000061020162114A111CD7
:105E300070310D23137004328A42FAD16F3A111C6B
:105E4000703101235B42137004328A42F9D16F3AF8
:105E5000111C703101235B42137004328A42F9D164
:105E60006F3A111C703101235B42137004328A4275
:105E7000F9D170476102016270B50006040E1A4E36
:105E8000002C03D1194B0020336013E0201CFEF7D7
:105E900005F9174D800040193060FF2104221EF0E3
:105EA0007BFC0E2C17D1281CFF21042254301EF03D
:105EB00073FC10E00F4B10491B185A181C210123CA
:105EC0005B4213704B1E1B06190E04320029F6D1DB
:105ED00001300428EED1094A04231370084A022332
:105EE000137070BC01BC004798230162DD0201629F
:105EF000610201623801016229010000612301622F
:105F00003601016200B52720FFF7B6FF01BC00474C
:105F100000B51B20FFF7B0FF01BC004700B51820FB
:105F2000FFF7AAFF01BC004700B52620FFF7A4FF3A
:105F300001BC004700B52120FFF79EFF01BC0047D0
:105F400000B51F20FFF798FF01BC004700B52420D3
:105F5000FFF792FF01BC004700B51C20FFF78CFF44
:105F600001BC004700B51020FFF786FF01BC0047C9
:105F700000B50320FFF780FF01BC004700B50120FA
:105F8000FFF77AFF01BC004700B50420FFF774FF5C
:105F900001BC004700B50220FFF76EFF01BC0047BF
:105FA00000B50F20FFF768FF01BC004700B51720C0
:105FB000FFF762FF01BC004700B51120FFF75CFF4F
:105FC00001BC004700B50E20FFF756FF01BC00479B
:105FD00000B50D20FFF750FF01BC004700B51320AE
:105FE000FFF74AFF01BC004700B50C20FFF744FF54
:105FF00001BC004700B50B20FFF73EFF01BC004786
:1060000000B50A20FFF738FF01BC004700B50920A2
:10601000FFF732FF01BC004700B54320FFF72CFF1C
:1060200001BC004700B54120FFF726FF01BC004737
:1060300000B54420FFF720FF01BC004700B5422017
:10604000FFF71AFF01BC004700B51220FFF714FF4D
:1060500001BC004700B50020FFF70EFF01BC004760
:10606000124A111C703101235B42137004328A42C0
:10607000F9D16F3A111C703101235B421370043265
:106080008A42F9D16F3A111C703101235B421370BF
:1060900004328A42F9D16F3A111C703101235B42FC
:1060A000137004328A42F9D170470000F101016295
:1060B00070B50006040E1A4E002C03D1194B0020B7
:1060C000336013E0201CFDF7E9FF174D80004019F5
:1060D0003060FF2104221EF05FFB0E2C17D1281C1C
:1060E000FF21042254301EF057FB10E00F4B1B1809
:1060F0001A1CB9321C2101235B4213704B1E1B0674
:10610000190E04320029F6D101300428EED1084AD4
:1061100004231370074A0223137070BC01BC0047AC
:106120009823016219010162F101016238010162E3
:10613000612301623601016200B52720FFF7B8FF35
:1061400001BC004700B51B20FFF7B2FF01BC0047B0
:1061500000B51820FFF7ACFF01BC004700B52620B2
:10616000FFF7A6FF01BC004700B52120FFF7A0FF05
:1061700001BC004700B51F20FFF79AFF01BC004794
:1061800000B52420FFF794FF01BC004700B51C2098
:10619000FFF78EFF01BC004700B51020FFF788FF16
:1061A00001BC004700B50320FFF782FF01BC004798
:1061B00000B50120FFF77CFF01BC004700B50420BB
:1061C000FFF776FF01BC004700B50220FFF770FF24
:1061D00001BC004700B50F20FFF76AFF01BC004774
:1061E00000B51720FFF764FF01BC004700B5112080
:1061F000FFF75EFF01BC004700B50E20FFF758FF18
:1062000001BC004700B50D20FFF752FF01BC00475D
:1062100000B51320FFF74CFF01BC004700B50C2070
:10622000FFF746FF01BC004700B50B20FFF740FF1A
:1062300001BC004700B50A20FFF73AFF01BC004748
:1062400000B50920FFF734FF01BC004700B543202B
:10625000FFF72EFF01BC004700B54120FFF728FFE4
:1062600001BC004700B54420FFF722FF01BC0047F6
:1062700000B54220FFF71CFF01BC004700B512200B
:10628000FFF716FF01BC004700B50020FFF710FF25
:1062900001BC004730B52A4B19682A4B0006000E96
:1062A000994211D1284B1A7804239B1A1B06274ABE
:1062B0001B0ED218B9321C23013B1B061B0E10709B
:1062C0000432002B38D0F7E7214B994212D11E4BF4
:1062D0001A7804239B1A1B061C4A1B0ED2181D4B4E
:1062E000D2181C23013B1B061B0E10700432002B1E
:1062F00022D0F7E7184A914209D3141C131D383CE9
:10630000994204D2F53B1B1B5B18D4330EE0134AB1
:1063100091420CD3141C131D383C994207D2104DE6
:1063200053191B1BA2225B1852009B18587008704F
:10633000034A13680133136030BC01BC00470000FE
:10634000982301621901016261230162380101622F
:10635000DD02016229010000290201629902016245
:106360009FFEFFFF0006000EC02318421AD1182816
:1063700018D0182805D8431E1B061B0E072B16D84D
:1063800010E01C2813D31D280CD926280FD109E0B2
:10639000FE2903D80B061B0E834205D3002A01D029
:1063A000914201D8002010E0012040420DE0074B4F
:1063B000C318013B064A1B789B181A1C34335878C3
:1063C000503252780028E3D1E8E77047BDA403605B
:1063D0003801016210B50006000EC0230C1C1842E3
:1063E0001AD1182818D0182805D8431E1B061B0ED2
:1063F000072B16D810E01C2813D31D280CD92628EB
:106400000FD109E00278FF2A08D0A24217D001314B
:106410000130022902D0F5E7002011E001204042BE
:106420000EE0FDF73BFE084A400083186C335B78B2
:10643000FF2BF1D01318181C6D300021E2E701206A
:1064400010BC02BC08470000380101620006000EC3
:10645000C02318421BD1182819D0182805D8431E6C
:106460001B061B0E072B17D811E01C2814D31D2860
:106470000DD9262810D10AE0FE290AD88B4206D071
:10648000131C34331B78FF2B03D08B4201D1012026
:1064900009E00120404206E0034A131C33331B7815
:1064A000FF2BE9D1002070473801016230B50006AA
:1064B000040E201C0D1CFFF78DFF431C0FD000287D
:1064C0000FD1201C291CFFF7C1FF431C07D0002857
:1064D00007D1201C291CFFF745FF013001D1002006
:1064E00000E0012030BC02BC084700000548064916
:1064F0000022535C135401321C2AFAD1034A0523AB
:10650000137070476D0101629CA403603601016243
:10651000044805490022535C135401321C2AFAD165
:10652000704700006D0101629CA40360F0B56E4EDF
:10653000311C52310B781B06002B0BDB6B4B1A1CEA
:106540005232127851330A701A78331C51331A7050
:1065500006F082FD664C00211822201C1EF01CF95A
:10656000644FD22200215200381C1EF015F921235D
:1065700005227B746F2394465B42BA73BA1C0021D8
:10658000D377FB777B1CD97703223B1DDA77132364
:10659000BB7017237B711623FB712023FB723F23F3
:1065A0005B4211227B7563467A723A733B76624690
:1065B000BB1DDA773A1C08322923D37720322823EF
:1065C000402013703B1C3874B8717873F876293307
:1065D000022018700233012519700233F973BD745B
:1065E000F974FD703972B972FD757D767D77B87773
:1065F00019700233197008320C2313703B1C3133AD
:1066000018703D4BF954CD235B00FD543B4B1922D0
:10661000FA54CE235B00F954394BF954CF235B0075
:106620000A22FA54374BF954D0235B003C22FA5427
:10663000354B0F22FA54D1235B00FD54334BF954F0
:10664000E1235B02E3604523237104236371032389
:10665000A37201235B42A170E170A171E17121720B
:106660006172E17221746174A174E3742175F37C29
:10667000FF2B0ED0341C1B34301C2549254A3E30DC
:10668000231C1FF0F1FD301C2D302349221C1FF06C
:10669000EBFDFFF7E5FCFFF7A1FBFDF70FF9381C59
:1066A0001E4C002135300B5D0B5401311C29FAD1F1
:1066B0001C30031C1C330024047001309842FAD1B2
:1066C000FDF72EF9FDF736F9154B1C70154B1C70B4
:1066D000154B8C221C70FF21D20014481EF05CF870
:1066E000F0BC01BC00470000540001621CA1036023
:1066F0003C00016238010162990100009B01000029
:106700009D0100009F010000A1010000A301000005
:10671000808704608C870460948704609CA4036075
:10672000EC020162E2020162E0020162CC0E01624F
:1067300000B5FFF7FBFE024A0123537201BC00477C
:106740005400016200B5002006F0B8FD830615D4A0
:106750000E480378C42B0CD80D49002B01D1C5225B
:1067600005E001380139C5221818D21A59181DF050
:1067700097FFFFF7DBFE06F06FFC01E0FFF7D6FEA8
:10678000044A0023137001BC00470000540001625A
:106790001CA1036036010162054A111C1C31002353
:1067A000137001328A42FAD1024A062313707047ED
:1067B0008901016236010162044A111C1C31002367
:1067C000137001328A42FAD17047000089010162D8
:1067D000F0B5B64B1B6888B00190002B03D0B44BCA
:1067E0001B68013329D068460922163000211DF0AC
:1067F000D3FFB04A1378019E072B03D1AE4B1B7811
:10680000002B04D101231370AB4A00231370AB4B50
:1068100000221A70A74A1378072B0AD001996846FC
:106820000B7816300370002B03D04B784370002B8D
:1068300002D00022039226E01370FDF773FA039052
:1068400000F0FFFC9B4B1A7000F0FBFC237014E07F
:10685000237001246442039400F0F3FC984B1878F1
:1068600006F0C6FE934B1D70934B1D7083E0914B59
:106870001E7000F0DDFC8F4B1E7001235B42039302
:1068800000F0DFFC261C37786C46A775002F62D11C
:10689000884B1A78D31E1B061B0E032B07D9112A0F
:1068A00005D0122A03D00F2A01D0102A05D1854A1B
:1068B000002313707F4A012313707E4B1A78531EF6
:1068C0001B061B0E012B09D9072A09D00B2A3DD024
:1068D0000C2A3BD001214942039137E0072A35D1E8
:1068E000754B1B78013B1C2B29D8774A9B009B5882
:1068F0009F46764B1A68764B1B78D21801235B4271
:10690000937500F09EFC734B1B78002B11D06F4BDE
:106910001D682B7C2F2B0CD9392B0AD8E8896E4B9C
:10692000041C1C406D4B0A21184024F00BFF04434B
:10693000EC81684A0BE000F01BFF00F082FC604B2A
:10694000187806F055FE012252420392594A00235C
:10695000137000F076FC731C029375786C46E57535
:10696000544C002D0CD12378072B03D1544B1878AD
:1069700006F03EFE257001214942039100F061FCC2
:106980002278022A0CD00B2A0AD00C2A08D00F2A0F
:1069900006D0102A04D0112A02D0122A00D0A1E079
:1069A0006B4616331C785B2C11D1242D0FD1B07897
:1069B0009870002801D100F03BFCF178D9700029D3
:1069C00001D100F035FC0122FCF7F2FF0AE00022C1
:1069D000201C291CFCF7ECFF421C05D1201C291CA3
:1069E000FDF79EF8431C54D0324B1B780B2B02D082
:1069F0000C2B16D109E0334B1B78002B49D0384BB8
:106A0000C25C07231A420FD010E02E4B1B78002BDC
:106A10003FD0334BC25C44231A4205D0940700D5C3
:106A20002038411C02D134E0022040426B4616332C
:106A30001B785B2B01D0022300E00423F61800280A
:106A400000DA82E30006000EFFF724FC1D4A1378EB
:106A5000002B00D179E3013B1B061B0E1370002BAA
:106A600000D072E33278694616310A70002A00D1EC
:106A7000E8E673780F4C4B70002B00D1E6E62378E4
:106A80000B3B1B061B0E012B00D85EE3012323707A
:106A90005BE3084A13780B2B01D10D2302E00C2B8A
:106AA00002D10E23137050E30123FBE72C54016243
:106AB0003054016236010162EC020162E0020162BF
:106AC000E20201626123016244C10360E4020162E7
:106AD000E10201623E04016200C0FFFFFF3FFFFFD1
:106AE000F06D0460D31E1B061B0E032B00D9E1E0E2
:106AF000131F1B061B0E022B00D9B7E0C8490B78E9
:106B0000002B00D084E0B3786A461376002B01D1C5
:106B100001232370F37869464B76002B01D10123C2
:106B20002370202F03D05F2F01D001234BE06D464F
:106B300016356878FDF772F8FF2811D0031C093B61
:106B40001B061B0E1C2B0BD8AC78231C303B1B06E2
:106B50001B0E092B04D8ED782F2D01D9392D03D91F
:106B6000B04A012313702FE0AE4A00921378052B30
:106B70000BD1AD4A03061B0E9B18013B1A78AB499B
:106B8000A300521834321B190CE0A700062B0ED1BB
:106B9000A54A03061B0E9B18013B1A78A3495218FD
:106BA00050323B195B005B19103B53700CE03919F4
:106BB0004900491910390906090EFDF781FA01301B
:106BC00002D1009C0123237096490A78012A00D142
:106BD000C7E2531F1B061B0E341D012B00D9B9E25F
:106BE0003379202B00D1B5E25F2B00D1B2E2002334
:106BF0000B706A46337916321370002B00D120E3F4
:106C000073795370002B00D112E301230B709BE2C8
:106C100000230B70042A00D11AE65B2F14D1242D17
:106C200012D1B07869460876002800D100E3F178E7
:106C30006A465176002900D1FAE27D4B01221C6898
:106C4000FCF7B6FE20700436764900230B706A46C6
:106C5000337816321370002B00D1F2E27378537040
:106C6000002B00D1E4E201230B706EE23B1C303BB1
:106C70001B061B0E092B03D82F2D01D9392D03D943
:106C8000684A012313700EE0032A0CD1B800C01922
:106C90004000401910380006000EFCF7F1FF0130EB
:106CA00001D1012323705F4B1A78012A00D158E2E9
:106CB000B41C4FE2072A00D0C2E05E4B1A786B4644
:106CC0001F331A7001981FF03FFC032849D03C1C69
:106CD0005B2F10D1242D0ED1B0786B46187600288A
:106CE00000D1A5E2F1785976002900D1A0E2012275
:106CF000FCF75EFE0DE06B4616335D78201C291C08
:106D00000022FCF755FE411C05D1201C291CFCF774
:106D100007FF421C25D06C461F3400060122000EDE
:106D2000211C01F015FF434D22782B789A4203D0A5
:106D3000414B1B78002B0DD0404B187806F058FCC7
:106D40003D4B0021374A19700123137001235B4228
:106D5000297003936B4616331B785B2B4FD00221AF
:106D60004EE001981FF0F0FB021C032804D16B4693
:106D700016331B78412B0BD06846163003785B2BFB
:106D800040D14378412B3DD1032A01D0029902E042
:106D900068461630311C6C461634032200251DF05F
:106DA0007FFCE570201C1FF0CFFB032800D055E5C9
:106DB000201CFCF7B7FF013003D01F4B1B78002BC2
:106DC00016D01E4B187806F013FC1B4B0021154AF9
:106DD000197001231370174B019819701FF0B4FB41
:106DE000032800D1B1E16B465B2216331A70ACE187
:106DF00001981FF0A9FB032801D1032100E0042121
:106E000074183FE50D4B187806F0F2FB0A4B002191
:106E1000044A197001231370064B197095E10000A4
:106E20006123016236010162BDA403603801016281
:106E300098230162EC020162E0020162E202016257
:106E4000082A00D081E100240494FF2433E0012FBC
:106E500029DDBA5D6B461633FA54062F05D11B782F
:106E6000202B02D05F2B00D09BE0002A1BD1062FE5
:106E700008D16B4616331B78202B00D191E05F2B95
:106E80000DD18EE0042F00D18CE0022F07D16B468C
:106E900016331B78202B02D05F2B00D082E0C44A2F
:106EA000012313707EE0072F62D8C24ABB006D46F3
:106EB0009B5816359F466B4616331B78202B09D0FE
:106EC0005F2B07D0303B1B061B0E092B02D9B84A9B
:106ED00001231370002155E02B78202B01D05F2B6C
:106EE00006D16878FCF7EAFE041CFF2848D105E0CB
:106EF0006B78303B1B061B0E092B41D9AC4A012392
:106F000013703DE07A5D131C303B1B061B0E162BE5
:106F10002ED8131C3A3B1B061B0E062B28D92878AB
:106F2000202801D05F282CD1402A2AD920E07A5D80
:106F3000131C303B1B061B0E162B05D8131C3A3BAB
:106F40001B061B0E062B1CD84B1F012B04D82B78BD
:106F5000202B11D05F2B0FD0CB1E012B08D8287807
:106F6000202805D05F2803D001210427049108E0E0
:106F70008F4A0123137004E001220627049200E0E7
:106F80000127391C8A4B1B78012B00D1BBE0049BE5
:106F9000012B04D04F1C072F00DC58E707E00F1C23
:106FA00005E00627824B1B78012B00D144E16D469A
:106FB0001635FF2C5ED06200A9787F4B1219920023
:106FC000D2188B005B18E9785B007C4C5B181919B0
:106FD000137A5068994248D24418042F3CD028793B
:106FE000392801D8302100E03721431A1B07180E39
:106FF0006B4616335B79392B01D8302200E03722FB
:107000009B1A1B066A461B0E163253711843072F34
:1070100001DC207075E02378834323709379392B4A
:1070200001D8302200E037229B1A1B07190E6B464D
:107030001633DB79392B01D8302200E037229B1A36
:107040001B066A461B0E1632D37122780B4313437C
:107050002370341C083463E02078291CFCF740FEC0
:10706000281C0221FAF710FF2BE0514A0123341C9F
:10707000137055E02A7893009B186A785B009B1880
:107080004E4A4F499B185C18022F40D0A8783928E7
:1070900001D8302100E03721431A1B07180E6B4638
:1070A0001633DB78392B01D8302200E037229B1AC7
:1070B0001B066A461B0E1632D3701843052F02DCDE
:1070C0002070341D2CE02378834323701379392BEF
:1070D00001D8302200E037229B1A1B07190E6B469D
:1070E00016335B79392B01D8302200E037229B1A06
:1070F0001B066A461B0E1632537122780B4313434C
:107100002370B41D0CE001235B4203931DE0207843
:10711000291CFCF7E5FD281C0221FAF7B5FEB41C7A
:10712000234A1378012B00D187E0002313706946AE
:10713000237816310B70002B00D182E063784B70FE
:10714000002B75D001231370261C194B1A78012AC5
:1071500007D0341C0D2A05D00E2A01D0FFF792FB70
:1071600000E0341C6D4616352E785D2E15D1611C5D
:10717000281C042200261DF093FA2E71281C1FF0F3
:10718000E3F9042801D0FFF772FB281CFCF7CAFDC5
:1071900003990534014303913DE001981FF0D4F9B0
:1071A00003280FD05B2E2DD1611C281C0CE00000A1
:1071B00036010162B8C10360E4A10360F0FDFFFF86
:1071C0003C000162281C211C6D4616350322002656
:1071D0001DF066FAEE70281C1FF0B6F9032801D0E6
:1071E000FFF749FB281CFCF79DFD039A024303921D
:1071F00001981FF0A9F9032801D1032300E004231B
:10720000E41808E00023AB70281CFCF78BFD039BFF
:107210000343039302340D4A1378002B01D1FFF787
:1072200031FB01210023494213700391FFF72AFB30
:1072300001225242039204E0341C01235B42039377
:1072400090E7039808B0F0BC02BC0847E002016276
:1072500000B5FDF723FE054A137B01210B43137391
:10726000537A0B43537201BC00470000380101629E
:1072700000B5FDF713FE054A137B40210B43137342
:10728000537A0B43537201BC00470000380101627E
:1072900000B5FDF703FE054A8021137B49420B43ED
:1072A0001373537A0B43537201BC004738010162D8
:1072B00000B5FDF7F3FD054A537D01210B435375DE
:1072C000D37D0B43D37501BC004700003801016238
:1072D0000047184700B5074B00221A70064B1A707A
:1072E000064B1A708C220648D200FF211DF054FA7A
:1072F00001BC0047EC020162E2020162E0020162AD
:10730000CC0E016230B5134A13780006000E072B2D
:1073100003D1114B1B78002B16D1072313700E4A93
:10732000012313700D4B00251D700D4B18708C231D
:1073300058430C4B0C4CC0182060FF218C221DF0D0
:107340002BFA2368DD7602E0084A0123137030BC73
:1073500001BC004736010162EC0201623E04016299
:10736000E2020162CC0E0162E4020162E00201620B
:1073700000B50020FFF7C6FF01BC004700B50120A3
:10738000FFF7C0FF01BC004700B50220FFF7BAFFBE
:1073900001BC004700B50320FFF7B4FF01BC004764
:1073A00000B50420FFF7AEFF01BC004700B5052083
:1073B000FFF7A8FF01BC004700B50620FFF7A2FFBA
:1073C00001BC004700B50720FFF79CFF01BC004748
:1073D0000A4B1B780006000E072B03D1084B1B78C5
:1073E000002B06D1074B0122D97982400A43DA717A
:1073F00002E0054A01231370704700003601016264
:10740000EC0201623C000162E002016200B5002072
:10741000FFF7DEFF01BC004700B50120FFF7D8FFF2
:1074200001BC004700B50220FFF7D2FF01BC0047B6
:1074300000B50320FFF7CCFF01BC004700B50420D6
:10744000FFF7C6FF01BC004700B50520FFF7C0FFEE
:1074500001BC004700B50620FFF7BAFF01BC00479A
:1074600000B50720FFF7B4FF01BC004710B5114B72
:107470001B780006000E072B03D10F4B1B78002B47
:1074800011D10E490124CB79221C824093431B0663
:107490000A7A180EC871224208D0002806D1131C9F
:1074A000A3430B7202E0064A0123137010BC01BC17
:1074B0000047000036010162EC0201623C000162FB
:1074C000E002016200B50020FFF7D0FF01BC0047D9
:1074D00000B50120FFF7CAFF01BC004700B502203C
:1074E000FFF7C4FF01BC004700B50320FFF7BEFF54
:1074F00001BC004700B50420FFF7B8FF01BC0047FE
:1075000000B50520FFF7B2FF01BC004700B506201B
:10751000FFF7ACFF01BC004700B50720FFF7A6FF4F
:1075200001BC0047084B1B78072B03D1074B1B7886
:10753000002B05D1064B1A7A02218A431A7202E007
:10754000044A01231370704736010162EC020162A4
:107550003C000162E0020162084B1B78072B03D15B
:10756000074B1B78002B05D1064B1A7A02210A43E0
:107570001A7202E0044A0123137070473601016257
:10758000EC0201623C000162E0020162084B1B78E0
:10759000072B03D1074B1B78002B05D1064B1A7A1A
:1075A00001218A431A7202E0044A012313707047D2
:1075B00036010162EC0201623C000162E0020162FC
:1075C000084B1B78072B03D1074B1B78002B05D1E9
:1075D000064B1A7A01210A431A7202E0044A012377
:1075E0001370704736010162EC0201623C000162D7
:1075F000E00201620F4B1B78000609061206000E1E
:10760000090E120E072B0DD1FF2810D00A4B1B7844
:1076100098420CD0FF2905D0994208D0FF2A01D00A
:107620009A4204D0054A0123FF20137000E0002095
:107630007047000036010162EC020162E002016263
:1076400000B50120FF21FF22FFF7D4FF002805D15C
:10765000034A03231370034B1B68187001BC0047D7
:10766000EC020162E402016200B50120FF21FF2269
:10767000FFF7C0FF002802D1024A0223137001BCA9
:1076800000470000EC02016200B50320FF21FF2249
:10769000FFF7B0FF002807D1044A06231370044BFC
:1076A0001870044B1B68588001BC0047EC02016253
:1076B0003E040162E402016200B50320FF21FF22C3
:1076C000FFF798FF002802D1024A0423137001BC7F
:1076D00000470000EC02016200B50620FF21FF22F6
:1076E000FFF788FF002809D1054A0C231370054BCA
:1076F0001870054B1A687F231371D07601BC0047C0
:10770000EC0201623E040162E402016200B506205F
:10771000FF21FF22FFF76EFF002808D1054A092349
:107720001370054B1870054B1A687E23137101BC4A
:1077300000470000EC0201623E040162E4020162C3
:1077400000B50620FF21FF22FFF754FF002807D1D4
:10775000044A07231370044B1870044B1B681871FC
:1077600001BC0047EC0201623E040162E4020162D6
:1077700005490B78002B06D0044B1A68D37E0133E1
:10778000D37600230B7070473E040162E40201626D
:1077900000B50C201621FF22FFF72CFF002818D17E
:1077A000FFF7E6FF0C4B1868C37E02336D2B0DDC30
:1077B0000A4A152313700A4A08231370C37E102245
:1077C000C118524201330A77C37602E0054A012309
:1077D000137001BC00470000E4020162EC02016288
:1077E0003E040162E002016210B50C201621FF2266
:1077F000FFF700FF041C002817D1FFF7B9FF0C4B5F
:107800001968CB7E04336D2B0CDC0A4A0D231370F0
:10781000CB7ECA1801331B061B0ECB76CB18147710
:107820001C7702E0044A0123137010BC01BC00471E
:10783000E4020162EC020162E002016210B50C2078
:107840001621FF22FFF7D6FE041C002818D1FFF7EF
:107850008FFF0D4B1868C37E04336D2B0DDC0B4A74
:107860000D231370C37EC11801331B061B0E10229B
:10787000C376C3180A771C7702E0054A0123137008
:1078800010BC01BC00470000E4020162EC0201628E
:10789000E002016200B50C201621FF22FFF7AAFECC
:1078A000002817D1FFF764FF0B4B1868C37E043321
:1078B0006D2B0CDC094A0F231370094A082313703F
:1078C000C37E2022C11801330A77C37602E0054A3D
:1078D0000123137001BC0047E4020162EC02016263
:1078E0003E040162E002016200B50C201621FF2275
:1078F000FFF780FE002817D1FFF73AFF0B4B1868FF
:10790000C37E04336D2B0CDC094A0F231370094A24
:1079100008231370C37E4022C11801330A77C3764F
:1079200002E0054A0123137001BC0047E402016232
:10793000EC0201623E040162E002016210B5122015
:107940001421FF22FFF756FE041C00280FD1FFF779
:107950000FFF084A13231370074B1968CB7ECA1810
:1079600001331B061B0ECB76C91814770C7710BC9D
:1079700001BC0047EC020162E402016210B5122072
:107980001421FF22FFF736FE041C002810D1FFF758
:10799000EFFE094A13231370084B1968CB7EC818F1
:1079A00001331B061B0E1022CB76C91802770C7709
:1079B00010BC01BC00470000EC020162E40201625D
:1079C00000B512201421FF22FFF714FE00280FD16A
:1079D000FFF7CEFE074A15231370074A08231370DA
:1079E000064B1968CB7E2022C81801330277CB766C
:1079F00001BC0047EC0201623E040162E402016244
:107A000000B512201421FF22FFF7F4FD00280FD14A
:107A1000FFF7AEFE074A15231370074A08231370B9
:107A2000064B1968CB7E4022C81801330277CB760B
:107A300001BC0047EC0201623E040162E402016203
:107A400010B50C201621FF22FFF7D4FD041C0028DE
:107A500019D1FFF78DFE0D4B1868C37E04336D2BD3
:107A60000EDC0B4A0D231370C37EC11801331B06B5
:107A70001B0E80225242C376C3180A771C7702E09D
:107A8000044A0123137010BC01BC0047E4020162E8
:107A9000EC020162E002016210B50C201621FF2207
:107AA000FFF7A8FD041C002819D1FFF761FE0D4B5C
:107AB0001868C37E04336D2B0EDC0B4A0D23137044
:107AC000C37EC11801331B061B0E70225242C376BF
:107AD000C3180A771C7702E0044A0123137010BC14
:107AE00001BC0047E4020162EC020162E0020162B3
:107AF00000B50C201621FF22FFF77CFD002818D1CD
:107B0000FFF736FE0C4B1868C37E04336D2B0DDC7B
:107B10000A4A0F2313700A4A08231370C37E602297
:107B2000C118524201330A77C37602E0054A0123A5
:107B3000137001BC00470000E4020162EC02016224
:107B40003E040162E002016200B50C201621FF2212
:107B5000FFF750FD002818D1FFF70AFE0C4B1868FC
:107B6000C37E04336D2B0DDC0A4A0F2313700A4ABF
:107B700008231370C37E4022C118524201330A7792
:107B8000C37602E0054A0123137001BC00470000E0
:107B9000E4020162EC0201623E040162E002016261
:107BA00010B50C201621FF22FFF724FD041C00282D
:107BB00013D1FFF7DDFD0A4B1B6810229A770422D0
:107BC000DA76012252425A7401225242DA81054A7F
:107BD0001C775C77DC771D23137010BC01BC004759
:107BE000E4020162EC02016210B51D4C2378162BF1
:107BF00001D10C2323700C200E210B22FFF7FAFC7D
:107C000000282AD123780B2B08D1164B1A68164B63
:107C10001B78D21801235B42937503E00C2B01D132
:107C2000FFF7A6FD104B00221A700E4B186805E0F6
:107C300083185B7CFF2B07D0531C0B700A490A7812
:107C4000042AF5D9052A03D0054A0A23137004E053
:107C5000064B01221A7000230B7010BC01BC0047B8
:107C6000EC020162E4020162E1020162E0020162EF
:107C700000B50C201621FF22FFF7BCFC002809D11B
:107C8000FFF776FD044A0E231370044B1A68012394
:107C90005B42537401BC0047EC020162E4020162E2
:107CA00030B5194C23780004050C162B01D10C2398
:107CB00023700C200E210B22FFF79CFC00281FD103
:107CC00023780C2B07D1FFF753FD104B1A680123C3
:107CD0005B42537409E00B2B07D10C4B1A680C4B19
:107CE0001B78D21801235B4293750A4B064A074959
:107CF0009D4201D11D2300E0192313700B68DD8123
:107D000030BC01BC00470000EC020162E4020162E9
:107D1000E1020162FFFF000000B50248FFF7C0FF6B
:107D200001BC0047FFFF000000B580200002FFF704
:107D3000B7FF01BC0047000000B50020FFF7B0FF0F
:107D400001BC004700B58020C001FFF7A9FF01BCBE
:107D50000047000000B5C0200002FFF7A1FF01BCF2
:107D60000047000030B51D20FF21FF22FFF742FC35
:107D7000002829D1174B1B78042B25D0002B11D0BC
:107D8000154B1D682B7C2F2B0CD9392B0AD8E88971
:107D9000124B041C1C40124B0A21184023F018FD02
:107DA0000443EC810B4B00241C700E4B01201B780C
:107DB0000D49021C9A40131CCA791343CB710B4B1B
:107DC0001C700B4B187002E00A4A0123137030BC80
:107DD00001BC00473E040162E402016200C0FFFFF3
:107DE000FF3FFFFFE20201623C000162EC02016220
:107DF00036010162E002016200B50E4B1B78072BD1
:107E000003D10D4B1B78002B0FD10C490B7A0122AB
:107E100093430B720A4B00208C22C8711870FF210B
:107E2000D20008481CF0B8FC02E0074A0123137096
:107E300001BC004736010162EC0201623C000162B4
:107E4000E2020162CC0E0162E00201620006020E53
:107E5000000F092801D8302300E03723C3180B7026
:107E6000101C0F2318400131092801D8302300E0ED
:107E70003723C3180B707047F0B5C44B1B7886B01E
:107E8000072B04D1C24B1B78002B00D0BEE2C14CA3
:107E9000C149201C1EF028FB382363740D23A374F2
:107EA0000023E374201CFAF74DF8BC49201C1EF097
:107EB0001BFBBB4B1B7AD80701D5BA4900E0BA4976
:107EC000201C1EF065FAB34C201CFAF73BF8B749AA
:107ED000201C1EF009FBB24B1B7A990701D5B14952
:107EE00000E0B149201C1EF053FAAA48FAF72AF81C
:107EF000AF4B00221B3B04920093A64CAD49201CC3
:107F00001EF0F2FA049B31332372202363720023A4
:107F1000A372A34B0498DB790341D90702D5A64984
:107F2000201C01E0A549201C1EF032FA994C201CAF
:107F3000FAF708F8201CA2491EF0D6FA009B1A781E
:107F4000531E1B061B0EFD2B00D8A27100984588FE
:107F50006B1E1B049B4A1B0C934211D8261C123625
:107F60000E34281C0A2123F085FC303030700A21A1
:107F7000281C23F0E7FB013E0004050CA642F0D1CB
:107F800000990C797F2323407F2B12D07E2C10D0B8
:107F90008D4DAE1E201C0A2123F06CFC3030287061
:107FA0000A21201C23F0CEFB013D0006040EB54241
:107FB000F0D1049C8C23221C5A43844B9B185C1DDB
:107FC000002600252078031C213B1B061B0E5D2B81
:107FD00007D8704BEB18DA1DD07708332022DA77F8
:107FE0000DE0FF2804D07A496918FFF72FFF06E05B
:107FF000684BEB18DA1D2D210833D177D97701367C
:1080000002350134082EDDD1624C221C17320D23BB
:10801000D37700230132D377201CF9F793FF202375
:1080200023700099CB7EFF2B01D16A4E4CE1694E43
:10803000002044E1049C8C236343644A1B189B1872
:108040001A7F431C1B061F0EFF2A00D13CE11306BA
:10805000002B08DAF0231340F02B04D058233370A0
:108060007F2301361A401F2A31D80F2A01D8412315
:1080700000E05223337053237370049C0F231A4083
:108080008C2363435149DB195B181B7F1D1C831C28
:10809000042012021B06039015431F0E741D281C9A
:1080A0000A2123F0E7FB303020700A21281C23F03E
:1080B00049FB039B013B1B0600041B0E050C0393AD
:1080C000013C002BEBD12023B371073648E0F023AD
:1080D000111C1940202905D0402903D0F02900D0D7
:1080E000ECE00EE0F0290CD053233370701C2029F3
:1080F00001D1492300E0452300210236037002919B
:1081000001E0FF2302930F23134001330593741CF6
:1081100043230025337017E004988C2343432B4AF4
:10812000DB199B18187F7B1C1B061F0E031C213BB1
:108130001B061B0E5D2B02D82070013403E0211CAE
:10814000FFF784FE023401352B0605991B0E8B4286
:10815000E2D320232370029A661C002A00D0ADE0EF
:10816000049C8C2363431949DB195B181A7F7B1C21
:108170001B061D0E1F2A5BD8081CB11C0191B91CDF
:108180000F2A29D8412333704C2328E0360101629D
:10819000EC020162345401629C870460B087046081
:1081A0003C000162CC870460D8870460E4870460E7
:1081B000E70E0162FC87046008880460148804608C
:1081C00020880460FDFF000052540162CC0E016261
:1081D0005A5401623554016252233370452373703F
:1081E000049C0F231A408C2363435B191B181B7FCD
:1081F000019C1D1C12020B0615431F0E033404269E
:10820000281C0A2123F036FB303020700A21281C5C
:1082100023F098FA731E1B0600041E0E050C013C89
:10822000002EEDD10198061C20230536037137E09E
:10823000F023111C1940202901D040292FD14523BA
:108240003370701C202901D1492300E045230370BD
:108250004323B3700F231340F41C5F1C002617E068
:1082600004998C234B436D4A5B199B18187F6B1C38
:108270001B061D0E031C213B1B061B0E5D2B02D88B
:108280002070013403E0211CFFF7E0FD02340136C9
:1082900033061B0EBB42E3D320232370661C2F1C26
:1082A0005F48331A272B09DD0D23337000237370C9
:1082B000F9F748FE5A4A202313705A4E381C009C86
:1082C000E37E834200D9B5E6554D731B012B06DDD5
:1082D0000D23337000237370281CF9F733FE0098C8
:1082E000C489077C5049281C1EF0FEF8631E1B043D
:1082F0004E4A1B0C934235D8610401D5422200E05E
:108300004622474BDA752304002B01DA422300E0B2
:108310004623434A5376464B251C161C1D400B36FC
:10832000D41D281C0A2123F0A5FA303030700A2110
:10833000281C23F007FA013E0004050CA642F0D1E8
:108340003B1C213B1B061B0E5D2B04D8F21F202378
:10835000D774137506E0FF2F04D0311C381C0C3184
:10836000FFF774FD2E48F9F7EDFD002401E0002C25
:1083700002D12B482F4901E02F49281C1EF0B4F8E8
:1083800004988C23021C5A43244B25499B181E1C1D
:108390000D3111360027002C01D1307800E07079C2
:1083A000FF2804D12D230B704B7002310DE0031C0C
:1083B000213B1B061B0E8D1C5D2B03D82023087050
:1083C0004B7001E0FFF742FD291C7B1C1B061F0EB2
:1083D000052F02D020230B7001310136052FDAD191
:1083E0000D230F4D0B7000234B70281CF9F7AAFDCD
:1083F000631C1B061C0E012CB9D90499009A01318B
:108400008C3204910092082903D076E50B4A0123AF
:10841000137006B0F0BC01BC00470000CC0E016236
:10842000345401623554016248880460FDFF000045
:10843000FF3F00006888046078880460E002016201
:10844000F0B584B00006029101920093050E281C3D
:108450001C78FBF7DDFFA04203D0002C01D00027E1
:1084600054E0281CFBF7D4FF0023A04200D10123D5
:1084700000991F1C019A4B889A4202D0002B03D00E
:1084800044E07B1C1B061F0E009B1E797F2E38D0FC
:1084900000211A1C039105321378FF2B05D0039B92
:1084A000013303930132082BF6D17E2E04D1002133
:1084B0008C46029D65441AE0B446FAE722780378B8
:1084C000013401309A4203D10131039A9142F5D32C
:1084D000039B994206D17B1C1B0680221B0E524235
:1084E000134311E001357E2E10D101218C44019AF5
:1084F0000399531A9C4509D8009C281C0534002177
:10850000E3E780235B423B431B061F0E381C04B08D
:10851000F0BC02BC08470000F0B5000684B0000EB5
:10852000009201910290154AD279171C1F4002D186
:10853000012464421CE001246442039400250026C7
:108540000123AB401F420FD00D4B0298F318019945
:10855000009AFFF775FF8023184205D09843039BCC
:10856000984201DD03902C1C01358C36082DE7D193
:10857000201C04B0F0BC02BC084700003C000162B3
:10858000CC0E0162F0B595B0CA4B0192CA4A039075
:108590001A600291C94A0021C9481CF0FDF80198EF
:1085A000027F012100230591079332E21306002B7D
:1085B00008DAF0231340F02B04D07F2301251A4062
:1085C000049501E0002604960F2A09D80599019820
:1085D00043181B7F1202151C1D430B1C0133B7E00F
:1085E000111C10390B061B0E0F2B15D8059E019D73
:1085F000AB191B7F02980A021A4303689B1A5D1E7F
:10860000331C01331B061B0E0593AE4B9D4200D855
:10861000C0E000210025C2E0F0231340202B4CD104
:108620000F2313400199059A01339C468B181B7F39
:108630001393029B039E1B6800200F932CE033785A
:10864000139DAB4226D19E4FC308DB5D072202403B
:108650001341D9071ED4059B019A1D33D418711CF0
:1086600001250EE00A7823789A4211D1944AFB083A
:108670009B5C07223A40134101340131DA0707D4E9
:108680000135654504D20F9A131A2F189D42E9D17E
:10869000654505D0013001360F9B9842CFD304E0E9
:1086A000894B984201D0051C00E0884D059B63442E
:1086B0001B061B0E614605936DE0402B4CD10F232A
:1086C000019D1340059E013302989C46AB191B7F08
:1086D0000068039F002512930E9033E03978994289
:1086E0002ED1774EEB089B5D07222A401341DA0713
:1086F00025D4059B01991D33C8180124791C0EE06F
:108700000A7803789A4211D16D4AF3089B5C0722DC
:108710003240134101300131DE0707D40134644592
:1087200004D20E9A531B66199C42E9D1644501D0CC
:10873000129B05E0644B65449D4207D105E00B1C8C
:10874000013501370E9EB542C8D3604D059B634489
:108750001B061B0E05931DE0F02B00D050E10F23EC
:108760001340544C5A1C002011E0059D01994B19EF
:10877000197F2B1C01331B061B0E0593079E544BC0
:108780009E4203D82368F154013607960130904287
:10879000EBD335E100214C4B9D4200D130E10198F3
:1087A000059A8318187F131C01331B061B0E0093B8
:1087B0000F280AD80302019E00983218127F134333
:1087C000EB18581E059B0233DEE0021C103A13061C
:1087D0001B0E0F2B13D80199009E8B191B7F02983B
:1087E00012021A4303689B1A581E059B02331B068C
:1087F0001B0E0593334B984200D8C8E06EE0F0237F
:108800000340202B66D10F2303400133019A009EC1
:10881000149393191B7F681811930299039B09689D
:108820001B180993119B0A1A0D9108923AE0099EB0
:10883000317899422FD1224FC308DB5D07220240D5
:108840001341DA0726D4009B019E099C1D33F118C1
:10885000013401260EE022780B789A4211D1184A91
:10886000FB089B5C07223A40134101310134DA07CF
:1088700007D40136149B9E4203D2089A37189642B9
:10888000E9D1149B9E4201D0119B04E0149E8319F0
:10889000581E0BE00B1C0899099A01390132089106
:1088A000099201300D9EB042C1D307481499009A35
:1088B0008B1869E0E8020162400401625101000086
:1088C000ED020162FF0F0000FFFF0000FEFF00004D
:1088D0008B0A0000402B03D0009B0593584856E0BC
:1088E0000F23034001330098019E069333181B7F2A
:1088F000681810930299039B09681B180B93109B2F
:108900000A1A0C910A9238E00B9E317899422DD1C7
:108910004C4FC308DB5D072202401341DA0724D421
:10892000009B019E0B9C1D33F118013401260EE0C3
:1089300022780B789A4211D1424AFB089B5C0722AD
:108940003A40134101310134DA0707D40136069B5E
:108950009E4203D20A9A37189642E9D1069B9E425C
:1089600001D0109B02E001380BE00B1C0A9E0B9912
:10897000013E01310A960B9101300C9A9042C3D30B
:108980002F48069E009973181B061B0E0593029A2A
:1089900013689D4234D22A4A904231D0984202D381
:1089A000581E90422CD085422AD8049B002B12D10D
:1089B000039E291C7419244D244B079A9A4205D80A
:1089C000079E23782A68B354013607960131013493
:1089D000814215D8F0E70499012911D12C1C194DB9
:1089E0001A4B079A9A4208D80723221C1A40E1081A
:1089F000012393404A5D13434B5501348442EFD920
:108A0000059E019DAB191A7F331C01331B061B0EFB
:108A1000059301980599C37E8B4200D9C6E50A49A2
:108A2000079D0A680023AB542A1C01320968039889
:108A30001BF036FE029E15B03560F0BC01BC00474D
:108A4000FFFF0000ED020162E80201628B0A0000F4
:108A5000F0B5161C1A4BD289051C0F1C9A422BD05C
:108A6000C0231B02111C1940164B141C1C40164B32
:108A70009C4221D83A68944211D9A31A480403D5DC
:108A8000317CA8181A1C07E0291CE8181BF03CFED2
:108A90003A68317CA21A281C1BF07EFE09E0944241
:108AA00007D20B04002B04DB111B4118221C1BF006
:108AB0002BFE002363553C60F0BC01BC0047000066
:108AC000FFFF0000FF3F00008C0A0000F0B584B0FB
:108AD0000D1C0021161C0090029111363278039271
:108AE0007779FF2A2CD0BA4224D0009C002301932E
:108AF0001CE0FF2F01D027700CE0019B0133934253
:108B000005D2019B611CD21A201C1BF0FDFD2B68B5
:108B1000013B2B60237803998B4203D12A68019B88
:108B20009342E6D301990131019101342B68019AF6
:108B30009A42EFD3029B013302930136052BCDD12C
:108B40002A680099002304B05354F0BC01BC0047CC
:108B5000F0B500060C1C050E002A03D12B06002BD5
:108B600000DAD2E1CE4B19788B1E1B2B00D9CCE159
:108B7000CC4A9B009B589F46CB4B1868C77E002F62
:108B800013D14379FF2B10D0821D01211378FF2BC5
:108B900004D0013101320829F8D1B6E12378013B34
:108BA0002370C14B1B685B183BE10C2934D12F2D7E
:108BB00000D8AAE1392D00D9A7E1BC4A1378002BCF
:108BC00000D1A2E1013B13702378013B2370B64B27
:108BD0001C68E17E4B1EE7183E7F0F23321C611894
:108BE0001A400B7F12021A4393009B185B005B191B
:108BF000181CAF4B3038984200DDD9E010235B429F
:108C000033403B77E37E013BE31801041A7F080CF5
:108C1000090E11431977C7E0162900D075E1A34E5C
:108C20003278002A00D170E1BA18083A8218117F10
:108C300010235B42194011773178C37E5B18083BE3
:108C4000C3180822521A197F0A431A77C37E0133C8
:108C50001B061B0EC376C3181D77D6E0281CFAF737
:108C6000DDFFFF2800D150E18F4B1B688C4A1D703F
:108C700003234CE12B1C303B1B06180E092800D99E
:108C800043E10D2920D00D2905D8042909D0072951
:108C900000D03DE10FE0132919D0192900D037E1A8
:108CA00021E07F4A06231370804A032313707E4B12
:108CB0001B6858802CE17A4A082313707A4B1A6893
:108CC00083001B185B0043E0754A122301E0744ADD
:108CD0000C231370754A03231370734B1B68DA7EE1
:108CE0009B18187714E16E4A1D2313706F4A0423F2
:108CF00013706D4B1A68D389C318D38108E12B1CFC
:108D0000303B1B06180E092800D9FEE0082918D0B0
:108D100012291FD0062900D0FAE0644A1378002BEC
:108D200000D1F2E0013B13702378013B23705E4BCE
:108D300019684A8893009B185B041B0C1B184B8016
:108D4000E6E0574A09231370574B1A681379C31882
:108D50001371DDE0554A1378002B00D1D5E0013BBB
:108D600013702378013B23704F4B1C68E27E531E27
:108D7000E618357F0F23A218127F2B401B021343E6
:108D80009A00D1184B004A4A1B18934210DC1A046F
:108D900010235B422B403377E37E013BE318197FBE
:108DA000100C120E0A431A77E37EE318187702E0DC
:108DB000404A012313703D4B1B78002B00D0A7E0E5
:108DC000E37E0133E376A3E0384E3178002900D109
:108DD0009BE0354B1868C27E5218083A8218117F02
:108DE00010235B42194011773178C37E5B18083B32
:108DF000C3180822521A197F0A431A77C37E013317
:108E00001B061B0EC376C01805773378013B337001
:108E10002378013B23707BE0214A0C231370224B03
:108E20001B685D7174E01E4A0B2313701E4B224AAF
:108E30001B6812789B185D746AE0194A0E23137040
:108E4000194B1D4A1B6812789B189D7560E0174AE4
:108E50001378013B1370124A142305E0134A137868
:108E6000013B13700E4A162313700F4B1B68DA7EFA
:108E70009B181D774CE00D490A78012A07D02B1C5E
:108E8000303B1B061B0E092B18D9002A16D023785D
:108E9000013B237000230B70034B1B681D7437E0EC
:108EA000EC020162D8C10360E40201623E04016287
:108EB0008B0A0000E0020162E1020162012A24D96A
:108EC0002F2D22D9392D20D8134E531E33702378DD
:108ED000013B2370114B1968CC89114B221C1A409D
:108EE00093009B18580043190E4A303B934208DC0C
:108EF0000D4B234003431B041B0C5B19303BCB8100
:108F000001E0002333700D7402E0084A012313705E
:108F1000F0BC01BC004700003E040162E4020162B3
:108F2000FF3F00008B0A000000C0FFFFE00201626B
:108F3000054B1B881B045B0C012098430123584000
:108F40000006000E704700000C3000E0054B1B8847
:108F50001B049B0C01209843012358400006000E7F
:108F6000704700000C3000E0024B1B8801201840C5
:108F7000704700000C3000E000B5064BDB7A002B98
:108F800005D003200421044A0023F8F7BFF901BCEF
:108F9000004700003C000162AC0D000010B50A4C17
:108FA000236800215868022200231DF0B9F82368C5
:108FB00059688B8960229343044A8B810023138074
:108FC00010BC01BC004700003474002078540162DA
:108FD000034B18880004000C4042C00F704700008B
:108FE0007854016200B5094B1B685B68994208D14F
:108FF000074A03041B0C13808B89602293438B81E7
:1090000001E01EF0B1FD02BC0847000034740020EE
:10901000785401620020704700B5184A012313609C
:10902000FFF7AAFF03200021F7F7E8FE144ACE233A
:109030005B00D35C1A0711D4124B1B78002B0DD1A7
:1090400011490868002809D1104B52331B780F22B0
:1090500013400B600E4B186001F012FC8020800062
:10906000F8F7A4FD0B4A802313800B4B1B6859684B
:109070008B89602293438B8101BC0047805401623D
:1090800038010162360101626C2301625400016201
:1090900078230162785401623474002000B5124ACA
:1090A00001231360FFF768FF03200021F7F7A6FEF6
:1090B0000E4ACE235B00D35C1A0705D40C4B1B78F9
:1090C000002B01D101F088FC8020C000F8F76EFD74
:1090D000084A81231380084B1B6859688B896022DA
:1090E00093438B8101BC00477C54016238010162CB
:1090F000360101627854016234740020064A1388F4
:109100001B04002B01D1002004E013881B04180C61
:1091100000231380704700007854016200B5FFF708
:109120003DFF054B1B881B04002B02D103F0F8F90F
:10913000F7E701BC004700007854016210B5124CFB
:109140002368002B10D0114B1A880223181C1040E2
:109150000AD10F4B52331B780E490F221340206067
:109160000B60002001F0BAFA0B490B68002B07D006
:10917000064B1A880423134002D10B6001F072FBE6
:1091800010BC01BC00470000805401620C3000E0BC
:10919000540001626C2301627C54016200B5134BE0
:1091A00000221A60124B09201A600121114AF8F7B7
:1091B000E3FB114A01210A20F8F7DEFB0F48F7F71D
:1091C000EBFDFFF7EBFE0E4B1A880223134205D18D
:1091D0000B4B1A880423134205D002E0FFF71CFF53
:1091E000F6E7FFF75BFF01BC004700008054016217
:1091F0007C540162199000609D9000603D91006078
:109200000C3000E000B5144A00231380134B0022F9
:109210001A60134B1A60134B01201A8006F0EAF90A
:1092200011490B8880221B0452011B0C13431B04A1
:109230001B0C0B800D4A0E200121F8F79DFB0C4AF8
:1092400006200021F8F798FB0A4A13200F21F8F7AF
:109250000FFB01BC0047000030130162885401621B
:109260008454016214A000E00C3000E0819400609E
:1092700005960060C8070060034B1B680020012BA7
:1092800000D101207047000084540162034B1B6829
:109290000020012B00D1012070470000885401629A
:1092A00030B5234B9A7906231A40022A09D0042AA2
:1092B0000ED0002A39D11F491F4B0A8813400B805A
:1092C00033E01C4B1A8880211204120CC90128E0DB
:1092D0001A4C0F2322881D1C154006D02388184ADB
:1092E0001B049B181B0C23801FE080202388400058
:1092F00018420BD00F4B1A8880211204120CC9019E
:109300000A431204120C1A80258005E009490A4B11
:109310000A8813400B802080084B1A881204120C14
:109320000F210A431204120C1A8030BC01BC004702
:109330003C0001620C3000E0FFBF00008C54016271
:109340000000FFFFF0B53B4B1B68012B6DD13A4984
:109350000A880423134232D0384F3948394E00244A
:1093600005E04B00DB5B1B041B0C8A005351038898
:1093700022041B04110C0134351C9342F1D80388DC
:10938000314A1B049B0B9A5103881B049B0B04332B
:109390009A512E4A0023136003881B042C4A1B0C8D
:1093A000013313602B4A244916609B002A4A9B19FB
:1093B00013600A88294B012013400B8036E00A888D
:1093C0000823134231D0264E26481E4C002505E0C6
:1093D0004B009B5B1B041B0C8A00135103882A045F
:1093E0001B04110C01359342F2D80388164A1B0462
:1093F0009B0B1A5103881B049B0B04331A51134A0D
:109400000123136003881B04114A1B0C01331360F2
:10941000104A094914609B000F4A1B1913600A88FF
:10942000114B022013400B8000E00020F0BC02BC76
:109430000847000084540162321301625465002021
:10944000905401623C130162FFFF00003813016277
:1094500048230162341301622C130162FBFF0000F8
:10946000545D00208E540162F7FF0000034B1B681F
:109470000122534058421843C00F70478454016280
:10948000F0B54F4A13881B04002B13D013884D49A5
:109490001B045B181B0C138013881B04002B09D1C1
:1094A000494B1A8880211204120C89000A431204C5
:1094B000120C1A8045490A88012313425BD0444BA1
:1094C0001B8844481B041B0C038003881B04002BCF
:1094D0004CD00388404E1B041B0CB34246D83F4B74
:1094E0001B881B041D0C3E4B1A8880235B010F1C3C
:1094F0003C4C13421AD003881B041B0C59006A1CF5
:10950000013312041B041B0C120C0A530380038842
:109510001B041B0CB34219D8334B02881B881B0455
:109520001B0C12045B1B120C1B0408E02E4B028860
:109530001B88802112041B044902120C5B18510085
:10954000013212041B0C120C0B5302802749284BCA
:109550000A8813400B80224B00221A803B881B0490
:109560001B0C042213431B041B0C3B801749214B8B
:109570000A8813400B80FFF793FE144802880823E3
:1095800013421AD1124A012313801B4BB622D20078
:109590001A801649194A023313600B88184A1B04B3
:1095A0001B0C13431B041B0C0B8003881B041B0C9C
:1095B000022213431B041B0C0380F0BC01BC0047B8
:1095C000301301620000FFFF0C4000E03213016223
:1095D0004C23016290540162FF01000004A000E0EE
:1095E0001CA000E05465002010A000E014A000E0E2
:1095F000FF7F0000FEFF0000545D00204023016259
:109600000080FFFFF0B54F4A13881B04002B13D0D6
:1096100013884D491B045B181B0C138013881B0413
:10962000002B09D1494B1A8880211204120C8900A1
:109630000A431204120C1A8045490A880223134275
:109640005BD0444B1B8844481B041B0C03800388DD
:109650001B04002B4CD00388404E1B041B0CB34250
:1096600046D83F4B1B881B041D0C3E4B1A88802399
:109670005B010F1C3C4C13421AD003881B041B0CCB
:1096800059006A1C013312041B041B0C120C0A53F0
:10969000038003881B041B0CB34219D8334B028888
:1096A0001B881B041B0C12045B1B120C1B0408E020
:1096B0002E4B02881B88802112041B044902120CC5
:1096C0005B185100013212041B0C120C0B53028068
:1096D0002749284B0A8813400B80224B00221A800E
:1096E0003B881B041B0C082213431B041B0C3B80F0
:1096F0001749214B0A8813400B80FFF7D1FD144C0A
:1097000022880423134219D1124B01201880B6225B
:109710001A4BD2001A801649194A023313600B887B
:10972000184A1B041B0C13431B041B0C0B802388BF
:109730001B041B0C03431B041B0C2380F0BC01BC4B
:1097400000470000301301620000FFFF0C4000E002
:10975000321301624C2301628E540162FF0100004A
:1097600004A000E01CA000E0545D002010A000E078
:1097700014A000E0FF7F0000FDFF00005465002002
:10978000402301620080FFFF30B5464A1368012B79
:1097900000D184E001251560434980230A681B033A
:1097A0001A4380240A6040200121E401F8F7BCF943
:1097B0000121201CF8F7B8F93C4A0023138001204E
:1097C00005F018FF3A493B4B0A8813400B803A4B8F
:1097D0000A8813400B800B881B041B0C23430B804F
:1097E0000B881B0404221B0C13431B041B0C0B8053
:1097F000324B0A8813400B8004310B88304A1B041B
:109800001B0C1340052213431B041B0C0B802D4A19
:109810002D4BD05C284209D02C4B1A881204120C14
:1098200080210A431204120C1A8004E02749284BB5
:109830000A8813400B8083070AD5244B1A8880219D
:109840001204120C49000A431204120C1A8004E09C
:109850001E49204B0A8813400B801C490B8880222C
:109860001B04D2001B0C13431B041B0C1A4A0B8055
:1098700005231380194B042252421A800C4A138884
:1098800017491B041B0C0B431B041B0C13800432D5
:1098900013881B041B0C0B431B041B0C138030BCD4
:1098A00001BC00478454016220F8FFFF32130162BB
:1098B00014A000E0FF7F0000FEFF0000F7FF0000A3
:1098C00000FFFFFF38010162A30100000C4000E02F
:1098D0007FFF0000FFFE00003013016210A000E0D7
:1098E0000080FFFF00B5FFF74FFF024A012313601E
:1098F00001BC00478854016200B50020FFF7F2FF69
:1099000001BC0047084A00231360084B1B68012B69
:1099100008D0074A074B11880B401380064B11886B
:109920000B40138070470000885401628454016228
:109930000C4000E0FFFD0000FFFB000010B51C4ADA
:109940001368012B31D1002414601A491A4A0B689C
:1099500013400B6019480021F8F7E6F8184A8023F5
:109960001B0313601548F8F721F9164B164A1C80A3
:10997000164B11880B401380154B11880B40138038
:109980001449154B0A8813400B8014490B88802218
:109990001B041B0C520113431B041B0C0B80104BAC
:1099A0001B68012B01D1FFF7A7FF10BC01BC0047CA
:1099B0008454016220F8FFFFFFFFF7FF40400000E2
:1099C00040F8FFFF301301620C4000E0FFFD000093
:1099D000FFFB000014A000E0FF7F00000C3000E05F
:1099E00088540162044A00231370044B00221A6059
:1099F000034B1A70704700003D56016238560162F1
:109A00003C56016210B51B4A002801D100241DE01C
:109A1000194B1360194B5360194B9360194BD3606A
:109A2000194B1361194B5361194B9361194BD36156
:109A3000194B1362194B5362194B9362194BD36242
:109A4000194B13630023536310E0013408CA002B41
:109A5000FBD1A100074B0A1DD018C91804E0026809
:109A60000B6808C004C101340C2CF8D910BC01BC2F
:109A7000004700009454016285330160198601603B
:109A80005152016039750160594701603D4A0160DA
:109A9000E94E0160C58C0160ED290160812C0160F7
:109AA000B14101602D3E016029A40160044A0023F8
:109AB0001370044B00221A60034B1A6070470000B9
:109AC00052230162305601622C56016210B50A4BD6
:109AD00000241C60094B1C60FFF730FF084B094A4B
:109AE0001C6013781B061B0E012B02D1064B147051
:109AF0001C7010BC01BC0047505601625C560162EC
:109B000078230162512301623601016200B511F030
:109B100027FC09F007FF01BC00470000054B1B684C
:109B2000054A002B02D0054B1B6800E0044B136074
:109B300070470000685601625C560162645601621B
:109B4000FFFF000000207047054ACD235B00D25C78
:109B5000044B01321A70044B1A60044B1A607047B0
:109B60003801016252230162305601622C560162B3
:109B7000014A00231370704734560162064B074AAE
:109B80001978074BD35C0020994200D201200123B1
:109B900058400006000E70473456016238010162D9
:109BA0009B01000000B5054B00221A60FFF764FB23
:109BB000002801D0FFF78AFF01BC00475056016220
:109BC00010B5021C0C1C002000210FE00132AD2B4F
:109BD00006D0AE2B02D0AB2B06D103E0023004E05E
:109BE000033002E0063000E0013001311378FF2B32
:109BF00001D0A142EAD310BC02BC0847F0B588B03E
:109C000002920D9A1B0612061B0E120E0391071CE0
:109C10004E490E980193009221F02CFEFA21890002
:109C200021F090FD30300006000EFA2106908900E8
:109C30000E9821F01FFE642121F084FD30300006D3
:109C4000000E079064210E9821F014FE0A2121F0E5
:109C500079FD30300006000E04900A210E9821F0A4
:109C600009FE30300006000E0025059067E00399DC
:109C70000A78131C55331B0601311B0E0391042B6C
:109C80005BD8131CAB3B042B59D8314A9B009B5823
:109C90009F460198FAF7BCFBE8554FE00E9B7C19F4
:109CA000AA1C632B05D86946097C21706B461B7D75
:109CB00001E039232370151C637040E05D23EB55F0
:109CC00000996E1C7C1903352D2907D00198FAF7ED
:109CD000B1FBF0556A461278A27030E05823F35574
:109CE0003023A3702BE07B193022EA555A70694665
:109CF000097E99706A46127FDA706946097C19718B
:109D00006A46127D06355A7119E0124B1B78002104
:109D1000012B00D10121104B1A6801234B40781907
:109D20000021002A00D101214B401B06002B01D14C
:109D3000462300E05223037000E0EA550135029B00
:109D40009D4294D308B0F0BC01BC0047102700002E
:109D500048C20360602301623813016200B50B4BF7
:109D60001B78002B04D0033B1B061B0E032B09D8CA
:109D700013F02EFD064B1A78002A01D0012002E0D4
:109D8000044B1A60002002BC084700003601016243
:109D9000962301627423016230B50F4B1B680433B4
:109DA000984215D9051F296804680B09A3420FD9E9
:109DB000031C083B1A68A023DB009A4208D9A82399
:109DC0008A185B019A4203D92C600160002000E0F0
:109DD000012030BC02BC084734130162F0B5234AAD
:109DE000234BD35C07220E1C1340041C543E072B4C
:109DF00003D1B04234D2051D33E0B04230D82DE05B
:109E0000251C08CD9A089B1A5A086368271C083736
:109E10009A4215D9A3689A4212D9E36852009A422D
:109E20000ED923699A420BD963699A4208D9A3696A
:109E30009A4205D9E3699A4202D9236A9A4210D814
:109E4000201CFFF7A9FF0128DAD10A4B9B790622D3
:109E50001340042B01D12C1C00E03C1CB442CFD396
:109E60000025281CF0BC02BC084700003801016234
:109E70009D0100003C00016230B50E4B0C1C994264
:109E800012D00D4B0D4AD25C0723151C1D4002D188
:109E9000814209D80AE0072D06D0072121F052FCA3
:109EA0002B1C43439C4201D9012000E0002030BC20
:109EB00002BC0847FFFF00009D010000380101625D
:109EC000F0B5051C696887B00291041C01CC029AA8
:109ED0000490291F904258D90968101C4908FFF7BF
:109EE000CBFF002800D1ADE00498029983088B4293
:109EF00000D2A7E0021C072101E008CCD2180139EA
:109F0000FBD2AF687B08D31AEA68944652089B1AC2
:109F100008331E095909F3005B189C190194049A2F
:109F2000029C1019984200D28CE0019A904200D90C
:109F300088E0029B7118D8198C19884200D281E000
:109F4000A0427FD860463B188B427BD3A34279D88E
:109F50002B69C2188A4275D3A24273D86A699B18CA
:109F60008B426FD3A3426DD8A86913188B4269D373
:109F7000A34267D87300CB189A19A118EA69801810
:109F800098425FD388425DD85EE00968049849082A
:109F9000FFF772FF002855D0296A049A8B080391B5
:109FA00093424FD30021092201E008CCC918013A9D
:109FB000002AFAD1AB68EF689C465B08CB1A7A0896
:109FC0009B1A08331E095C09F3001B1B98190090AB
:109FD0000399E8690A189A4234D3009B9A4231D80F
:109FE000A969331942189C1905919A422AD3A242B1
:109FF00028D82A690692D2199A4223D3A24221D89C
:10A0000060463A189A421DD3A2421BD8029B634471
:10A01000A119A34216D38B4214D8029A049BD018DC
:10A02000A0420FD388420DD86869059C22188B196D
:10A030008A4207D39A4205D8069A8018884201D3EB
:10A04000984201D9002000E0012007B0F0BC02BC1A
:10A050000847000030B5031FC91A89101A2919D9F9
:10A060000D1C1B3D041D201CFFF72AFF012812D0E8
:10A07000012D0FD9201C023DFFF78EFE0128F2D1E1
:10A08000074B9B7906221340042B01D10434EAE7E5
:10A090000834E8E70024201C30BC02BC084700005C
:10A0A0003C000162F0B581B0FFF74CF900280FD0F9
:10A0B0009D4B1B68002B0ED19C4ACE235B00D35CCA
:10A0C000C0221340402B06D1994A137801331370F4
:10A0D0000220404223E1944B1B68012B07D1934A95
:10A0E000CE235B00D35CC0221340802BECD0914B7D
:10A0F0001B789A0721D50D20F7F70AFE0D20F7F7F8
:10A1000007FE0D20F7F704FE002404E0A300985A90
:10A11000F8F752F80134884E884D32682B689B1A44
:10A120009B109C42F2D38648F7F70CFF28683368EF
:10A13000C01A8003000CF8F73FF8824B1B68142B01
:10A1400000D8E5E0804B1B78002B00D0BDE07A4BB7
:10A1500018687A4B1968FFF741FE7C4B186000289D
:10A1600000D1B2E07A4B1B78002B13D16F4B283310
:10A170001A7811231A420DD0764B1B78002B04D08D
:10A18000033B1B061B0E032B04D810F009FB002811
:10A1900000D1C3E0644B1B68002B01D109F0AAFB7E
:10A1A0006D4B00241C706D4B1C706A4B1B78002B90
:10A1B00010D0033B1B061B0E032B0BD909F0E2F852
:10A1C000002804D1664B1B78F02B00D1A6E0644B2D
:10A1D0001C7067E05E4B1978002908D05EE0009B98
:10A1E000604A99008B58800083508C5056E05E4A3C
:10A1F0001368002B03D011600020FFF703FC00223E
:10A20000584D042700922E1D7F42554A002313709B
:10A210002B68002B42D001F0E7FB831C0CD1009887
:10A2200034680130002CDAD001F0DFFB821C03D04F
:10A2300032682B6833602A6004350436002828D140
:10A24000009B002B06D0009A464B9100F858CA5844
:10A25000FA50C850374B1B78DA075FD54348F7F7F9
:10A2600071FE3F4B1878F7F7A7FF4148F7F76AFEF2
:10A27000404B1868404B1968F7F706FE3F48F7F760
:10A2800061FE3F4B1878F7F797FF0D20F7F740FD79
:10A2900044E0009B043701330093B6E7FFF75EFD0F
:10A2A00001283BD0374B9A7906231A402349274C83
:10A2B000042A01D1206801E0206804300968FFF712
:10A2C0008DFD2060002800D06AE7184B2B331B78E7
:10A2D000DA071DD51F4C2378012B19D0164B1868AF
:10A2E000164B1968FFF7B6FE184B186000280FD000
:10A2F0002378002B04D0033B1B061B0E032B07D82F
:10A3000011F0BCFA164B1A78002A07D11A4B1A60C2
:10A31000074A1378012001331370DAE6002001B0F8
:10A32000F0BC02BC0847000038130162380101622A
:10A330003C56016268230162341301622C130162EE
:10A3400088880460482301627C2301623C23016207
:10A350008423016236010162952301629423016224
:10A36000962301629454016288230162A0880460EC
:10A37000AC8804607023016274230162B8880460B1
:10A38000602301623C0001620A4B1B78012B10D153
:10A39000094B1A68012A0CD9084B18688318591EF2
:10A3A00005E002780B7803700A70013001398842A9
:10A3B000F7D3704760230162742301627023016246
:10A3C000F0B54C4B1B7885B0012B00D18CE04A4F87
:10A3D0003878F9F763FE494D84006219101C042196
:10A3E0000292FFF7EDFB2B1C7033E418061C0421CE
:10A3F000201C0394FFF7E4FB414B1A68B423921925
:10A4000012181B0104909A4201D900206DE03B789C
:10A410001B2B01D0252B35D12B1CB93BDB7F1B0619
:10A42000002B2FDA2C1C143C201C0821FFF7C8FB42
:10A43000002203E0135DAD2B02D001328242F9D33A
:10A44000824214D12C4B1878F9F728FE2B4B800050
:10A45000C418201C0421FFF7B3FB002203E0A35C17
:10A46000AD2B02D001328242F9D382420AD0244C71
:10A47000244B22681868033AC11C1AF045F9236876
:10A48000033B2360002E12D01E4C1D4D21682A680C
:10A4900088191AF039F91C4A174B127820681B7872
:10A4A00000922A6802990192321CFFF7A7FB049BD5
:10A4B000002B0FD0124B1968124B186872188018B5
:10A4C000114A0D4B12781B7800920191049A03995E
:10A4D000FFF794FB0A49049AB3180A68D218094B8B
:10A4E0000A60196800235354012005B0F0BC02BC77
:10A4F000084700009423016296230162F101016282
:10A50000742301627023016250230162014B1878A9
:10A51000704700009523016210B51B4B00241C708E
:10A520001A4B1C70FFF730F9194B1C70194B0024A3
:10A530001C60194B1C60194B1C70194B1C60194B8B
:10A540001C7010F049FD10F05DFD174A01231370D7
:10A55000FFF7DCFA01F022FD01F026FD134B1C7021
:10A56000134B1C70134B1C70134B1C70134B1C7043
:10A57000134B1C70134B1C70134B1C70134B1C7033
:10A5800010BC01BC0047000020550162215501624A
:10A5900052230162305601622C5601623D5601621F
:10A5A000385601623C560162E06F0020512301627F
:10A5B000360101621F5501621E550162CD540162D0
:10A5C000CC540162842301627C2301625323016223
:10A5D00010B5314B1B781B061B0E012B59D02F4B8E
:10A5E0001A68082A20D8012393401A1CAB231A4268
:10A5F0004FD1D30518D52A4C2368012B49D1294BBB
:10A600001B68002B45D0FFF77DF9FFF785FF02237C
:10A610002360254B1B68254A002B02D0244B1B6866
:10A6200000E0244B136034E01D4B1B68002B02D06C
:10A63000012B2ED104E01B4B1B68002B06D028E019
:10A64000184B1B68002B01D0FFF75CF9FFF75EFA8F
:10A65000154B1B68154A002B02D0154B1B6800E0F8
:10A66000144B1360FEF764FC00280AD10B4B1B68E7
:10A670000C2B01D00A2B04D10C4B1860084B18602E
:10A6800007E0074A02231360FFF746FF0A4A002348
:10A69000137010BC01BC0047512301628C2301627E
:10A6A0005056016260560162685601625C56016252
:10A6B00064560162FFFF00005323016200B5064AA1
:10A6C0001368002B05D0013B1360002B01D1FFF76D
:10A6D0007FFF01BC004700005856016270B5574B20
:10A6E0001B781B061B0E012B00D1A4E0002805D00F
:10A6F000534A00231360FFF7E9F99CE0514B1B68B4
:10A70000082B3FD801210A1C9A40151CAA231D4082
:10A7100005D1D3050DD40A4200D08CE032E0FEF71B
:10A72000ABFD494D00286DD02B78012213432B70CF
:10A7300081E0434C2368012B0FD0012B02D3022B65
:10A740001ED115E0414B1B68002B0CD0FEF794FD89
:10A75000002870D0022323606DE03C4B1B68002B67
:10A7600001D0FFF7CFF8364B00221A60384B38E0A3
:10A77000FEF782FD002801D120605CE0FFF7A6F91A
:10A78000256058E02E4E3368012B0ED0012B02D3EA
:10A79000022B4BD130E02D4B1B68002B4BD0FEF72A
:10A7A0006BFD002847D0022344E0284B1B68002B98
:10A7B00041D0FFF7A7F8FFF7A9F9264B1B682149FD
:10A7C000254A002B02D0254B1B6800E0244B136068
:10A7D0000B680C2B01D00A2B05D11F4B00221A60ED
:10A7E000174B1A6027E0164A02231360FFF794FE06
:10A7F000154A002313701EE0FEF73EFD124D00289F
:10A8000002D13060287016E02B78012213432B70A0
:10A810000C4B1B680C2B01D00A2B0CD10E4B0024C7
:10A820001C60FFF753F92C70346004E0064B0022E3
:10A830001A700023336070BC01BC004751230162D1
:10A84000505601628C2301625323016260560162FB
:10A8500058560162685601625C5601626456016294
:10A86000FFFF000000B5054BCE2252009B5C5A074B
:10A8700002D50020FFF732FF01BC0047380101621A
:10A88000F0B54B4B1B781B061B0E012B00D18BE048
:10A89000484E00233360484B1B68082B3AD80127E9
:10A8A0003A1C9A40111CAB2319407DD1D30531D5F8
:10A8B000424C2368012B18D0012B05D3022B27D142
:10A8C000FEF7DAFC00286FD13D4D2B68002B0CD031
:10A8D000FEF7D2FC002802D00223236064E0FFF7D9
:10A8E0000BF82B68276033605EE0324B1B68002B4F
:10A8F0005AD1334B1B68002B01D0FFF703F8FFF749
:10A900000BFE2E4A0223136012E02E4B13604BE025
:10A91000216049E029490B68012B26D0012B11D376
:10A92000022B3DD1FEF7A8FC002809D0FFF7EEF876
:10A93000254B1B68254A002BE7D0254B1B68E5E714
:10A94000244B18701E4C2368002B14D0FEF794FC87
:10A95000002802D0194A0223D8E7FEF7CDFF174A94
:10A9600001231360134A2368D0E7154B1B68002BA3
:10A9700001D0FEF7C7FFFFF7C9F8134B1B680F495B
:10A98000124A002B02D0124B1B6800E00D4B1360E3
:10A9900002230B60FFF7C0FD0E4A0023137003E093
:10A9A0000C4B00220A601A70F0BC01BC004700008A
:10A9B00051230162585601628C2301625056016294
:10A9C00060560162FFFF0000685601625C5601623A
:10A9D000645601625323016200B5054BCE2252003A
:10A9E0009B5C5A0702D50020FFF74AFF01BC0047D5
:10A9F0003801016230B5151C10280FD13E4B3F4A7B
:10AA00001B6813603E4B3F4A1B6813603E4B3F4A36
:10AA10001B6813603E4B3F4A1B6869E0202805D144
:10AA2000364B1868394B19683A4B1D680E2801D00F
:10AA3000092800D10820304B1860002804D0364B7C
:10AA4000994201D04A1C06D12D4A002313602E4A98
:10AA5000314B13600DE02A4A2B4C002906D1264BBE
:10AA600019602D4B00201160236002E00123136068
:10AA70002160274B1D60072829D80122131C834021
:10AA8000181CAA23184212D1104220D0234BCE22E8
:10AA900052009B5C1A0701D500292AD0FEF7F6FB6D
:10AAA000002801D0FEF72EFFFFF710F821E0144B2D
:10AAB0001B681B4A002B02D0134B1B6800E0164B8F
:10AAC0001360FEF7D9FB002801D1FFF725FDFEF743
:10AAD000D3FB00280DD00A4B1B68114A002B06D06F
:10AAE000094B196813688B4203D9116001E00A4BC6
:10AAF000136030BC01BC00478C2301624C560162DC
:10AB00006856016248560162645601624456016209
:10AB10006056016240560162FFFF00003801016289
:10AB20005C56016200B50022FFF764FF01BC0047DC
:10AB30000A4A002313700A4B00221A60094B1A704C
:10AB4000094B1A70094B1A70094B1A70094B1A609D
:10AB5000094B1A60094A0123137070473D56016280
:10AB6000385601623C56016220550162215501624E
:10AB700052230162305601622C5601626223016247
:10AB800030B54C4A1368002B01D0013B13604A4B8F
:10AB90001B68002B00D18AE0484A1378FF2B01D0B4
:10ABA00001331370464A1368002B05D0013B136034
:10ABB000002B01D108F0B6FE424A1368002B05D0E5
:10ABC000013B1360002B01D110F01CFA3E4A1368C0
:10ABD000002B05D0013B1360002B01D110F012FABD
:10ABE0003A4A1378002B01D0013B1370384A13788E
:10ABF000002B01D0013B1370364D2B78002B1ED05B
:10AC0000354C2378002B1AD0022B01D90223237054
:10AC1000324ACF235B00D05CFE280CD03049237829
:10AC20000A68D21883001B180A609A4207D9FFF7F6
:10AC30007FFF002302E02B4A002313702B70264A6B
:10AC40000023137001F0C0F9274A1378002B01D0BC
:10AC5000013B1370254C23781B061B0E012B19D1C9
:10AC6000FEF70AFB002803D1214B207018701EE06C
:10AC7000204C2378002B0AD0013B1B061B0E2370AF
:10AC8000002B14D1052003211B4AF6F73FFB32238A
:10AC900023700CE019490A68002A08D0184B9A4220
:10ACA00005D0531E0B60002B01D1FEF77BFF30BC9B
:10ACB00001BC00476C2301628C230162345601629F
:10ACC00090230162642301625C2301627C230162A0
:10ACD000842301623D5601623C56016238010162E3
:10ACE00038560162622301621F55016251230162DD
:10ACF000360101621E550162C40900005C56016202
:10AD0000FFFF000010B52E4B00241C602D4B1C6073
:10AD10002D4B1C602D4B1C602D4B1C602D4B1C6063
:10AD20002D4B1C602D4B1C602D4B1C602D4B1C7043
:10AD3000FEF768FA2C4B1C702C4B1C602C4B1C70C3
:10AD4000FFF7F6FE2B4B1C602B4B1C602B4B1C6043
:10AD50002B4B1C6010F040F910F054F9294B2A4A93
:10AD60001C7001231370FEF7D1FE284B1C70284B7A
:10AD70001C70284B1C70284B1C70284B1C70284BD7
:10AD80001C70284B1C70284B1C60284B1C60284BE7
:10AD90001C70284B1C70284B1C70284B1C60284BC7
:10ADA0001C60284B01201C60FEF72CFE2648F5F79E
:10ADB000F3FF2648F5F7F0FF10BC01BC0047000088
:10ADC0008C23016254560162585601625C5601623E
:10ADD0004C56016240560162445601624856016277
:10ADE00050560162532301623D560162385601629A
:10ADF0003C560162642301625C230162902301627C
:10AE00006C230162D4670162E06F0020512301626C
:10AE100068230162360101621F5501621E550162FD
:10AE2000CD540162CC5401626456016260560162E5
:10AE3000EC020162E2020162E00201627823016237
:10AE40005823016288230162BDA6006081AB0060C7
:10AE500010B5194B1C78194B1B78A3420FD1184B16
:10AE60001A68184B1B689A4209D11748802A00D9E2
:10AE700080220068154919F0E5FB002818D00F4B17
:10AE80001C700F4B1A680F4B10481A60802A00D9AB
:10AE900080220D4B196819F003FC0D4B00221A702B
:10AEA0000C4B1A700C4B00221A600C4B1A600120DC
:10AEB00010BC02BC084700009623016221550162C4
:10AEC000742301622855016270230162AC5501624E
:10AED0003456016252230162305601622C560162DF
:10AEE00030B5FFF7B5FF754A00231370744A137825
:10AEF00001331370734A744BD35C051C002B53D081
:10AF0000724B1B78013B092B4ED8714A9B009B5812
:10AF10009F466C4B9A7818E06A494A7AC0231A42D5
:10AF200000D0B7E0CB7A1B06002B3DDA694B1868DE
:10AF30000DF000FB012837D1ACE0624B5A7904E0F8
:10AF4000604BDA7901E05F4B1A7BC0231A4200D0D4
:10AF5000A0E029E05B4B9A7C03231A4200D199E0E0
:10AF600022E0574A002313705B4B00221A605B4BB0
:10AF70001A60012D18D15A4A13688B4214D24B1D06
:10AF8000136011E0534B18680DF0D4FA01280BD16F
:10AF9000E37A1B06002B07DB494A002313704E4B54
:10AFA00000221A604D4B1A60484B1C78272C3FD06A
:10AFB0001C2C3DD01D2C3BD01E2C39D0231C1F3BFC
:10AFC0001B061B0E042B33D93E4ACD235B00D15CFC
:10AFD000002901D1012017E0231C093B081C1B2B71
:10AFE00012D8404A9B009B589F463F4B1B68042B3E
:10AFF0000AD808E03C4B1B68082B05D803E03A4B05
:10B000001B68052B00D8481C2E4B384A9B5CDA077E
:10B0100001D4052C08D1304B1B68834238D32F4B09
:10B020001B68834204D233E0254B1B7883422FDB1D
:10B03000234A00231370284B00221A60274B1A6002
:10B040002B4B1A702B4B1B78A34211D12A4B1A6839
:10B050002A4B1B689A420BD11E48802A00D98022B5
:10B060000068274919F0EEFA002801D1022021E0FA
:10B07000204B1C70204B1A68204B21481A60802AF4
:10B0800000D98022134B196819F00AFB012011E046
:10B0900004200FE00C4B0B4CE15C154B1B788B42F2
:10B0A00000D25EE7FEF750FD084B1B78012B00D065
:10B0B0007AE767E730BC02BC084700006223016200
:10B0C00052230162380101629B0100009623016254
:10B0D0005CC2036070230162305601622C5601622B
:10B0E0005C56016284C20360542301629F01000028
:10B0F00034560162205501627423016224550162B5
:10B100002C550162F0B5BC4C237881B0061C002B95
:10B110004AD18368F02B1DD10068B8491BF0A0F913
:10B12000002800D0FAE1B64B01221A70B54B187016
:10B13000B54B2270B54A187032231370B448316889
:10B140001BF0D2F9B34A02231370B34A142301242B
:10B150001370E9E1F12B1DD14568042D00DCDBE122
:10B160000468A64F201C391C02221BF043FA002859
:10B1700000D0D1E160190238391C02221BF03AFAE2
:10B18000002800D0C8E12B1F7360E3189870306866
:10B19000023003E0F22B00D0C0E10068FBF718FB9F
:10B1A000002800D1BFE1B7E1FEF766F8002801D121
:10B1B0002070B3E1B268F02A00D058E17768012F1F
:10B1C00000DCAEE1042F00DDABE1934C2378002BD3
:10B1D0000BD0904B1B78BB4207D18D4930683A1C8D
:10B1E0001BF008FA002800D13EE1022F23D130687D
:10B1F000824902221BF0FEF9041C00281BD17E4D5F
:10B200002B78072B07D1854B187802F0F1F9012331
:10B210002B707C4B1C707A4B1C707C4B7E4A1C70D4
:10B2200014232C7013707A4831681BF05DF9794B48
:10B2300002241F7078E1704A1378033B1B061B0E33
:10B24000012B01D8012313701378053B1B061B0E3D
:10B25000012B0CD8724B1B78002B06D07368032B84
:10B2600003D133681B78242B01D001231370624B68
:10B270001A78012A00D1DAE07168072A70D0022911
:10B2800005D003295FD133681B78242B5BD1082AB2
:10B2900059D03368022903D118785978002202E086
:10B2A000587899780122F8F783FB431C09D1736819
:10B2B000022B48D1336818785978F8F731FC431CD1
:10B2C00041D04D4B1A78131C0B3B1B061B0E012B58
:10B2D00017D8534B1B78002B01D1012040420B2A79
:10B2E00005D1504BC25C07231A4227D009E00C2A33
:10B2F00007D14C4BC25C44231A421FD0930700D5A0
:10B300002038431C1FD00006000EFAF7C3FF444A42
:10B310001378002B00D198E0013B1B061B0E137025
:10B32000002B00D091E0344A13780B3B1B061B0E18
:10B33000012B00D889E00123137086E0013000D092
:10B3400081E0032400E005242B4A13780B2B01D164
:10B350000D2369E00C2B01D10E2365E0012363E08E
:10B36000284B1A786B4603331A70022904D13368CC
:10B3700018785978002208E003292FD13268137811
:10B38000242B06D1507891780122F8F711FB431C49
:10B3900009D17368022B1AD1336818785978F8F7F5
:10B3A000BFFB431C13D06C4603340006211C012252
:10B3B000000EFDF7CDFB134B22781B7812499A4201
:10B3C00003D10B78002B3BD131E00B7836E073686A
:10B3D000032B03D130680378412B29D00F4B187809
:10B3E00002F006F9084B0021034A1970012313707B
:10B3F000044B19701BE0000036010162CC88046028
:10B4000051230162EC020162E00201621E550162F9
:10B41000CD540162CC5401621F550162E202016207
:10B4200061230162F06D04601370052C0ED1306849
:10B43000F8F778FC002803D13E4B1B78002B04D092
:10B440003C4A00231370032400E004243A4A3223C8
:10B4500013703A4A14231370394831681BF044F8CA
:10B46000384A736813705FE01423237059E023781F
:10B47000033B1B061B0E032B53D8C0231340402B4A
:10B4800006D13F2313401B2B02DD00F093FD48E063
:10B49000FFF726FD022802D0042803D141E00FF077
:10B4A000B1FD3EE00FF0AEFD307AF8F74DFF002819
:10B4B00002D17368FD2B03DD1F4A322313702BE08A
:10B4C000214C2378052B05D1204B307A1978F8F7D9
:10B4D000B7FB1DE0062B05D11C4B307A1978F8F725
:10B4E000BFFB15E0032B04D1184B1878F8F7C8FB05
:10B4F00006E0042B0CD1154B307A1978F8F7E0FDF3
:10B50000013005D10C4B32221A700123237003E065
:10B51000094A3223137006E0032405E00124644243
:10B5200002E0052400E00424201C01B0F0BC02BCB1
:10B5300008470000E00201621E5501621F550162CA
:10B54000CD540162CC540162360101628023016254
:10B55000F0B587B00490FEF7A5FD00282BD1B54AC1
:10B56000137801331370B44B1B78002B2AD1B34BE3
:10B570001B7810331B061B0E022B23D81020002132
:10B58000FFF7D0FAAE4B1B680B2B0AD1AD4BAE497F
:10B5900018680B221BF02EF8002802D102F0A4FF3D
:10B5A00009E0A84B186803F009FC012806D1202007
:10B5B0000021FFF7B7FA01204042FBE1A34B9B7942
:10B5C000D807F8D5A24AA34B9B5CA3499B4A5807CE
:10B5D00009D59B4B1B680B6013780A2B06D19F4B38
:10B5E0001B68023301E09D4B1B680B60934B1A787C
:10B5F000C0231340402B14D13F2313401B2B10DDDD
:10B6000000F0D8FC964B1B68012BD4D9954B1B68D6
:10B61000954A002B02D0954B1B6800E0944B1360B9
:10B62000C9E704990029C6D0924A01231370924BAE
:10B6300000211960824C834B22681B68D154FEF7AD
:10B6400065FA04982268C3689A42B4D37A4B1B788F
:10B65000002B07D1794B18787F4B1968FAF726FF32
:10B660000028A8D0049A216813699942A3D8834B73
:10B670001B78002B01D1824A00E0824A1368013313
:10B6800013606D4B1B78002B0ED0049B18686D4B1C
:10B690004A1C196819F004F8684B04981B788360F9
:10B6A000674B1B68436084E1FFF71AFC022804D053
:10B6B000042880D001283BD11DE0694B196806237E
:10B6C0000B40042B07D0634A022B07D1CE235B002B
:10B6D000D35C1A0707D50FF095FC6CE7CE235B000F
:10B6E000D35C180724D40A0718D55F4B1A68604B3F
:10B6F0009A421DD112E05A4B1A6806231A40042AB6
:10B7000007D0022A0AD1534BCE2252009B5C180765
:10B7100004D55D4B1A7802218A431A70514B1B687D
:10B72000514A002B02D0514B1B6800E0504B136074
:10B730000FF068FC414C2278131C10331B061B0EC3
:10B74000022B00D8F2E0424B424AD25C03231A405B
:10B75000022A0AD0032A0FD0012A13D1394B1868C4
:10B76000374B1968F8F73AFC0CE0364B1868344B45
:10B770001968F8F71BFC05E0324B1868304B196864
:10B78000F8F744FC334C324D635D190704D52D4B5B
:10B790002B491868F8F752FC635DDA0604D5294B8B
:10B7A00027491868F8F766FC00F040FB002802D132
:10B7B000224B1870C1E0322000F018F91F4A204EC9
:10B7C000013004D10023137000233360F3E61D4DD4
:10B7D000107829683268FF23FCF79EFE07281CD8E2
:10B7E0008C23021C5A43294B294CD218226028680A
:10B7F000311CFCF7C7FE28682268311CFDF766F98A
:10B8000028682268311CFDF723F93368002B41D1E9
:10B810000E4B1B7A98073DD406E00C4B1B7AD907D8
:10B8200038D59A0700D5C6E60220F5F715FEF5F7DC
:10B83000BFFFC0E63C5601623601016296230162F9
:10B840007423016270230162D08804603C000162AD
:10B8500099010000380101628023016254230162D2
:10B860008C230162685601625C5601626456016273
:10B87000FFFF00003D5601623856016260230162FD
:10B88000305601622C56016253230162CC0E0162D4
:10B89000E4020162FEF794FD002800D18BE6474BDD
:10B8A0000821181C0393FEF78BF90821071C444854
:10B8B000FEF786F90690434804680699E219B42316
:10B8C00052181B0102909A4200D974E67A18059228
:10B8D000002A38D0002F05D03B4B1968221CC8190C
:10B8E00018F012FF394D384C2A78394E20683378D9
:10B8F000029900920A68039901923A1CFEF77EF9B8
:10B90000029A116820682A787B18C0183378009250
:10B910000191069A2A49FEF771F902980599036880
:10B920005B182168002203605A540CE0F22A0AD105
:10B9300000F07CFA002803D12070224B18603AE610
:10B940000E235B4223701F4C0498226803699A42BD
:10B9500000D930E61C4B01321968006818F0A0FECF
:10B960001B4B04991B788B60049A21685160126804
:10B9700000238B54174B1B781B061B0E012B00D189
:10B9800019E6154B51331A7814493F231A400B68B6
:10B99000934200D20A60124BCE2252009B5C1807E1
:10B9A00007D4104B1B6806221340022B01D1FEF76F
:10B9B0008DF8002007B0F0BC02BC0847DD01016231
:10B9C000E501016274230162702301625023016268
:10B9D0009623016251230162540001626C230162CB
:10B9E000380101628C23016218472047F0B5924B61
:10B9F0001A78131C1B3B88B0061C082B4FD88F4AA3
:10BA00009B009B589F468E4B2B331B782CE008F0F5
:10BA1000ABFB302804D08A4B2D331B781A077FD517
:10BA2000884A002300201370E9E1874B18680278E8
:10BA3000302A04D0824B2D331B781C070DD5804B48
:10BA400028331B78590665D4804C2268411C01328A
:10BA500018F05AFE2368013B5BE0101C60E0784B55
:10BA60002D331B781A070DD55C0714D4774C764B11
:10BA7000226818680132411C18F046FE2368013B19
:10BA8000236008E0704B1B68187849E06C4B2B333F
:10BA90001B78190743D56B4A002313709BE1C02321
:10BAA0001340402B01D0802B34D1530601D5022600
:10BAB00000E00526664C0421201C0694FEF780F861
:10BAC000071C002826D0614A5F4C136821689B1B25
:10BAD000181805920818321CC91818F015FE059B95
:10BAE0001D68AB1B5B4E20683178C018F324524BA5
:10BAF00021403A061B78120E0091ED190699019526
:10BB0000FEF77CF83378032293433370059C236857
:10BB1000DB1923604B4A0023012013706FE13020B2
:10BB20004A4B1A68C8235B009A4200D953E1454C3E
:10BB30002178002900D193E0474D2B68002B78DD58
:10BB40003D4B1A788A4208D13F4B444918681AF095
:10BB500087FC002828D12E604FE1131C223B1B06D6
:10BB60001B0E012B19D80B1C1B3B1B061B0E032B9A
:10BB700058D81C2902D1322875D00BE01D2902D1DA
:10BB800033284FD16FE01E2904D01B294AD1E36826
:10BB9000312B47D1342866D044E0202A07D11B2915
:10BBA00002D1E368322B5ED0002323705BE0131CCC
:10BBB0001C3B1B061B0E022B17D80B1C223B1B0623
:10BBC0001B0E012B2ED81C2A03D1E368322B4FD039
:10BBD00008E01D2A03D1E368332B23D148E01E2A55
:10BBE00020D1E368342B43D01CE01B2A1ED10B1C50
:10BBF000203B1A06130E032B14D8131601229A4069
:10BC00000D231A420ED00B1C223B1B061B0E012BD0
:10BC100004D8312802D1E368342B29D0202901D15E
:10BC2000322820D0074A002313701AE00023237023
:10BC3000D1E00023237014E096230162F4C2036074
:10BC4000380101626C560162702301627423016243
:10BC5000ED01016250230162805601628456016247
:10BC6000E060F5F78DFD68480178002900D1B4E067
:10BC7000664B65481A684468B4231219023A1B01DE
:10BC80009A4200D9A5E00B1C1C3B1B061B0E022B85
:10BC900004D85F4B28331B785A060AD50B1C223B6D
:10BCA0001B061B0E012B0DD8594B2D331B78590742
:10BCB00008D45848621C411C18F026FD524A5368AB
:10BCC000013B5360544B1A78131C1C3B1B061B0E84
:10BCD000022B04D84E4B28331B785C060AD5131C64
:10BCE000223B1B061B0E012B0FD8494B2D331B7813
:10BCF00059070AD4454C494B226818680132411C47
:10BD000018F002FD2368013B2360454A0421101C02
:10BD10000492FDF755FF404B03931B781B3B1B061A
:10BD200004061B0E0790384E3C4D384F0294032BEF
:10BD300019D83B6872681B1828680132C018354949
:10BD400018F0AEFC02990A0E71783C6828683378C6
:10BD50000091716800196418079964180499019496
:10BD6000FDF74CFF24E0079A7068296880183A684C
:10BD70000818013218F0C8FC28682649726818F0C3
:10BD80008FFC2868029B0399264D1A0E0B782978A0
:10BD900074680091396800190919079C0919019103
:10BDA0000499FDF72BFF337803990B7073782B7090
:10BDB0001C4B30221A70184A13781B2B01D12523F3
:10BDC000137011481149079B4268D2180B689B18E1
:10BDD0000B6000230370022011E00F4B1B780370EF
:10BDE000104B1B784370094B1A680C4B4260196862
:10BDF000084818F055FC0C4B1E600120404208B06A
:10BE0000F0BC02BC084700006C560162742301625A
:10BE10003801016284560162962301627023016237
:10BE2000ED0101625023016280560162F0B5534A70
:10BE3000137881B0492B15D0492B07D80D2B15D07D
:10BE40000E2B0CD0092B00D093E00BE04E2B06D02C
:10BE5000F22B02D04D2B09D08BE00E231370484BF0
:10BE6000013305E0464B1A7C202303E0444B0233A8
:10BE7000DA7F02231A4002D1424B1A7079E041481E
:10BE80000178002905D03D4B1B78402293438B421B
:10BE900001D0002343603C4B3A4C1E686568C823C0
:10BEA000AA195B009A4204D9F5F782FC002323709B
:10BEB0004DE0002D23D0A268AB1AB3421FD1334806
:10BEC000334B10181968321C18F0BCFB002816D12F
:10BED000304B1B68002B12D0284B1B785A060ED50E
:10BEE000274ACF235B00D25CFE2A02D101225242B4
:10BEF00002E093009B185A10264B1A6027E0234B50
:10BF0000E818234D321C2968009318F0C9FB1D4C1A
:10BF10001D4F63683A68A3609B186360174B1978DC
:10BF200040230A1C9A430E1C22701E4011D0144A52
:10BF3000CF235B00D25CFE2A02D10122524202E0F2
:10BF400093009B185A10134B1A60F5F719FC002048
:10BF500010E00E2903D1104A13780433137062687D
:10BF60002868009918F09CFB62682B683A60D654E8
:10BF70002670012001B0F0BC02BC08479623016284
:10BF8000380101626C5601627423016284560162B9
:10BF9000702301627C56016250230162014A002332
:10BFA000137070476C560162014A0023136070479A
:10BFB00080560162034A1368002B01DD32231360AF
:10BFC0007047000080560162034A1368002B01DDB0
:10BFD000013B13607047000080560162034B002252
:10BFE0001A60034B1A60034B1A6070474C58016289
:10BFF000245801622058016200B5034B18600348C1
:10C00000F4F7CAFE01BC00471458016239C200604F
:10C0100070B5494C22680006000E012A19D0012A89
:10C0200002D3032A59D143E04449102803D10B68B5
:10C03000012253401BE00B68002B52D000220A6003
:10C0400002284ED1012323603D4B1A603D4A122342
:10C0500041E03C4D2B6843402B60384910280AD101
:10C060000B68012B05D100230B6019E023600B60E6
:10C0700037E00A6035E00B680E1C002B10D0002161
:10C080003160022802D0032808D105E02C4B226041
:10C09000196012232B6024E0206022E0216020E060
:10C0A000274D2A680E2AE1D8274BD054531CF1E7BC
:10C0B000244B1B68834209D003280AD1204B1B68FC
:10C0C000012B06D1204B1B78002B02D105232360C6
